:020000040800F2
:1080000000800120A96B0208792B02087B2B020853
:108010007D2B02087F2B0208812B02080000000044
:10802000000000000000000000000000832B020898
:10803000852B020800000000872B020801A301081D
:10804000ED6B0208ED6B0208ED6B0208ED6B0208A8
:10805000ED6B0208ED6B0208A9C4010801C5010817
:10806000ED6B0208ED6B0208ED6B0208ED6B020888
:10807000ED6B0208ED6B0208ED6B0208ED6B020878
:10808000ED6B0208ED6B0208ED6B0208ED6B020868
:10809000ED6B0208ED6B0208ED6B0208ED6B020858
:1080A000ED6B0208ED6B0208ED6B0208ED6B020848
:1080B00041D00108ED6B0208ED6B0208ED6B020880
:1080C000ED6B0208ED6B0208ED6B0208ED6B020828
:1080D000ED6B0208ED6B0208F9B70108A5B40108C1
:1080E000ED6B0208ED6B0208ED6B0208ED6B020808
:1080F000ED6B0208ED6B0208ED6B0208ED6B0208F8
:10810000ED6B0208ED6B020859C50108ED6B020822
:10811000ED6B0208ED6B0208ED6B0208ED6B0208D7
:10812000ED6B0208ED6B0208ED6B0208ED6B0208C7
:10813000ED6B0208ED6B0208ED6B0208ED6B0208B7
:10814000ED6B0208ED6B0208ED6B0208F5AD01085E
:10815000ED6B0208ED6B0208ED6B020829B2010815
:10816000ED6B0208ED6B0208ED6B0208ED6B020887
:10817000ED6B0208ED6B0208ED6B0208ED6B020877
:04818000ED6B020899
:1081880010B5054C237833B9044B13B10448AFF349
:1081980000800123237010BDE00E002000000000C5
:1081A800249B020808B5034B1BB103490348AFF3EE
:1081B800008008BD00000000E40E0020249B020897
:1081C80038B5064C05462368C31AB3F5FA7F04D3BD
:1081D800034B9B699B699847256038BDFC0E0020BE
:1081E8007086020810B514F0D9F90022054B1A70F0
:1081F800054B1B689847BDE81040044B9B695B69B9
:10820800184700BFCC090020A8000020708602088B
:10821800431E2DE9F0471446052B00F22081DFE8C4
:1082280013F006000C000C004E007800CE00FFF79B
:10823800D9FF47F6A85323603FE08F4B8F4D0228A4
:1082480016BFA94699461D464FF0FF364FF0000865
:108258004FF0010A8A4BA9F10409DF68043D3B6825
:10826800D9F804001B6998473B686868DB68984739
:108278003B6855F8040F5B6998473B6859F8040F49
:108288005B6A984718B90AFA08F326EA03063B68B6
:1082980028689B6998473B68D9F800005B6A98474B
:1082A80018B10AFA08F326EA030608F10108B8F13A
:1082B800110FD4D1C6F310062660002030E02160EB
:1082C80003292CD8DFE801F0021A1E226C4BDB6967
:1082D8001B6818881DF06AFD63A3D3E900231DF00D
:1082E800F9FE63A3D3E900231DF0CAFD0022654B04
:1082F8001DF0C6FD1DF0D6FF2060DEE7604BDB6990
:108308005B68E6E75E4BDB699B68E2E75E4B1B69EF
:1083180091E70129216021D004D3022934D0022019
:10832800BDE8F087564BDC68D4E900309B68203004
:108338009847D4E90030DB683C309847D4E90030EE
:10834800DB6858309847D4E900305B693C3098477F
:10835800D4E900305B6958309847AEE7484BDC6891
:10836800D4E900309B683C309847D4E90030DB689A
:1083780020309847D4E90030DB6858309847D4E972
:1083880000305B692030E2E73D4BDC68D4E900301F
:108398009B6858309847D4E90030DB68203098470C
:1083A800D4E90030DB683C309847D4E900305B6999
:1083B80020309847D4E900305B693C30CCE701298C
:1083C800216036D01BD30229A9D12D4BDC68D4E912
:1083D80000309B6858309847D4E90030DB6820307B
:1083E8009847D4E90030DB683C309847D4E900303E
:1083F8005B6920309847D4E900309B69DDE7204B62
:10840800DC68D4E900309B6820309847D4E9003014
:10841800DB683C309847D4E90030DB68583098472F
:10842800D4E900305B693C309847D4E900309B6957
:1084380091E7134BDC68D4E900309B683C309847DF
:10844800D4E90030DB6820309847D4E90030DB6895
:1084580058309847D4E900305B692030E4E70420BD
:108468005EE700BFAFF300800000000000FEAF40F1
:10847800AAF1D24D62101440F0610020BC600020C7
:108488007086020800002440CC0900203B4B3C4A7F
:10849800DB685B6803F5B871116003F1AC015160EA
:1084A80003F1E401916003F58E71D16003F5AA71BF
:1084B800116103F5D471516103F5F071916103F510
:1084C8000671D16103F51471116203F522715162CD
:1084D80003F53071916203F53E71D16203F54C7179
:1084E800116303F55A71516303F56871916303F5DC
:1084F8007671D16303F582611164224A03F1740134
:10850800116003F19001516003F1C801916003F516
:108518008071D16003F59C71116103F5C6715161D9
:1085280003F5E271916103F5FE71D16103F50D71F7
:10853800116203F51B71516203F52971916203F50C
:108548003771D16203F54571116303F553715163B6
:1085580003F56171916303F56F7103F57D7313641E
:10856800D1630122084B1A70084B094A1A65094A57
:108578009A65094A5A651AF077B900BF70860208E9
:10858800BC600020F0610020CC09002000610020C0
:1085980019820008ED810008C9810008704702208F
:1085A80070470220704770477047022070470220CA
:1085B80070470220704701207047704702207047BB
:1085C80070474369134A10B5C3F80422C3F8082258
:1085D800114B12498365124B124AC0E9091312491B
:1085E8008361C0E90B13C361104B114C4364114BF9
:1085F80042658364104B84634363C0E90F330F4BB8
:10860800C0E913140366002383660D4BC265C0E9F5
:108618001B3310BDBF850008A5850008A785000885
:10862800AB850008C9850008B3850008AF85000838
:10863800BB850008B1850008B7850008C385000818
:10864800C5850008704700BF0022012110B44FF013
:10865800FF340848084B80F884205A7083F81012B9
:10866800C0E91F41C0F8883082671A70743010BCA6
:10867800FFF7A7BF006100200C0F002000234FF078
:10868800FF314FF0010C064A06481370537082F808
:1086980010324261C0E9021C03744360FFF791BFC6
:1086A8002C110020006100200023184610B5064C4C
:1086B8001A5D590002F0030201338A40072B40EA91
:1086C8000200F5D110BD00BF4C130020002304495F
:1086D8005A5C02F00302C2540133072BF8D17047E9
:1086E8004C130020074B1A7802705A7842709A7817
:1086F8008270DA78C2701A7902715A7942719B795C
:10870800837170474C130020F8B50024084B094FBB
:10871800094EDD68E15D726C2B6852F82400DB6954
:1087280001F0030101349847072CF3D1F8BD00BFCD
:10873800708602084C130020000000200023054A20
:1087480000F0030199540133072B4FEA9000F7D149
:10875800DAE700BF4C130020014B586AEEE700BF70
:108768000000002000230449C25C02F003025A54AE
:108778000133072BF8D1C7E74C1300200278074BC9
:108788001A7042785A7082789A70C278DA700279D0
:108798001A7142795A7182799A71B5E74C1300209F
:1087A8000022014B9A6770470061002010B503480A
:1087B800144615F0B4FA206010BD00BF7C130020E9
:1087C80010B50F4C0146204615F018FB002014F098
:1087D8006BFD6F21204615F0A2FAC0F3006100205E
:1087E80014F034FD012014F05FFD7F21204615F0C0
:1087F80096FABDE81040C0F30061012014F026BDD0
:108808007C130020014815F07CBA00BF7C130020BF
:10881800012808B503D814F08BFC002008BD0820F7
:10882800FCE7012808B503D814F060FC002008BD57
:108838000820FCE70021F4E74942F2E7F1E70148A4
:1088480015F0C3BA7C13002038B5002014F0B4FD2D
:1088580008B1002038BD012014F0AEFD05460028FF
:10886800F7D10C4C204615F09BFA14F01DFE2B4650
:10887800D4F88C22D4F88412284614F0BDFC0120C8
:108888002B46D4F89022D4F8881214F0B5FC0120B5
:10889800E0E700BF7C130020022804BF0C4B93F8CC
:1088A800E80038B90B4BDB681B685B690A4AD2F8E9
:1088B80094021847012809D1054B93F8E830012B99
:1088C80004D1044BDB681B689B69EFE7704700BF66
:1088D80000610020708602087C13002070B500201B
:1088E800FFF7DAFF0C4B0D4CDD68D4F894022B68C7
:1088F8009B6898472B68D4F8A4029B6898472B6814
:10890800D4F8A8029B68984714F042FEBDE870406E
:10891800034B5B68184700BF708602087C13002071
:10892800780900200346052B10B5084614460BD0DD
:1089380006D8022B06D314F093FD2060002010BD4A
:10894800182BF8D00420FAE714F098FDF5E7012871
:1089580038B504460D4605D820B914F02DFD286019
:10896800204638BD0820FCE7022810B5144611D06F
:10897800032817D0012819D10D4B0E4ADB68D2F80D
:10898800A4021B685B6A9847003018BF012020606A
:10899800002010BD064B074ADB68D2F8A8021B6806
:1089A8005B6AF0E7084614F003FCF0E70420F0E700
:1089B800708602087C130020012838B504460D464D
:1089C80008D814F0DDFC2B68C11829602046BDE8E2
:1089D80038401DE7082038BDA32A2DE9F041054697
:1089E8000C461E4600F090814BD8072A00F0EC8018
:1089F80024D8032A00F0BD800BD8012A00F0AA80F1
:108A080040F29A80002840F0AF80084614F0E2FC5B
:108A180096E0052A00F0C08040F2B180202101FADA
:108A280004F444F01004E4B22146B648002D40F0A6
:108A3800BD8015F074F9C0F3042081E0322A00F0FB
:108A4800F2800FD81C2A00F0D5801D2A00F0E7809C
:108A5800082A59D1002857D1084614F0A9FBC0F3B9
:108A680000106DE08C2A00F0ED80A22A00F035811C
:108A7800332A49D1002840F0E080084614F0F0FC81
:108A88005EE0AB2A00F0F88132D8A72A4FEA011439
:108A980000F0B6811AD8A52A00F05F8140F249811A
:108AA80044F06C04E4B22146964815F038F92146A2
:108AB80000F48040002D40F09681002800F08D8160
:108AC800904815F02CF9C0F3021039E0A92A00F0FB
:108AD800B68140F2A18144F06D04E4B22146894890
:108AE800002D40F0C08115F01AF9C0F3032027E0EB
:108AF800B32A00F0138209D8AD2A00F0DE81C0F055
:108B0800D081AE2A00F0EE81042520E0B52A00F0DD
:108B18002782C0F01882B82A00F02C82CE2AF3D11E
:108B28000028F1D1090141F06F01C9B2754815F06B
:108B3800F6F8C0F3090003E020B9084614F02EFC4B
:108B4800306004E01968204614F0F2FA002528463F
:108B5800BDE8F08118B9084614F012FCF0E719686E
:108B6800204614F0BFFBF1E71968204614F0BEFA5E
:108B7800ECE70028C8D1084614F01EFCE0E718B955
:108B8800084614F043FCDBE7196820460029B8BF03
:108B9800494214F0C1FBD9E718B9084614F028FC7B
:108BA800CEE71968204614F01AFDCFE715F0B7F89C
:108BB800336820F4F8521B0203F4F8531A43214691
:108BC800504815F09EF8C1E7202101FA04F444F05A
:108BD8001004E4B221464B4825B915F0A0F800F07E
:108BE8001F00ADE715F09BF8336820F01F0203F073
:108BF8001F03E3E70C0144F06C04E4B2214641484A
:108C080025B915F08CF8C0F3804099E715F087F87E
:108C1800336820F480229B0403F48023CEE70028E5
:108C28007FF472AFA8E718B9084614F00BFC87E781
:108C38001978204614F08AFB88E71968204614F052
:108C480095FB83E750B9090141F06C0101F0FC0183
:108C58002C4815F064F8C0F3036071E71B68102B0B
:108C680035D00DDC022B2ED004DC012B16D04FF0B2
:108C7800FF3314E0042B28D0082BF8D105230EE08D
:108C8800402B26D003DC202BF1D1032307E0802BD7
:108C980021D0B3F5807FEAD1002300E008233360B8
:108CA800336801333FF452AF240144F06C04E4B25A
:108CB8002146144815F033F8336820F070621B061B
:108CC80003F070637AE70723E9E70623E7E704235D
:108CD800E5E70223E3E70123E1E70C0144F06C0434
:108CE800E4B22146074825B915F019F8C0F3C13098
:108CF80026E715F014F8336820F4C032DB0303F4D8
:108D0800C0335BE77C1300200C0144F06C04E4B230
:108D18002146A34825B915F002F8C0F380300FE7C3
:108D280014F0FDFF336820F480429B0303F4804372
:108D380044E744F06C04E4B22146994825B914F09C
:108D4800EEFFC0F30030FBE614F0E9FF336820F4CF
:108D580080521B0303F4805330E744F06C04E4B200
:108D680021468F4814F0DBFF2146804600F48047F7
:108D78008B4885B927B114F0D2FFC0F3C310DFE6E2
:108D880014F0CDFF18F4006FC0F3021018BF40F0C4
:108D980008003060DAE647B114F0C1FF336820F408
:108DA800F062DB0103F4F06308E714F0B8FF3268FF
:108DB80020F07000120102F0700202432146784848
:108DC80014F09FFF2146764814F0A9FF336820F479
:108DD80000621B0203F40063F0E6714814F09FFF81
:108DE800C0F3C310D5E748B16D4814F098FF336855
:108DF80020F070021B0103F07003DFE66848CBE740
:108E080044F06C04E4B221466548002D4DD114F0BD
:108E180086FF00F00F0093E644F06D04E4B22146AB
:108E28005F4825B914F07BFFC0F3C03088E614F022
:108E380076FF336820F40042DB039BB2BEE644F0C1
:108E48006D04E4B22146564825B914F068FFC0F312
:108E5800413075E614F063FF336820F4C0425B03C9
:108E680003F4C043AAE614F05AFF336820F4706292
:108E78001B0203F47063A1E60C0144F06D04E4B234
:108E88002146474825B914F04AFFC0F3411057E678
:108E980014F045FF336820F060025B0103F06003C3
:108EA8008CE60C0144F06D04ACE714F038FF33682D
:108EB80020F00F0203F00F0380E60C0144F06D046C
:108EC800E4B22146364825B914F029FFC0F3006002
:108ED80036E614F024FF336820F080721B0603F096
:108EE80080736BE60C0144F06D04E4B221462C4813
:108EF8005DB914F014FF001400F07F0310F0400077
:108F080018BF6FF07F0018431AE614F008FF3368A3
:108F180020F4FE021B0403F4FE034FE60C0144F0A8
:108F28006C04E4B221461E4825B914F0F8FEC0F3DB
:108F3800404005E614F0F3FE336820F400325B0489
:108F480003F400333AE600287FF4DEAD090141F06E
:108F58006F01C9B2124814F0E2FEC0F30440EFE515
:108F680018B9084614F060FAEAE51968204614F0C2
:108F7800DFF9EBE50C0144F06C04E4B22146084843
:108F880025B914F0CCFEC0F34030D9E514F0C7FE83
:108F9800336820F400525B0303F400530EE600BF6D
:108FA8007C13002007B50129019207D8024601ABBE
:108FB8000120FFF711FD03B05DF804FB0820FAE774
:108FC8000129134602D80246002005E5082070470B
:108FD800022806D3052801D9182802D100201060DC
:108FE800704704207047034B0846D3F8B032114647
:108FF800DB6818477C1300202DE9F0415B4C5C4D81
:109008005C4F0121D4F8882028465B4B14F0ACFE55
:10901800FE68736803F1C802C5F8942203F59C72D0
:10902800C5F8A82203F5AA72C5F8A42203F5C672EA
:10903800C5F88C2203F5D47203F5B870C5F88822F8
:1090480003F5E27203F50D73C5F8AC323368C5F861
:109058009022DB68C5F8840298473368D5F88C02FB
:10906800DB6898473368D5F88802DB689847336827
:10907800D5F89002DB6898473368D5F89402DB6826
:1090880098473368D5F8AC02DB6898473B6903F129
:109098001402C5F8B022D5F8AC229A6114F004FA8B
:1090A8000023D5F88C22D5F88412184614F0A4F8B9
:1090B800D5F88812D5F890220023012014F09CF8E6
:1090C800D4F888302D4A0025C3F804222C4A5D7054
:1090D800C3F8082201221A702A4B3222C4F89430AD
:1090E800294B0220C4F89030284B84F88400C4F837
:1090F8008C30274BC4F89830264BC4F8AC30264B3C
:10910800C4F8A830254BC4F89C30254BC4F8A030CF
:10911800244BC4F8BC30244BC4F8B830234BC4F8F3
:10912800C830234BC4F8C430224BC4F8C030224B9B
:10913800C4F8D430214BC4F8D0304FF48F73C4E94D
:109148001F321F4BC4F8CC301E4BC4F8E0301E4B06
:10915800C4F8E4301D4CFFF79FFB23689847A368C9
:1091680029462846BDE8F041184700BF00610020A5
:109178007C13002070860208486E02085188000897
:10918800478800082B88000845880008418800089F
:109198003D880008C98F0008AD8F000819880008AD
:1091A800C18900080D880008B5870008C98700082C
:1091B8007189000857890008A1880008A987000854
:1091C800E5880008D98F00082D8900087809002053
:1091D800014B1046DB6B184700000020034B10B50D
:1091E8001B6C14469847206010BD00BF000000208B
:1091F800062873B504460E467BD8404D68462B6B4F
:10920800013C98472B46042C04D8DFE804F0086694
:10921800696C6F009DF80030336000200BE09DF80A
:109228000120E978914208D19DF80200297B884203
:1092380003D10020306002B070BD1979914206D187
:109248009DF80200597B884201D10123E4E759794E
:10925800914206D19DF80200997B884201D10223F0
:10926800DAE79979914206D19DF80200D97B8842C4
:1092780001D10323D0E7D979914206D19DF80200A4
:10928800197C884201D10423C6E7597A914206D154
:109298009DF80200997C884201D10523BCE7997AA0
:1092A800914206D19DF80200D97C884201D106235B
:1092B800B2E7197A914206D19DF80200597C88429A
:1092C80001D10723A8E7D97A914214D19DF8022049
:1092D8001B7D9A420FD108239EE79DF803309BE738
:1092E8009DF8043098E79DF8053095E79DF806301D
:1092F80092E704209FE710209DE700BF00000020B0
:1093080007B5034B68461B6B984703B05DF804FB31
:109318000000002070B50020FFF7F2FF1E4B1F4C25
:10932800DD68206B2B689B6898472B68E06A9B6810
:1093380098472B68E0689B6898472B68A0689B68EB
:1093480098472B6860689B6898472B6820689B68DB
:1093580098472B68A0699B6898472B68E0699B68C9
:1093680098472B68A06A9B6898472B6860699B6838
:1093780098472B68206A9B6898472B68606A9B68A7
:1093880098472B6820699B68984714F001F9BDE855
:109398007040034B5B681847708602083C16002033
:1093A80078090020002013F07FBF10B5044618B9D3
:1093B80013F0BEFE204610BD0820FCE710B5044699
:1093C80018B913F093FE204610BD0820FCE70021D1
:1093D800F4E74942F2E7F1E7062873B505460C467B
:1093E8005DD8022903D901285BD10F2959DC2E4EFB
:1093F8006846336B98473346052D06D8DFE805F0F5
:10940800030B4346494C8DF800406846DB6A984791
:10941800002002B070BD082CF7D8DFE804F0050C76
:1094280011161B20252A2F00F2788DF80120327B97
:109438008DF80220E9E732798DF80120727BF7E791
:1094480072798DF80120B27BF2E7B2798DF80120AC
:10945800F27BEDE7F2798DF80120327CE8E7727A49
:109468008DF80120B27CE3E7B27A8DF80120F27C16
:10947800DEE7327A8DF80120727CD9E7F27A8DF82E
:109488000120327DD4E78DF80340BEE78DF8044013
:10949800BBE78DF80540B8E78DF80640B5E704202E
:1094A800B7E71020B5E700BF0000002038B5154623
:1094B80018B1012807D0042004E0084613F078FE0C
:1094C8002860002038BD094B094DDC68094B6068ED
:1094D80000F5B870D8616B6C58612368DB689847F1
:1094E8006A6C236850699B699847EAE770860208A6
:1094F800000000203C16002038B50D46044648B947
:1095080013F03EFF2B68C1182960204613F010FEA7
:10951800204638BD0820FCE770B5054616460C46BF
:1095280000295DD10B2810D806283CD202282ED05D
:1095380004D808B3012825D0042421E004282ED01B
:1095480029D9084613F054FF1FE013280CD80E2819
:109558003CD20C282FD00D28EED1224B224ADB68B2
:10956800106B1B685B6A2CE0322835D03328E3D1B6
:10957800084613F075FF08E013F010FF2C46306022
:10958800204670BD084613F0FBFE3060F8E7084639
:1095980013F020FFF9E7084613F00EFFF5E7084639
:1095A80013F034FFF1E70828C6D1084613F000FE8F
:1095B800C0F30010E9E70B4B0B4ADB68D06A1B6865
:1095C8005B6A9847003018BF0120DEE70E38114665
:1095D800C0B2FFF70DFED3E7084613F033FFD4E718
:1095E8000824CDE7708602083C16002030B585B007
:1095F800054601920C4600296ED10B2812D8062880
:1096080046D2022837D004D848B301282CD00424E5
:109618002EE0042834D00528F9D11146204613F04D
:10962800DEFF25E013280FD80E2845D20C2836D0A7
:109638000D28ECD142F210739A42E8D8274B91B228
:109648009B682046984713E0332837D08C283AD0B7
:109658003228DCD1D1B2204613F078FE08E011465A
:1096680013F066FD2C4603E01146204613F03AFE3F
:10967800204605B030BD1146204613F037FDF7E708
:1096880082EAE271A1EBE271204613F045FEEFE7B2
:1096980006381146C0B2FFF79FFE0446E8E7104BB4
:1096A8001049DB68C86A1B68154612B15B699847A0
:1096B800DEE79B699847D5E70E38EAE7114620466A
:1096C80013F054FED4E701A90120FFF791FD064BE2
:1096D80004469B6B02A8EAE70824C9E7780900203A
:1096E800708602083C160020000000206D4B2DE912
:1096F800F041DE686C4C7068002500F5FE7323634A
:1097080000F5F073E36200F52973E36000F5307348
:10971800A36000F52273636000F50D73236000F504
:109728005A73A36100F55373E36100F1C803A362A0
:1097380000F5C673636100F56873236200F56F7303
:109748006362336800F5B870DB6820619847336856
:109758006069DB6898473368206BDB689847336833
:10976800E06ADB6898473368206A1B699847336862
:109778004E4F1B69606A98477B6CE2681A60A26862
:109788005A6062689A602268DA60A2691A61E269BE
:109798005A61A26A9A617A6C33685059DB689847B3
:1097A8007A6C336850599B69043598471C2DF2D15F
:1097B8004FF000083E4DD5F8883083F8008013F04C
:1097C80073FED4E904124346404613F015FD44F6EF
:1097D8002061404613F0A0FD46F2A811404613F060
:1097E800FEFE344B0220C5F89430334BC5F8903058
:1097F800324BC5F88C30324BC5F89830314BC5F830
:10980800AC30314BC5F8A830304BC5F89C30304BE4
:10981800C5F8A0302F4BC5F8BC302F4BC5F8B83071
:109828002E4BC5F8C4302E4BC5F8C8302D4BC5F8A3
:10983800D430012385F884302B4BC5F8CC30FFF7A2
:109848005FFD404613F0B8FD10B1284B9B789BB1E3
:10985800BB6A984713F028FED4E90412002318467F
:1098680013F0CAFC44F62061002013F055FD46F2BF
:10987800A811002013F0B3FE0222236B197C5A743E
:109888001868012219F062F93368206B184C1B68BC
:109898009847236898470021A3680846BDE8F04127
:1098A800184700BF708602083C1600200000002000
:1098B80000610020C5930008DF930008DB930008CF
:1098C800D793000821950008F5950008B393000880
:1098D80001950008D9910008E5910008B5940008A1
:1098E800AD930008099300081D930008CC090020D7
:1098F800780900201B4B70B5DD681B4C2B68A068ED
:109908005B6998472B6820689B6898472B68606854
:109918009B6898472B68206A9B6898472B68606A01
:109928009B6898472B68E0689B6898472B68206974
:109938009B6898472B6860699B6898472B68A06963
:109948009B6898472B68E0699B6898472B68A068D4
:109958009B68984713F01CFEBDE87040034B5B689A
:10996800184700BF708602087C160020780900207E
:1099780010B5144605284DD8DFE800F0032321323E
:109988003D4244F6206314689C4245D842F2107167
:10999800224B234ADB688C421B6898BF0021DB6995
:1099A80088BF0121106A984742F21173B4FBF3F1A2
:1099B80003FB11411B4B89B29B680020984700208C
:1099C80010BD164B2468DA68D2E9003000F506703D
:1099D8001CB10021DB699847F1E79B689847EEE7DF
:1099E8000E4B1168DB680E4A1B680031DB6918BF33
:1099F80001211069EFE7084613F0DAFB2060DEE783
:109A0800064B074ADB6858681B6800F5B870106198
:109A1800DB68E3E70420D3E71020D1E7708602086B
:109A28007C1600207809002010B50348144614F06D
:109A380062FA206010BD00BF3462002010B5094CE6
:109A48000146204614F0C6FA002013F02DFC6F21C1
:109A5800204614F050FABDE81040C0F30061002021
:109A680013F0F4BB34620020014814F036BA00BF8A
:109A78003462002010B5044618B913F059FB20468B
:109A880010BD0820FCE710B5044618B913F02EFBEA
:109A9800204610BD0820FCE70021F4E74942F2E720
:109AA800F1E7014814F07DBA34620020022804BFAF
:109AB8000B4B93F8E80030B90A4BDB681B685B690D
:109AC800094A90681847012809D1054B93F8E830EE
:109AD800012B04D1034BDB681B689B69F0E77047D7
:109AE80000610020708602087C1600200346052BC2
:109AF80010B5084614460BD006D8022B06D313F02F
:109B0800AFFC2060002010BD182BF8D00420FAE725
:109B180013F0B4FCF5E738B50D46044620B913F048
:109B28004BFC2860204638BD0820FCE7012903D1FA
:109B3800024A702114F0D1B9704700BFC80405006B
:109B4800A52970B50446154600F0538200F28C80B2
:109B5800172900F077812DD8042900F036810CD818
:109B6800012900F01481C0F00781022900F0188152
:109B7800032900F01F810424F9E1072900F0498135
:109B88000ED8052900F02D810629F4D11021C048EE
:109B9800002C40F0308114F0AEF9C0F30420EEE060
:109BA800082900F046811529E5D10028E3D012687C
:109BB80011212AE1322900F0A1812FD81B2900F0B8
:109BC80079810ED8182900F05C811A29D3D16C212B
:109BD800AF48002C40F0638114F08DF9C0F3804049
:109BE800CDE01C2900F077811D29C4D10028C2D1FD
:109BF800204613F035FC12210646A54814F07BF9DF
:109C0800C0F313027A20D317A6FB00011CF00EFE46
:109C180000F11303262B98BF0020B0E0A22900F022
:109C2800BD8112D8332900F072818C29A3D1002874
:109C380040F077816C21964814F05DF94FF48073F9
:109C4800C0F3036043FA00F099E0A32900F0B7815C
:109C5800A42990D16C218E48002C40F0C18114F0C9
:109C68004AF9C0F300308AE0B42900F0BF823FD837
:109C7800AA2900F0658214D8A72900F03682C0F01E
:109C88000982A82900F04182A9297FF474AF6D21C7
:109C98007F48002C40F04B8214F02DF9C0F341307E
:109CA8006DE0AD2900F0708212D8AB2900F059821E
:109CB800AC297FF460AF6D217548002C00F0188244
:109CC80014F019F92B6820F00F0203F00F032BE2B0
:109CD800AE2900F06A82B3297FF44DAF6C216C483D
:109CE800002C40F07A8214F006F9C0F3404046E0B8
:109CF800BB2900F0CF821BD8B82900F099820BD875
:109D0800B52900F07D82B6297FF435AF614E002871
:109D180040F08082142198E0B92900F09A82BA298B
:109D28007FF429AF5B4E002840F0A68213218CE017
:109D3800C02900F0EE820FD8BC2900F0CB82BF29E1
:109D48007FF419AF002840F0D4827021504814F0F5
:109D5800D2F8C0F3014012E0CC2900F0EA82CE2903
:109D68007FF409AF00287FF406AF6F21484814F04C
:109D7800C2F8C0F3090002E018B913F00FFB28601D
:109D8800F5E01168002013F0D3F90024EFE010B9D2
:109D980013F0F6FAF3E71168002013F0A3FAF4E7DA
:109DA80018B9002013F016FBE9E71168002013F03A
:109DB8009DF9EAE700287FF4DEAE13F043FB0028A4
:109DC8007FF416AF13F0F8FAD9E710B913F01EFBB9
:109DD800D5E7116800200029B8BF494213F09CFA62
:109DE800D3E718B9002013F003FBC8E71168002077
:109DF80013F0F5FBC9E714F07EF82B6820F4F8524D
:109E08001B0203F4F85310211A43214814F065F893
:109E1800BBE710211E4824B914F06DF800F01F00AC
:109E2800ADE714F068F82B6820F01F0203F01F0359
:109E3800E9E700287FF49FAE002013F0B9F9C0F3DA
:109E480000109CE7134E70B91521114814F053F80F
:109E5800002800F00F824FF0807393FBF0F0B042BF
:109E6800A8BF3046E2E013684BB14FF0807292FB16
:109E7800F3F2B242A8BF32462A601521C5E732463E
:109E8800FAE748B93321024814F035F877E700BFFC
:109E980034620020FFFF0F0012683321B5E714F089
:109EA8002AF82B6820F480229B0403F480231A43A9
:109EB8006C21AAE76C21B34824B914F01CF8C0F34C
:109EC800C0405CE714F017F82B6820F40022DB048C
:109ED80003F40023EBE70021AA4824B914F00BF897
:109EE800C0F340004BE714F006F82B6820F002029C
:109EF8005B0003F002031A43002186E710B913F050
:109F0800A1FA3CE71178002013F020FA3DE718B9D0
:109F1800002013F0A5FA32E71168002013F026FAA2
:109F280033E71368102B28D00DDC022B21D004DC7A
:109F3800012B16D04FF0FF3314E0042B1BD0082B55
:109F4800F8D105230EE0402B19D003DC202BF1D1EA
:109F5800032307E0802B14D0B3F5807FEAD10023D8
:109F680000E008232B602B6801330CD11024204615
:109F780070BD0723F6E70623F4E70423F2E702237C
:109F8800F0E70123EEE76C217E4813F0B4FF2B685D
:109F980020F070621B0603F0706388E76C21794833
:109FA80024B913F0A8FFC0F3C130E8E613F0A3FF0B
:109FB8002B6820F4C032DB0303F4C03377E76C214D
:109FC800704824B913F097FFC0F38030D7E613F038
:109FD80092FF2B6820F480429B0303F4804366E7DA
:109FE80013F089FF2B6820F480521B0303F480537D
:109FF8005DE76C216348DCB913F07DFF10F48046FF
:10A008004FF06C015F4804D013F075FFC0F3C31024
:10A01800B5E613F070FF6C2104465A4813F06BFF45
:10A02800C0F30210230548BF40F008002860ACE6E2
:10A0380013F061FF10F480444FF06C01514808D0D0
:10A0480013F059FF2B6820F4F062DB0103F4F0638E
:10A058002DE713F050FF6C214A4813F04CFF2A6893
:10A0680020F40060120202F4006202436C214548A9
:10A0780013F033FF6C21434813F03DFF2B6820F0A9
:10A0880070021B0103F070031A436C213D4813F062
:10A0980024FF6CE76C213B48B4B913F02CFF10F493
:10A0A800804F4FF06C01374804D013F024FFC0F301
:10A0B800021064E613F01FFF6C210446314813F0C8
:10A0C8001AFFC0F3C310ADE713F015FF10F4804F6B
:10A0D8004FF06C012B48B3D013F00DFF2B6820F024
:10A0E80070021B0103F07003E1E66C21254824B9D6
:10A0F80013F001FF00F00F0041E613F0FCFE2B689F
:10A1080020F00F0203F00F03D1E66D211D4824B99A
:10A1180013F0F1FEC0F3C03031E613F0ECFE2B680B
:10A1280020F40042DB039BB21A436D216DE613F065
:10A13800E2FE2B6820F4C0425B0303F4C043F3E75C
:10A148006D21104824B913F0D6FEC0F3032016E69B
:10A1580013F0D1FE2B6820F470621B0203F47063C5
:10A16800E2E76D21074824B913F0C5FEC0F341109A
:10A1780005E613F0C0FE2B6820F060025B0103F0D7
:10A188006003D1E7346200206D21724824B913F0CE
:10A19800B2FEC0F30060F2E513F0ADFE2B6820F0CC
:10A1A80080721B0603F08073BEE76D2169485CB9B5
:10A1B80013F0A1FE001400F07F0310F0400018BF58
:10A1C8006FF07F001843DAE513F095FE2B6820F452
:10A1D800FE021B0403F4FE03A6E713F08CFE2B68B3
:10A1E80020F400325B0403F4003360E600287FF4B7
:10A1F800C2AC6F21574813F07EFEC0F30440BEE5A1
:10A2080018B9002013F010F9B9E51168002013F00F
:10A218008FF8BAE513684BB14FF0807292FBF3F2F6
:10A22800B242A8BF32462A601421EEE53246FAE768
:10A238006C21484824B913F05EFEC0F340309EE517
:10A2480013F059FE2B6820F400525B0303F400530B
:10A258002DE66C213F4824B913F04DFEC0F303509E
:10A268008DE513F048FE2B6820F470021B0503F4FB
:10A2780070031CE63046D9E613684BB14FF0807284
:10A2880092FBF3F2B242A8BF32462A601321BCE522
:10A298003246FAE770212F4824B913F02CFEC0F398
:10A2A80007206CE513F027FE2A6820F47F4012028D
:10A2B80092B202437021274813F00FFE002125486F
:10A2C80013F019FE2B6820F00402002BCCBF0423E6
:10A2D800002310E670211F481CB913F00CFEC0B211
:10A2E8004DE513F008FE2A7820F0FF0002437021A4
:10A2F8008BE51368032B3FF639AE7021154813F030
:10A30800FAFD2B6820F440321B0403F440331A434F
:10A31800EDE770210F48002C3FF45EAC13F0EBFD25
:10A328002B6820F48022002B14BF4FF480230023D5
:10A33800EDE77021074824B913F0DDFDC0F30150A3
:10A348001DE513F0D8FD2B6820F440121B0503F41B
:10A358004013DCE7346200200B4619B90146184661
:10A36800FFF7EEBB0820704708B5002013F024F86B
:10A3780010B1084B987858B1074813F0FDFD13F059
:10A3880093F800230549184606C912F035FF012045
:10A3980008BD00BFCC090020346200207C160020D4
:10A3A80038B50D46044648B912F0EAFF2B68C118C3
:10A3B8002960204612F0BCFE204638BD0820FCE784
:10A3C80007B5019239B9014601AA0120FFF7B8FB88
:10A3D80003B05DF804FB0820FAE7022806D3052835
:10A3E80001D9182802D10020106070470420704756
:10A3F800044B08469B6E114603B11847024B1B6875
:10A40800DB68FAE700610020B86400202DE9F0411C
:10A418006B4D6C4CD5F888206B4B20466B4F012157
:10A4280013F08EFD6A49204613F0D0FDFE68694C92
:10A4380073684FF0000803F1C802A26003F5B87210
:10A44800226003F5C672626003F5F072226203F5BA
:10A45800FE72626203F55372E26003F55A7203F505
:10A468006870226103F5617203F56F73E361336805
:10A4780062611B69A06198473368E0691B69984766
:10A48800336860691B69984733682068DB689847B8
:10A4980033686068DB6898473368A068DB6898476A
:10A4A80033682069DB6898473368E068DB68984759
:10A4B8003368606ADB6898473368206ADB689847C6
:10A4C8003368606A9B6998473368206A9B69984734
:10A4D800336860699B6998473368E0689B69984767
:10A4E8003A693D4B02F1140119607368012703F5BD
:10A4F8000D73936112F0D8FFD4E9001200231846B7
:10A5080012F07AFED5F88830344A1F70C3F8042256
:10A51800334A83F80180C3F80822324B3222C5F847
:10A528009430314B0220C5F89030304B85F8847058
:10A53800C5F88C302E4BC5F898302E4BC5F8AC308A
:10A548002D4BC5F8A8302D4BC5F89C302C4BC5F8C1
:10A55800A0302C4BC5F8BC302B4BC5F8B8302B4B72
:10A56800C5F8C8302A4BC5F8C4302A4BC5F8C030E6
:10A57800294BC5F8D4304FF4F073C5E91F32274B87
:10A58800C5F8CC30264BC5F8E030264BC5F8E4308A
:10A59800FFF78CFA0222636A197C5A7418683A46E3
:10A5A80018F0D4FA3368606A1F4C1B689847236810
:10A5B8009847A36841464046BDE8F041184700BFA8
:10A5C800006100203462002048700208708602088A
:10A5D800359B00087C160020B864002071A3000891
:10A5E800AB9A00088F9A0008A99A0008A59A000853
:10A5F800A19A000861A30008C9A300087D9A000871
:10A60800A9A30008719A0008319A0008459A000821
:10A61800799900081F9B0008B59A0008FD98000862
:10A62800E3A30008F59A00087809002038B5184B0C
:10A63800184CDD6820682B685B6998472B68606850
:10A648009B6898472B68A0689B6898472B68E068C8
:10A658009B6898472B6820699B6898472B686069B6
:10A668009B6898472B68A0699B6898472B68E069A6
:10A678009B6898472B68206A9B68984712F088FF68
:10A68800054B5B689847002384F8243038BD00BF29
:10A6980070860208B01600207809002010B503481B
:10A6A800144613F014FD206010BD00BFC0640020E4
:10A6B800014813F0FEBC00BFC064002010B504467A
:10A6C80018B912F035FD204610BD0820FCE710B57A
:10A6D800044618B912F00AFD204610BD0820FCE710
:10A6E8000021F4E74942F2E7F1E7014813F06BBDB6
:10A6F800C0640020022804BF0B4B93F8E80030B96F
:10A708000A4BDB681B685B69094A1068184701280F
:10A7180009D1054B93F8E830012B04D1034BDB68D2
:10A728001B689B69F0E7704700610020708602088B
:10A73800B016002010B51446062844D8DFE800F00B
:10A748000416142530353F00136844F620629342FE
:10A758003BD842F21172B3FBF2F102FB11311C4BF0
:10A7680089B29B6800209847002010BD194B2468C7
:10A77800DA68D2E9003000F506701CB10021DB6907
:10A788009847F1E79B689847EEE7124B1168DB683A
:10A79800114A1B680031DB6918BF01215069EFE7D6
:10A7A800084612F005FD2060DEE70A4B0A4ADB681E
:10A7B80058681B6800F5B8705061DB68E3E7022051
:10A7C800FFF798FFD0E70420CFE71020CDE700BFC0
:10A7D8007809002070860208B01600200346052B71
:10A7E80010B5084614460BD006D8022B06D312F033
:10A7F80037FE2060002010BD182BF8D00420FAE79F
:10A8080012F03CFEF5E738B50D46044620B912F0C3
:10A81800D3FD2860204638BD0820FCE738B5194C20
:10A82800054694F8240001281CD002281FD0294688
:10A83800154813F0E1FC002012F036FD002012F05C
:10A84800B7FC10F008041BD1820619D56F210E48F9
:10A8580013F03DFCC30113D52046BDE83840022162
:10A8680012F07CBC0223A56284F82430DFE7A36AD7
:10A87800EB1AB3F5FA6FDAD9FFF73CFF0323F3E7D6
:10A8880038BD00BFB0160020C0640020A52970B5EF
:10A898000446154600F0538200F28C80172900F018
:10A8A80077812DD8042900F036810CD8012900F0D1
:10A8B8001481C0F00781022900F01881032900F0F3
:10A8C8001F810424F9E1072900F049810ED80529E0
:10A8D80000F02D810629F4D11021C048002C40F049
:10A8E800308113F0F4FBC0F30420EEE0082900F0F7
:10A8F80046811529E5D10028E3D0126811212AE103
:10A90800322900F0A1812FD81B2900F079810ED8B7
:10A91800182900F05C811A29D3D16C21AF48002C8A
:10A9280040F0638113F0D3FBC0F38040CDE01C29D5
:10A9380000F077811D29C4D10028C2D1204612F029
:10A948008FFD12210646A54813F0C1FBC0F3130280
:10A958007A20D317A6FB00011BF068FF00F1130350
:10A96800262B98BF0020B0E0A22900F0BD8112D8A4
:10A97800332900F072818C29A3D1002840F0778117
:10A988006C21964813F0A3FB4FF48073C0F3036067
:10A9980043FA00F099E0A32900F0B781A42990D1E7
:10A9A8006C218E48002C40F0C18113F090FBC0F35D
:10A9B80000308AE0B42900F0BF823FD8AA2900F00D
:10A9C800658214D8A72900F03682C0F00982A82928
:10A9D80000F04182A9297FF474AF6D217F48002CD3
:10A9E80040F04B8213F073FBC0F341306DE0AD29AA
:10A9F80000F0708212D8AB2900F05982AC297FF49C
:10AA080060AF6D217548002C00F0188213F05FFBD1
:10AA18002B6820F00F0203F00F032BE2AE2900F0A1
:10AA28006A82B3297FF44DAF6C216C48002C40F04A
:10AA38007A8213F04CFBC0F3404046E0BB2900F09B
:10AA4800CF821BD8B82900F099820BD8B52900F01D
:10AA58007D82B6297FF435AF614E002840F08082B0
:10AA6800142198E0B92900F09A82BA297FF429AF15
:10AA78005B4E002840F0A68213218CE0C02900F02C
:10AA8800EE820FD8BC2900F0CB82BF297FF419AF22
:10AA9800002840F0D4827021504813F018FBC0F30E
:10AAA800014012E0CC2900F0EA82CE297FF409AFF8
:10AAB80000287FF406AF6F21484813F008FBC0F365
:10AAC800090002E018B912F069FC2860F5E0116885
:10AAD800002012F02DFB0024EFE010B912F050FC1A
:10AAE800F3E71168002012F0FDFBF4E718B9002025
:10AAF80012F070FCE9E71168002012F0F7FAEAE7B3
:10AB080000287FF4DEAE12F09DFC00287FF416AF1B
:10AB180012F052FCD9E710B912F078FCD5E71168A9
:10AB280000200029B8BF494212F0F6FBD3E718B954
:10AB3800002012F05DFCC8E71168002012F04FFDFC
:10AB4800C9E713F0C4FA2B6820F4F8521B0203F487
:10AB5800F85310211A43214813F0ABFABBE7102130
:10AB68001E4824B913F0B3FA00F01F00ADE713F044
:10AB7800AEFA2B6820F01F0203F01F03E9E7002854
:10AB88007FF49FAE002012F013FBC0F300109CE787
:10AB9800134E70B91521114813F099FA002800F0E6
:10ABA8000F824FF0807393FBF0F0B042A8BF30469D
:10ABB800E2E013684BB14FF0807292FBF3F2B242BD
:10ABC800A8BF32462A601521C5E73246FAE748B9D8
:10ABD8003321024813F07BFA77E700BFC0640020F6
:10ABE800FFFF0F0012683321B5E713F070FA2B68E6
:10ABF80020F480229B0403F480231A436C21AAE7E3
:10AC08006C21B34824B913F062FAC0F3C0405CE782
:10AC180013F05DFA2B6820F40022DB0403F4002310
:10AC2800EBE70021AA4824B913F051FAC0F3400019
:10AC38004BE713F04CFA2B6820F002025B0003F09C
:10AC480002031A43002186E710B912F0FBFB3CE728
:10AC58001178002012F07AFB3DE718B9002012F0B5
:10AC6800FFFB32E71168002012F080FB33E713681E
:10AC7800102B28D00DDC022B21D004DC012B16D0A0
:10AC88004FF0FF3314E0042B1BD0082BF8D1052319
:10AC98000EE0402B19D003DC202BF1D1032307E071
:10ACA800802B14D0B3F5807FEAD1002300E008237D
:10ACB8002B602B6801330CD11024204670BD07236C
:10ACC800F6E70623F4E70423F2E70223F0E701237B
:10ACD800EEE76C217E4813F0FAF92B6820F07062D9
:10ACE8001B0603F0706388E76C21794824B913F0D8
:10ACF800EEF9C0F3C130E8E613F0E9F92B6820F467
:10AD0800C032DB0303F4C03377E76C21704824B901
:10AD180013F0DDF9C0F38030D7E613F0D8F92B68CB
:10AD280020F480429B0303F4804366E713F0CFF9D5
:10AD38002B6820F480521B0303F480535DE76C21D9
:10AD48006348DCB913F0C3F910F480464FF06C0186
:10AD58005F4804D013F0BBF9C0F3C310B5E613F095
:10AD6800B6F96C2104465A4813F0B1F9C0F3021041
:10AD7800230548BF40F008002860ACE613F0A7F9A7
:10AD880010F480444FF06C01514808D013F09FF93B
:10AD98002B6820F4F062DB0103F4F0632DE713F075
:10ADA80096F96C214A4813F092F92A6820F4006059
:10ADB800120202F4006202436C21454813F079F94B
:10ADC8006C21434813F083F92B6820F070021B01B3
:10ADD80003F070031A436C213D4813F06AF96CE7DD
:10ADE8006C213B48B4B913F072F910F4804F4FF05E
:10ADF8006C01374804D013F06AF9C0F3021064E616
:10AE080013F065F96C210446314813F060F9C0F37A
:10AE1800C310ADE713F05BF910F4804F4FF06C01ED
:10AE28002B48B3D013F053F92B6820F070021B01A4
:10AE380003F07003E1E66C21254824B913F047F9C3
:10AE480000F00F0041E613F042F92B6820F00F02E2
:10AE580003F00F03D1E66D211D4824B913F037F92B
:10AE6800C0F3C03031E613F032F92B6820F4004209
:10AE7800DB039BB21A436D216DE613F028F92B68AA
:10AE880020F4C0425B0303F4C043F3E76D2110488C
:10AE980024B913F01CF9C0F3032016E613F017F9D0
:10AEA8002B6820F470621B0203F47063E2E76D21E3
:10AEB800074824B913F00BF9C0F3411005E613F065
:10AEC80006F92B6820F060025B0103F06003D1E70C
:10AED800C06400206D21724824B913F0F8F8C0F35B
:10AEE8000060F2E513F0F3F82B6820F080721B067F
:10AEF80003F08073BEE76D2169485CB913F0E7F889
:10AF0800001400F07F0310F0400018BF6FF07F00BE
:10AF18001843DAE513F0DBF82B6820F4FE021B0473
:10AF280003F4FE03A6E713F0D2F82B6820F40032EE
:10AF38005B0403F4003360E600287FF4C2AC6F21A1
:10AF4800574813F0C4F8C0F30440BEE518B9002010
:10AF580012F06AFAB9E51168002012F0E9F9BAE5C9
:10AF680013684BB14FF0807292FBF3F2B242A8BF64
:10AF780032462A601421EEE53246FAE76C21484849
:10AF880024B913F0A4F8C0F340309EE513F09FF8FD
:10AF98002B6820F400525B0303F400532DE66C2168
:10AFA8003F4824B913F093F8C0F303508DE513F02C
:10AFB8008EF82B6820F470021B0503F470031CE65E
:10AFC8003046D9E613684BB14FF0807292FBF3F22A
:10AFD800B242A8BF32462A601321BCE53246FAE7DE
:10AFE80070212F4824B913F072F8C0F307206CE5DC
:10AFF80013F06DF82A6820F47F40120292B20243DF
:10B008007021274813F055F80021254813F05FF800
:10B018002B6820F00402002BCCBF0423002310E689
:10B0280070211F481CB913F052F8C0B24DE513F057
:10B038004EF82A7820F0FF00024370218BE5136850
:10B04800032B3FF639AE7021154813F040F82B68F2
:10B0580020F440321B0403F440331A43EDE7702117
:10B068000F48002C3FF45EAC13F031F82B6820F445
:10B078008022002B14BF4FF480230023EDE77021BA
:10B08800074824B913F023F8C0F301501DE513F065
:10B098001EF82B6820F440121B0503F44013DCE76C
:10B0A800C06400200B4619B901461846FFF7EEBBED
:10B0B8000820704708B5002012F07EF910B1084B3F
:10B0C800987860B1074813F069F812F0EDF9002399
:10B0D800054918468A68496812F08EF8012008BDAB
:10B0E800CC090020C0640020B0160020012910B54A
:10B0F80004460DD1074A702112F0DBFF2046064AAC
:10B108000A2112F0D6FF2046BDE8104013F020B8FF
:10B1180010BD00BF1E000CC40004080038B50D4661
:10B12800044648B912F02CF92B68C118296020464A
:10B1380011F0FEFF204638BD0820FCE707B5019254
:10B1480039B9014601AA0120FFF7A0FB03B05DF859
:10B1580004FB0820FAE7022806D3052801D9182895
:10B1680002D100201060704704207047044B084645
:10B178009B6E114603B11847024B1B68DB68FAE760
:10B1880000610020BC6400202DE9F0415A4C5B4D61
:10B19800D4F888205A4B28465A4F012112F0BCFF98
:10B1A8005949284613F024F8FE68584D736803F18E
:10B1B800C8022A6003F5B8726A6003F5C672AA600D
:10B1C80003F5FE72EA6003F553722A6103F55A72B9
:10B1D80003F561706A6103F5687203F56F732B629A
:10B1E8003368EA611B69A861984733682868DB6897
:10B1F800984733686868DB6898473368A868DB68ED
:10B2080098473368E868DB68984733686869DB689B
:10B21800984733682869DB6898473368E8685B694A
:10B2280098473368A8699B699847336828699B6978
:10B2380098473A69364B02F1140119607368002681
:10B2480003F50D73936112F02FF9D5E9011200236C
:10B25800184611F0D1FFD4F888302E4A5E70C3F832
:10B2680004222D4A3221C3F8082201221A702B4BDE
:10B2780084F88420C4F89430294B85F82420C4F835
:10B288009030284BC4F88C30274BC4F89830274BA3
:10B29800C4F8AC30264BC4F8A830264BC4F89C3010
:10B2A800254BC4F8A030254BC4F8BC30244BC4F857
:10B2B800B830244BC4F8C830234BC4F8C430234BEF
:10B2C800C4F8C030224BC4F8D4304FF4F073C4E94A
:10B2D8001F31204BC4F8CC301F4BC4F8E0301F4B53
:10B2E800C4F8E4301E4C23689847A36831463046BA
:10B2F800BDE8F041184700BF00610020C06400208D
:10B308004872020870860208F5B00008B0160020DE
:10B31800BC640020BDB00008F3A60008D7A600084A
:10B32800F1A60008EDA60008E9A60008ADB00008DF
:10B3380045B10008C5A6000825B10008B9A600084F
:10B34800A5A6000825A800083DA700080FA8000822
:10B35800FDA6000835A600085FB10008E5A70008AB
:10B36800780900200022014B9A677047006100208D
:10B37800F8B50A4E0C46304650F8047B154613F0D3
:10B388000CF82B4622460146384610F0C8FA736876
:10B3980004F07F0403EB84046560F8BDE816002020
:10B3A80008B50146034812F083FFBDE808400020B5
:10B3B80011F07ABFEC16002038B51546044628B9B6
:10B3C800084611F0F5FE2860204638BD0420FCE749
:10B3D80010B5044618B911F0ABFE204610BD082080
:10B3E800FCE710B5044618B911F080FE204610BDE0
:10B3F8000820FCE70021F4E74942F2E7F1E70148B9
:10B4080012F0C1BFEC16002010B512F04DF8002361
:10B41800064C1846D4F8A022D4F89C1211F0ECFE81
:10B42800201DBDE8104012F096BF00BFE8160020AE
:10B43800022804BF0C4B93F8E80038B90B4BDB68C3
:10B448001B685B690A4AD2F898021847012809D193
:10B45800054B93F8E830012B04D1044BDB681B68DB
:10B468009B69EFE7704700BF006100207086020803
:10B47800E816002038B50020FFF7DAFF144B154C0A
:10B48800DD68D4F898022B689B6898472B68D4F835
:10B498009C029B6898472B68D4F8A0029B68984741
:10B4A8002B68D4F8A4029B6898472B68D4F8A802A4
:10B4B8009B6898472B68D4F8AC029B6898472B6820
:10B4C800D4F8B0029B689847BDE8384012F060B8DD
:10B4D80070860208E816002070B50E4801F07F0358
:10B4E8001446C21892F814220D46D2070BD550F80C
:10B4F800046B12F052FF23462A4601463046BDE847
:10B50800704010F0C5B9416801EB83014B682360B6
:10B5180070BD00BFE816002038B50D46044648B98E
:10B5280011F02EFF2B68C1182960204611F000FE8B
:10B53800204638BD0820FCE710B5144629BB06286C
:10B5480025D8DFE800F0040A0E12161A1E000020A3
:10B5580011F024FF2060002010BD002011F010FF22
:10B56800F8E7002011F036FFF4E7002011F024FF7F
:10B57800F0E7002011F04AFFECE7002011F038FF57
:10B58800E8E7044812F009FFE4E70820E4E70420AC
:10B59800E2E700BFEC16002008B549BB062829D809
:10B5A800DFE800F0040A0F28141C210011460020CF
:10B5B80011F0BEFD002008BD1146002011F092FEDA
:10B5C800F8E71146002011F091FDF3E782EAE271F5
:10B5D800A1EBE271002011F09FFEEBE7114600207D
:10B5E80011F0FDFFE6E7D1B2034812F0D9FEE1E71A
:10B5F8000820E0E70420DEE7EC1600200122F8B579
:10B60800544E1146072012F0E3F8F568524C6B6867
:10B61800274603F5B872C4F89C2203F5C672C4F82D
:10B62800A02203F58E72C4F8A42203F59C7203F1DC
:10B63800C800C4F8A82203F1E40203F58073C4F833
:10B64800B0322B68C4F8AC22DB68C4F8980298477B
:10B658002B68D4F89C02DB6898472B68D4F8A002C2
:10B66800DB6898472B68D4F8A402DB6898472B68F6
:10B67800D4F8A802DB6898472B68D4F8AC021B6999
:10B6880098472B680025D4F8B0021B699847F36ADD
:10B69800012647F8043B1D705B6898472F4B3049DB
:10B6A800D3F888203220C2F804122E491670C2F846
:10B6B80008122D495570C3F894102C4983F88460FA
:10B6C800C3F890102A49C3F88C102A49C3F8981077
:10B6D8002949C3F8AC102949C3F8A8102849C3F868
:10B6E8009C102849C3F8A0102749C3F8BC10274963
:10B6F800C3F8B8102649C3F8C4102649C3F8D410B3
:10B708002549C3F8D0104FF4C371C3E91F1023496A
:10B718003846C3F8CC102249C3F8C8102946214B33
:10B7280012F0A6FD11F0C0FE2B46D4F8A022D4F8E2
:10B738009C12284611F060FD28464FF4484111F04C
:10B74800EBFD28464FF4484111F049FF3046BDE86B
:10B75800F8406DE670860208E816002000610020B7
:10B7680011B4000807B40008EBB3000805B40008DA
:10B7780001B40008FDB3000841B50008A1B50008F0
:10B78800D9B3000821B5000879B30008E1B400086E
:10B79800C1B3000839B400086DB300087DB40008CF
:10B7A800A9B30008487402080022014B9A67704741
:10B7B80000610020074870B550F8044B0D46164646
:10B7C80012F04CFE33462A4601462046BDE870403A
:10B7D80010F0A5B8A8190020074870B550F8044B18
:10B7E8000D46164612F03AFE33462A4601462046D2
:10B7F800BDE8704010F04CB8A819002008B5064AFA
:10B808000146D2F894320020043212F006FEBDE858
:10B818000840002011F048BDA819002038B5154689
:10B82800044628B9084611F0C3FC2860204638BDF4
:10B838000420FCE710B5044618B911F079FC20463D
:10B8480010BD0820FCE710B5044618B911F04EFCED
:10B85800204610BD0820FCE70021F4E74942F2E742
:10B86800F1E7024BD3F8940212F0EFBDA8190020BB
:10B8780010B511F019FE0023064C1846D4F8A02282
:10B88800D4F89C1211F0B8FCD4F89402BDE810402A
:10B8980012F0D2BDA8190020022804BF0C4B93F85F
:10B8A800E80038B90B4BDB681B685B690A4AD2F8B9
:10B8B80098021847012809D1054B93F8E830012B65
:10B8C80004D1044BDB681B689B69EFE7704700BF36
:10B8D8000061002070860208A819002038B50020F1
:10B8E800FFF7DAFF164B174CDD68D4F898022B687F
:10B8F8009B6898472B68D4F89C029B6898472B68EC
:10B90800D4F8A0029B6898472B68D4F8A4029B68D7
:10B9180098472B68D4F8A8029B6898472B68D4F8F6
:10B92800AC029B6898472B68D4F8B0029B6898478C
:10B9380023689B689847BDE8384011F029BE00BFCE
:10B9480070860208A819002038B50D46044648B983
:10B9580011F016FD2B68C1182960204611F0E8FB8C
:10B96800204638BD0820FCE710B5144629BB062838
:10B9780025D8DFE800F0040A0E12161A1E0000206F
:10B9880011F00CFD2060002010BD002011F0F8FC23
:10B99800F8E7002011F01EFDF4E7002011F00CFD7F
:10B9A800F0E7002011F032FDECE7002011F020FD57
:10B9B800E8E7044812F052FDE4E70820E4E7042031
:10B9C800E2E700BFAC19002008B549BB062829D812
:10B9D800DFE800F0040A0F28141C2100114600209B
:10B9E80011F0A6FB002008BD1146002011F07AFCDA
:10B9F800F8E71146002011F079FBF3E782EAE271DB
:10BA0800A1EBE271002011F087FCEBE71146002062
:10BA180011F0E5FDE6E7D1B2034812F022FDE1E7B7
:10BA28000820E0E70420DEE7AC190020012270B509
:10BA3800534C1146534E072011F0CAFE201D12F038
:10BA4800B3FCF5686B6803F5B872C4F89C2203F57B
:10BA5800C672C4F8A02203F58E72C4F8A42203F5B6
:10BA68009C7203F1C800C4F8A82203F1E40203F5AC
:10BA78008073C4F8B0322B68C4F8AC22DB68C4F811
:10BA8800980298472B68D4F89C02DB6898472B6883
:10BA9800D4F8A002DB6898472B68D4F8A402DB68C6
:10BAA80098472B68D4F8A802DB6898472B68D4F825
:10BAB800AC021B6998472B68D4F8B0021B699847F9
:10BAC8000025F36A012623605B6898472E4B2F49AF
:10BAD800D3F88820C2F804122D4916705570C4F89E
:10BAE8009422C2F808122B4A3221C3F894202A4A19
:10BAF80083F88460C3F89020284AC3F88C20284A29
:10BB0800C3F89820274AC3F8AC20274AC3F8A820CE
:10BB1800264AC3F89C20264AC3F8A020254AC3F821
:10BB2800BC20254AC3F8B820244AC3F8C420244AB4
:10BB3800C3F8D420234AC3F8D0204FF4C372C3E912
:10BB48001F21214AC3F8CC20204AC3F8C82011F08D
:10BB5800ABFC2B46D4F8A022D4F89C12284611F04E
:10BB68004BFB28464FF4484111F0D6FB28464FF4CA
:10BB7800484111F034FD3046BDE870408CE600BF06
:10BB8800A8190020708602080061002079B8000812
:10BB98006BB800084FB8000869B8000865B8000815
:10BBA80061B8000871B90008D1B900083DB80008AB
:10BBB80051B90008BDB70008E1B7000825B800086A
:10BBC800A1B80008B1B70008E5B8000805B8000832
:10BBD800012810B514460CD003D3022810D0042035
:10BBE80006E01368094AB3FA83F35B0993730020EC
:10BBF80010BD1368064AB3FA83F35B091360F6E7CE
:10BC0800084611F0D5FA2060F1E700BF681C002053
:10BC18006400002010B50348144612F06DFC206043
:10BC280010BD00BF681C0020014812F053BC00BFC3
:10BC3800681C0020F8B5374C06460021204612F053
:10BC48005BFC354DC0F3C0172A79BA4217D00621DC
:10BC58002046002F4CD012F04FFC00F01F00E0737C
:10BC68000621204612F048FC237903F01F0320F038
:10BC78001F021A430621204612F02CFC2F71274A76
:10BC8800217B936F00293ED043F00103617B00299B
:10BC98003CD043F002030020936711F08DFB6369E9
:10BCA8000028B8BF4042984234BF0027012794F8C3
:10BCB8004C20BA4213D098424FF0050115482CBFCA
:10BCC800657C257C12F018FC05F00F0520F00F02AA
:10BCD8002A4305210F4812F0FDFB84F84C703146C9
:10BCE8000C4812F053FCBDE8F840002011F0DCBA13
:10BCF80012F002FC00F01F0020710621204612F00D
:10BD0800FBFBE37BB1E723F00103BFE723F002036A
:10BD1800C1E700BF681C002064000020006100200B
:10BD280010B5044618B911F003FA204610BD0820D2
:10BD3800FCE7014812F09BBC681C0020022804BFE5
:10BD48000B4B93F8E80030B90A4BDB681B685B695A
:10BD5800094AD06D1847012809D1054B93F8E830F6
:10BD6800012B04D1034BDB681B689B69F0E7704724
:10BD78000061002070860208681C002038B5002089
:10BD8800FFF7DCFF0F4B104CDD68E06D2B685B693B
:10BD980098472B68206D9B6898472B68A06D9B6817
:10BDA80098472B68E06D9B6898472B68206E9B68C6
:10BDB80098472B68606D9B689847BDE8384011F03C
:10BDC800E7BB00BF70860208681C00200346052BED
:10BDD80010B5084614460BD006D8022B06D311F02E
:10BDE8003FFB2060002010BD182BF8D00420FAE794
:10BDF80011F044FBF5E738B50D46044620B911F0BB
:10BE0800DBFA2860204638BD0820FCE710B5044658
:10BE180028B9044B988111F069F9204610BD082013
:10BE2800FCE700BF681C00200021EFE74942EDE76E
:10BE3800ECE7A729F8B504460E46154600F01D8222
:10BE480067D81D2900F0038121D8042900F0068154
:10BE58000CD8012900F0E880C0F0DA80022900F04F
:10BE6800EC80032900F0F3800424D5E0062900F0D3
:10BE78000A81C0F0FF80072900F01E810829F3D14C
:10BE88000028F1D111F094F9C0F30010C3E0A12902
:10BE980000F08F811BD8332900F0298108D8322976
:10BEA800E2D1002840F01E81002011F0CBFAB2E068
:10BEB8008C2900F02581A029D6D1002840F06E8178
:10BEC8000821B44812F018FBC0F34020A3E0A429CD
:10BED80000F0A2810ED8A22900F07E81A329C3D147
:10BEE800002840F08E810C21AA4812F005FBC0F30F
:10BEF800803090E0A52900F0A281A629B4D10028BD
:10BF080040F0B0810C21A34812F0F6FAC0F30210F9
:10BF180081E0B22900F04D8241D8AC2900F0FC81C3
:10BF280013D8A92900F0CD81C0F0B981AA2900F061
:10BF3800D981AB2998D105219648002C40F0E3819E
:10BF480012F0DAFAC0F3411065E0AF2900F005827B
:10BF580015D8AD2900F0E781AE2985D106218D4895
:10BF6800002C40F0F18112F0C7FA000A00F07F03BC
:10BF780010F0400018BF6FF07F0018434BE0B02965
:10BF880000F0FD81B1297FF46FAF07218148002CB3
:10BF980040F0068212F0B0FAC0F380203BE0B729E7
:10BFA80000F0408210D8B42900F02582C0F0128237
:10BFB800B52900F02A82B6297FF456AF754B0028C0
:10BFC80040F02D825B6961E0CE2900F04F8213D8E2
:10BFD800B82900F03782B9297FF446AF07216D48A8
:10BFE800002C00F0A38112F087FA2B6820F480322D
:10BFF8001B0403F48033BFE1D02900F04D82D62919
:10C008007FF432AF634B002840F04F829B683DE0DD
:10C0180020B911F0C3F928602046F8BD1168002046
:10C0280011F086F80024F7E710B911F0A9F9F2E742
:10C038001168002011F056F9F4E718B9002011F042
:10C04800C9F9E8E71168002011F050F8EAE7002C78
:10C058007FF40AAF204611F0AFF9DCE710B911F010
:10C06800D5F9D8E7116800200029B8BF494211F076
:10C0780053F9D7E710B911F0BBF9CCE711680020E4
:10C0880011F0ADFACEE7434F10B9FB7B2B60C3E745
:10C098001368FB73404B1C79002CC3D1384612F04F
:10C0A8002BFAFB7B20F01F0203F01F031A433146D3
:10C0B800384612F00FFAAFE7364E08B93379E5E79C
:10C0C80013683371344B1B79012BABD106213148EE
:10C0D80012F012FA337920F01F0203F01F031A43FB
:10C0E800062148E01178002011F030F99AE710B9DC
:10C0F80011F0B6F98FE71168002011F037F991E7D0
:10C1080040B90821234812F0F7F900F00F00C0F1F8
:10C11800080080E71368102B35D00DDC022B2ED0D9
:10C1280004DC012B16D04FF0FF3314E0042B28D089
:10C13800082BF8D105230EE0402B26D003DC202B5A
:10C14800F1D1032307E0802B21D0B3F5807FEAD11A
:10C15800002300E008232B602B68013300F0A8813E
:10C1680000210C4812F0C8F92B6820F00F0203F0E8
:10C178000F0300211A43074812F0ACF952E70723CE
:10C18800E9E70623E7E70423E5E70223E3E70123DA
:10C19800E1E700BF681C0020640000200021B248CD
:10C1A80012F0AAF92B6820F400725B0203F4007302
:10C1B800DFE730B90821AC4812F09EF9C0F300203F
:10C1C80029E70021A84812F097F92B6820F480721B
:10C1D8001B0203F48073CCE730B90C21A24812F09B
:10C1E8008BF9C0F3C13016E704219F4812F084F997
:10C1F8002B6820F4C032DB0303F4C0331A43042154
:10C20800B9E70421984812F077F92B6820F48042A6
:10C218009B0303F48043F1E730B90C21924812F0F4
:10C228006BF9C0F3C120F6E604218F4812F064F9D7
:10C238002B6820F4C052DB0203F4C053DEE730B9A8
:10C248000C21894812F058F9C0F3C310E3E6042121
:10C25800854812F051F92B6820F4F062DB0103F4F1
:10C26800F063CBE70421804812F046F92B6820F0F0
:10C2780070021B0103F07003C0E730B90C217A4843
:10C2880012F03AF900F00F00C5E60421764812F0E2
:10C2980033F92B6820F00F0203F00F03AEE70521F6
:10C2A800714824B912F028F9C0F3C030B3E612F08F
:10C2B80023F92B6820F40042DB039BB21A430521C3
:10C2C80059E70521684824B912F016F9C0F341303E
:10C2D800A1E612F011F92B6820F4C0425B0303F4C5
:10C2E800C043EBE70521604824B912F005F9C0F313
:10C2F800032090E612F000F92B6820F470621B020C
:10C3080003F47063DAE712F0F7F82B6820F06002A4
:10C318005B0103F06003D1E7534B08B95B7CB5E6DA
:10C3280012685A747EE606214F4824B912F0E4F8E0
:10C33800C0F300406FE612F0DFF82B6820F480327B
:10C348001B0403F48033CAE612F0D6F82B6820F4F5
:10C35800FE421B0203F4FE43C1E60721424824B90A
:10C3680012F0CAF8C0F3813055E612F0C5F82B6810
:10C3780020F440429B039BB21A430721FBE60721A6
:10C38800394824B912F0B8F8C0F3013043E612F086
:10C39800B3F82B6820F440521B0303F44053EBE737
:10C3A80012F0AAF82B6820F480629B0203F48063E1
:10C3B800E2E707212C4824B912F09EF8C0F30120C7
:10C3C80029E612F099F82B6820F440721B0203F456
:10C3D8004073D1E70721244824B912F08DF8C0F33F
:10C3E800801018E612F088F82B6820F040029B01B4
:10C3F80003F04003C0E700287FF436AD02211A4855
:10C4080012F07AF8C0F3842005E618B9002011F07C
:10C418000BF800E61168002010F08AFF02E61268A7
:10C428005A61FFE50721104824B912F065F8C0F3F6
:10C43800C010F0E512F060F82B6820F08002DB01F4
:10C44800DBB299E70421084824B912F055F8C0F383
:10C458004030E0E512F050F82B6820F400525B03FE
:10C4680003F40053CAE600BF681C002000287FF4CC
:10C47800FBAC104B1B6843B102210F4812F03CF88B
:10C48800800A00F478702860CCE501210A4812F08F
:10C4980033F8C0F38920F6E700287FF4E5AC0321E0
:10C4A800054812F029F8C0B2B5E512689A60B9E5F6
:10C4B8001024B1E564000020681C00200B4611B967
:10C4C80001461846B5E40820704770B5002010F002
:10C4D80073FF064698B901240A4D284612F0ABF8B6
:10C4E800094B02201C60FFF729FC10F0DDFFD5E99D
:10C4F800151230462B6E10F07FFE204670BD0020CE
:10C50800FCE700BF681C00206400002038B50D4619
:10C51800044648B910F034FF2B68C118296020463A
:10C5280010F006FE204638BD0820FCE707B501924A
:10C5380039B9014601AA0120FFF77BFC03B05DF879
:10C5480004FB0820FAE7022806D3052801D9182891
:10C5580002D100201060704704207047044B084641
:10C568009B6E114603B11847024B9B6EDB68FAE7D6
:10C5780000610020681C00202DE9F04101274B4C88
:10C588004B4D4C4BDFF8808100211F60D4F8882088
:10C598002846494B11F0D4FFD8F80C60736803F1B2
:10C5A800C802EA6503F1E40203F5B8702A6603F5E8
:10C5B800C67203F50D732B653368AA65DB68686579
:10C5C80098473368A86DDB6898473368E86DDB687F
:10C5D80098473368286E1B6998473368286DDB686D
:10C5E80098477068336820309B6868669847D8F821
:10C5F800103003F11402AA662A6D9A6105232B7183
:10C608004FF47A73AB6010F04FFFD5E915122B6E1B
:10C61800002010F0F1FDD4F88830284A0220C3F831
:10C628000822274AC3F8042200225A701A70254BA0
:10C638003222C4F89430244B84F88470C4F89030C3
:10C64800224BC4F88C30224BC4F89830214BC4F8E4
:10C65800AC30214BC4F8A830204BC4F89C30204B98
:10C66800C4F8A0301F4BC4F8BC301F4BC4F8B83016
:10C678001E4BC4F8C8301E4BC4F8C4301D4BC4F858
:10C68800C0301D4BC4F8D4304FF41673C4E91F32C0
:10C698001A4BC4F8CC301A4BC4F8E030194BC4F824
:10C6A800E430BDE8F041FFF749BB00BF006100205E
:10C6B800681C002064000020487602083BBD000882
:10C6C800D3C4000815BE000839BE000835BE0008EE
:10C6D80031BE0008C5C4000835C5000829BD0008DA
:10C6E80015C5000831BC00081DBC00083DBC000889
:10C6F800D9BB0008FFBD000845BD000885BD00087E
:10C708004FC50008D5BD000870860208012810B57D
:10C7180014460CD003D3022810D0042006E0136876
:10C72800094AB3FA83F35B099372002010BD1368BA
:10C73800064AB3FA83F35B091360F6E7084610F07C
:10C7480037FD2060F1E700BFE01C00206C000020EE
:10C7580010B5044618B910F0EBFC204610BD0820AF
:10C76800FCE7024B986C12F036B800BFE01C0020C2
:10C77800022804BF0B4B93F8E80030B90A4BDB687A
:10C788001B685B69094A906D1847012809D1054B58
:10C7980093F8E830012B04D1034BDB681B689B69D5
:10C7A800F0E770470061002070860208E01C002056
:10C7B80038B50020FFF7DCFF0F4B104CDD68A06D8B
:10C7C8002B685B6998472B68E06C9B6898472B68D7
:10C7D800606D9B6898472B68A06D9B6898472B688D
:10C7E800E06D9B6898472B68206D9B689847BDE86B
:10C7F800384010F0CDBE00BF70860208E01C002053
:10C8080038B50D46044620B910F0D6FD28602046FC
:10C8180038BD0820FCE710B5044628B9034B188139
:10C8280010F064FC204610BD0820FCE7E01C002046
:10C838000021F0E74942EEE7EDE770B5002010F07F
:10C84800BBFD0646A0B901240A4DA96C284611F083
:10C85800A5FF094B02201C60FFF78AFF10F024FE99
:10C86800D5E914123046EB6D10F0C6FC204670BDB9
:10C878000020FCE7E01C00206C00002038B50D46C5
:10C88800044648B910F07CFD2B68C1182960204681
:10C8980010F04EFC204638BD0820FCE738B51F4C88
:10C8A8000546636E00219B68C0F30740984794F8DB
:10C8B8006820A36C000203EB82035860636E0021BA
:10C8C8009B68C5F30720984794F86830A26C01214B
:10C8D80002EB830253681843636E000250609B6842
:10C8E800E8B29847A26C94F8681002EB81014B6893
:10C8F80018430011AB0C486010610AD0C5F34243DD
:10C90800072B03D1C5F3011184F8681043F008031D
:10C9180000E0082302EB83035D6038BDE01C0020C3
:10C9280010B40A4C00F07702A36C42F0080203EB43
:10C938008203C1F313015960A37A23B941EA404045
:10C9480010BCFFF7ABBF10BC704700BFE01C002055
:10C9580008461146E4E738B504460F2000F013F8FE
:10C968000323B4FBF3F3054603EB4303E41AE4B2F1
:10C9780020F0300040EA0410FFF790FF2846BDE899
:10C988003840FFF78BBF38B5074D0446AA7A1AB965
:10C99800030701D4FFF7DFFFAB6C04F07F0403EB60
:10C9A8008404606838BD00BFE01C0020A72970B56A
:10C9B8000446154600F0F58164D81D2900F0F4807E
:10C9C80021D8042900F0F7800CD8012900F0D9807B
:10C9D800C0F0CB80022900F0DD80032900F0E4805C
:10C9E8000424C6E0062900F0FB80C0F0F080072987
:10C9F80000F010810829F3D10028F1D110F0D8FBFC
:10CA0800C0F30010B4E0A12900F077811AD83329C7
:10CA180000F01B8108D83229E2D1002840F01081AB
:10CA2800002010F00FFDA3E08C2900F01781A02949
:10CA3800D6D10820002C40F05781FFF7A4FFC0F39F
:10CA4800402095E0A42900F083810DD8A22900F0A8
:10CA58006481A329C4D10C20002C40F07081FFF719
:10CA680092FFC0F3803083E0A52900F08181A629D8
:10CA7800B6D10C20002C40F08B81FFF784FFC0F367
:10CA8800021075E0B22900F02F823ED8AC2900F0E0
:10CA9800D78112D8A92900F0A781C0F09181AA29CD
:10CAA80000F0B381AB299BD1002840F0BF8105205D
:10CAB800FFF769FFC0F341105AE0AF2900F0E781A2
:10CAC80014D8AD2900F0C881AE2989D1002840F0DA
:10CAD800D4810620FFF757FF000A00F07F0310F00B
:10CAE800400018BF6FF07F00184341E0B02900F004
:10CAF800E081B1297FF474AF002840F0EB81072072
:10CB0800FFF741FFC0F3802032E0B72900F024820C
:10CB180010D8B42900F00A82C0F0F781B52900F0D6
:10CB28000E82B6297FF45CAFAE4B002840F011822C
:10CB38001B6958E0CE2900F03A820AD8B82900F0DB
:10CB48001B82B9297FF44CAF002840F026820720C9
:10CB580084E1D02900F03F82D6297FF441AFA14B70
:10CB6800002840F040825B683DE020B910F016FCD8
:10CB78002860204670BD1168002010F0D9FA002402
:10CB8800F7E710B910F0FCFBF2E71168002010F08D
:10CB9800A9FBF4E718B9002010F01CFCE8E71168BD
:10CBA800002010F0A3FAEAE7002C7FF419AF204622
:10CBB80010F002FCDCE710B910F028FCD8E7116887
:10CBC80000200029B8BF494210F0A6FBD7E710B9EA
:10CBD80010F00EFCCCE71168002010F000FDCEE745
:10CBE800804E10B9F37A2B60C3E713680020F37204
:10CBF800FFF7C9FE10F08004C1D10E20FFF7C3FE75
:10CC0800F37A20F01F0103F01F0319430E20FFF7EA
:10CC180087FEAEE7734E08B93378E4E7136800205F
:10CC28003370FFF7B0FE0306A9D50E20FFF7ABFE61
:10CC3800337820F01F0103F01F0319430E2046E04C
:10CC48001178002010F082FB99E710B910F008FC69
:10CC58008EE71168002010F089FB90E738B90820AA
:10CC6800FFF791FE00F00F00C0F1080080E713689D
:10CC7800102B33D00DDC022B2CD004DC012B16D06A
:10CC88004FF0FF3314E0042B26D0082BF8D10523EE
:10CC98000EE0402B24D003DC202BF1D1032307E046
:10CCA800802B1FD0B3F5807FEAD1002300E0082352
:10CCB8002B602B68013300F099810820FFF763FE91
:10CCC8002B6820F00F0103F00F0308201943FFF72A
:10CCD80027FE54E70723EBE70623E9E70423E7E702
:10CCE8000223E5E70123E3E7FFF74DFE2B6820F475
:10CCF80000715B0203F40073E7E7082024B9FFF72B
:10CD080042FEC0F3002033E7FFF73DFE2B6820F416
:10CD180080711B0203F48073D7E70C2024B9FFF756
:10CD280032FEC0F3C13023E7FFF72DFE2B6820F455
:10CD3800C031DB0303F4C03319430C20C7E7FFF706
:10CD480022FE2B6820F480419B0303F48043F3E721
:10CD58000C2024B9FFF717FEC0F3C12008E7FFF73E
:10CD680012FE2B6820F4C051DB0203F4C053E3E742
:10CD78000C2024B9FFF707FEC0F3C310F8E6FFF74D
:10CD880002FE2B6820F4F061DB0103F4F063D3E7C3
:10CD9800FFF7F9FD2B6820F070011B0103F0700309
:10CDA800CAE70C2024B9FFF7EEFD00F00F00DFE61C
:10CDB800FFF7E9FD2B6820F00F0103F00F03BBE735
:10CDC80028B90520FFF7DFFDC0F3C030D0E60D20FD
:10CDD800FFF7D9FD2B6820F40041DB039BB2194310
:10CDE8000D2074E7E01C002028B90520FFF7CBFDD3
:10CDF800C0F34130BCE60D20FFF7C5FD2B6820F4D9
:10CE0800C0415B0303F4C043E9E728B90520FFF7F5
:10CE1800BAFDC0F30320ABE60D20FFF7B4FD2B6885
:10CE280020F470611B0203F47063D8E70D20FFF74C
:10CE3800AAFD2B6820F060015B0103F06003CEE7D8
:10CE480008B90520AFE70D20FFF79DFD2B6820F0FE
:10CE58000F0103F00F03C2E728B90620FFF793FD7F
:10CE6800C0F3004084E60E20FFF78DFD2B6820F408
:10CE780080311B0403F48033DFE60E20FFF783FDC7
:10CE88002B6820F4FE411B0203F4FE43D5E628B9C3
:10CE98000720FFF778FDC0F3813069E60F20FFF720
:10CEA80072FD2B6820F440419B039BB219430F206D
:10CEB8000DE728B90720FFF766FDC0F3013057E6F4
:10CEC8000F20FFF760FD2B6820F440511B0303F48B
:10CED8004053EBE70F20FFF756FD2B6820F48061E5
:10CEE8009B0203F48063E1E728B90720FFF74BFDB5
:10CEF800C0F301203CE60F20FFF745FD2B6820F426
:10CF080040711B0203F44073D0E728B90720FFF7EC
:10CF18003AFDC0F380102BE60F20FFF734FD2B6895
:10CF280020F040019B0103F04003BFE700287FF495
:10CF380057AD0220FFF727FDC0F3842018E618B983
:10CF4800002010F071FA13E61168002010F0F0F9D3
:10CF580015E612681A6112E628B90720FFF713FDD3
:10CF6800C0F3C01004E60F20FFF70DFD2B6820F07A
:10CF78008001DB01DBB299E728B90420FFF703FD44
:10CF8800C0F34030F4E50C20FFF7FDFC2B6820F4DB
:10CF980000515B0303F40053CEE60F20FFF7F3FCC8
:10CFA8002B6820F480311B0403F480337EE70028CB
:10CFB8007FF416AD0E4B1B683BB10220FFF7E3FC74
:10CFC800800A00F478702860D9E50120FFF7DBFCBF
:10CFD800C0F38920F7E700287FF402AD0320FFF7AC
:10CFE800D2FCC0B2C4E512685A60C8E51024C0E596
:10CFF8006C0000200B4611B901461846D6E40820FB
:10D00800704707B5019239B9014601AA0120FFF717
:10D01800CDFC03B05DF804FB0820FAE710B508461C
:10D028001446FFF7B0FC206010BDF8B50646002096
:10D03800FFF7A9FC324CC0F3C01594F86930AB4235
:10D0480015D00E20002D4BD0FFF79DFC00F01F00DF
:10D05800E0720E20FFF797FC237803F01F0320F0FF
:10D068001F0119430E20FFF75BFC84F86950254A1D
:10D07800217A936F00293DD043F00103617A00299A
:10D088003BD043F002030020936710F095F9236921
:10D098000028B8BF4042984234BF0027012794F8BF
:10D0A8006A20BA4211D098424FF00D002CBF657B20
:10D0B800257BFFF768FC05F00F0520F00F012943D9
:10D0C8000D20FFF72DFC84F86A70A36C3146002010
:10D0D8000B4A11F00EFBBDE8F840002010F0E4B850
:10D0E800FFF751FC00F01F0020700E20FFF74BFCEB
:10D0F800E37AB2E723F00103C0E723F00203C2E7B3
:10D10800E01C0020006100200A4810B4836C01F084
:10D11800770444F0080403EB8403C2F313025A6053
:10D12800837A23B942EA414010BCFFF7B7BB10BC71
:10D13800704700BFE01C002038B5084D0C46AA7A9D
:10D1480022B90B0702D40846FFF705FCA96C04F0C6
:10D158007F0401EB8404606838BD00BFE01C002038
:10D1680038B50D461E4C0021636EC5F307409B6819
:10D17800984794F86B20A36C000203EB8203586075
:10D18800636E00219B68C5F30720984794F86B30BD
:10D19800A26C012102EB830253681843636E0002FC
:10D1A80050609B68E8B29847A26C94F86B1002EB49
:10D1B80081014B6818430011AB0C486010610AD01C
:10D1C800C5F34243072B03D1C5F3011184F86B1053
:10D1D80043F0080300E0082302EB83035D6038BDD9
:10D1E800E01C0020F8B50126444C454B454F20462D
:10D1F8001E6011F05DFAFD686B6803F1C802A26554
:10D2080003F1E40203F5B870E26503F5C67203F5AD
:10D218000D73E3642B686265DB68206598472B68AB
:10D22800606DDB6898472B68A06DDB6898472B68B2
:10D23800E06D1B6998472B68E06CDB689847686865
:10D248002B6820309B68206698473B6903F11402DD
:10D258006266E26C9A61052323704FF47A73636007
:10D2680010F022F9D4E91412E36D00200FF0C4FF86
:10D27800254B2649D3F888200220C2F808122449F1
:10D28800A264C2F80412002151701170214A32219F
:10D29800C3F89420204A83F88460C3F890201F4A7A
:10D2A800C3F88C201E4AC3F898201E4AC3F8AC2045
:10D2B8001D4AC3F8A8201D4AC3F89C201C4AC3F87D
:10D2C800A0201C4AC3F8BC201B4AC3F8B8201B4A3C
:10D2D800C3F8C8201A4AC3F8C4201A4AC3F8C020A1
:10D2E800194AC3F8D4204FF41672C3E91F21174A0C
:10D2F800C3F8CC20BDE8F840FFF73ABAE01C00209C
:10D308006C00002070860208006100206BC70008CE
:10D3180043C800081FC8000841C800083DC80008E5
:10D3280039C80008FDCF00080BD0000859C700080D
:10D3380085C8000859C9000825D0000833D000085E
:10D3480015C7000809C8000879C70008B9C7000848
:10D358000022014B5A6070470061002070B5184EDA
:10D36800184CF56860682B689B6998472B68A0691A
:10D378009B6898472B6860699B6898472B68206969
:10D388009B6898472B68E0689B6898472B68A0685B
:10D398009B6898472B68206A9B6898472B68E069C8
:10D3A8009B6898472B6820689B6898472B6860683B
:10D3B8009B6898473369BDE870405B6A184700BFAF
:10D3C80070860208581D0020022870B5144649D0FE
:10D3D80004D890B1012836D0042432E003284FD075
:10D3E800FF28F9D12B4CD4F88830D3F80432984769
:10D3F8006369D3F80432984703E0126832F00303F4
:10D4080001D000241DE0244B244DDE68D207686952
:10D4180033680AD51B6998472468326814F00204F7
:10D42800A86908D013699847EBE7DB689847336821
:10D4380068699B69EFE7D36898473368A8699B696F
:10D448009847204670BD144B144DDE68146828694F
:10D4580033680CB11B69E6E7DB68984733682869CD
:10D468009B69EDE70C4B0D4DDE6814683368A868BE
:10D47800002CEFD1DB6898473368A8689B69DFE721
:10D488000121074811F0DAFA20600028B9D12024D8
:10D49800D7E700BF0061002070860208581D0020F1
:10D4A8007C1D00200146014811F07EBB7C1D002038
:10D4B80010B50348144611F0F0F9206010BD00BF04
:10D4C8007C1D0020014811F0DAB900BF7C1D002046
:10D4D80008B50448D0F8B822243011F09FFA00208B
:10D4E80008BD00BF581D002008B50448D0F8B82270
:10D4F800243011F077FA002008BD00BF581D002025
:10D5080008B50021024811F04FFA002008BD00BFFD
:10D518007C1D002008B54942024811F045FA002058
:10D5280008BD00BF7C1D002008B5024811F03CFA78
:10D53800002008BD7C1D002038B50A4B0A4CDD6868
:10D5480060682B689B69984701200CF0FFFE2B68E8
:10D5580060685B69984704F1240011F0FAF901202A
:10D5680038BD00BF70860208581D002038B50A4B28
:10D578000A4CDD6860682B689B69984701200CF0AD
:10D58800E5FE2B6860685B69984704F1240011F098
:10D59800CBF9012038BD00BF70860208581D002055
:10D5A8006E2970B50446154600F0BB8170D8122963
:10D5B80000F06C8138D8052900F0298118D8022993
:10D5C80000F0018107D8002900F0E880012900F067
:10D5D800F4800424E8E0032900F002810429F8D14A
:10D5E800B64E002840F00181D6F8B8322B60DBE057
:10D5F8000F2900F030810DD8082900F01B810E2971
:10D60800E7D1002840F020812021AD4811F045F9EC
:10D618004000C8E0102900F024811129D9D1002840
:10D6280040F02B812921F4E0182900F05C8117D8FB
:10D63800152900F0408109D8132900F02D811429FB
:10D64800C7D1002840F034812621A9E0162900F02E
:10D6580041811729BDD1002840F042812E219FE049
:10D668001B2900F04F8109D8192900F042811A2995
:10D67800AFD1002840F04381332191E06C2900F0BC
:10D6880047816D29A5D1002840F04881612187E0B4
:10D698007E2900F0B0813CD8742900F0798119D82E
:10D6A800712963D009D86F2900F04B81702990D176
:10D6B800002840F05681592172E0722900F0548107
:10D6C800732986D1002840F060817C4B5B6AD3F8CF
:10D6D8006C318BE7772900F07F810FD8752900F02E
:10D6E800608176297FF475AF7448436AD3F8702156
:10D6F800002C40F06781C2F307422BE07C2900F040
:10D7080071817D297FF465AF002840F071815F2128
:10D7180046E0892900F0B2811ED8852900F093815E
:10D728000AD8812900F0788184297FF452AF002833
:10D738007FF44FAF652133E0862900F09181882975
:10D748007FF447AF5D48436AD3F89021002C40F03E
:10D758008D81D2B22A6027E0D12900F0AE8112D89B
:10D768008A2900F09A81C8297FF433AF05215448EB
:10D77800002C00F0E98011F090F82A7820F0FF00E2
:10D788000243052114E0D42900F09D81D6297FF4B5
:10D7980020AF002840F09F81152101E030B93721E2
:10D7A800474811F07AF82860204670BD3721126882
:10D7B800434811F064F80024F6E708B92121EFE79F
:10D7C80012682121F4E728B924213D4811F065F8B1
:10D7D8000012E8E7106811F0D5F824210246E7E7BF
:10D7E80000287FF4F6AE2221DAE71368202106F13B
:10D7F8002400C6F8B83211F050F84207DBD5D6F845
:10D80800B80211F0BFF8242102467018D1E728B9F0
:10D8180028212B4811F041F88010C4E71268940DB4
:10D82800A405002C40F05C8128219200244811F0C6
:10D8380026F8B9E700287FF4CCAE0F21204811F074
:10D848002CF800F00100AEE713682021002B0CBF74
:10D8580001220222ACE708B92521A1E71268252197
:10D86800A6E708B92A21D4E71268940DA405002C6C
:10D8780040F0368192002A21D8E71268940DA40559
:10D88800002C40F02D8192002921CFE708B92721EB
:10D8980086E7126827218BE708B92B21B9E71268B8
:10D8A800940DA405002C40F01B8192002B21BDE7AC
:10D8B800126826217CE728B92C2171E7581D002021
:10D8C8007C1D00201268940DA405002C40F00881EE
:10D8D8002C21ABE708B92D2162E712682D2167E7F3
:10D8E80012682E2164E708B92F2159E712682F2101
:10D8F8005EE708B9302153E71268302158E712680B
:10D90800332155E708B934214AE7126834214FE733
:10D9180008B9602144E71268602149E7126861216B
:10D9280046E71C216F481CB910F0B7FF00143AE70E
:10D9380010F0B3FF2A68C0F3080040EA02421C2135
:10D9480036E71C2167481CB910F0A7FFC0B22AE7C8
:10D9580010F0A3FF2B6800F47F02C3F308031A43F7
:10D96800EDE71268592123E705215E4824B910F034
:10D9780094FFC0F3072016E710F08FFF2B6820F400
:10D988007F421B029BB21A43FBE612685A210FE73B
:10D9980020B9554B5B6AD3F8703127E612685B21D2
:10D9A80006E7514B5B6AD3F8703110B9C3F30E0325
:10D9B8001CE6126823F4FF4323F07F03C2F30E0230
:10D9C8001A43ECE75B212B6822F47F021B0403F463
:10D9D8007F031A432430ECE608B95E21E0E61268BA
:10D9E8005E21E5E608B95C21DAE612685C21DFE62B
:10D9F80012685F21DCE605213A4824B910F04DFF92
:10DA0800C0F30740CFE610F048FF2B6820F47F02F0
:10DA18001B0403F47F03B6E700283FF4CCAE146878
:10DA28004CB101212F4811F009F8286000287FF433
:10DA3800C2AE2024B8E607212A4810F02EFF07219D
:10DA480020F48002F2E600287FF4B5AE07212548CD
:10DA580010F023FFC0F38150431E58425841A2E6FC
:10DA680008B952219CE612685221A1E62B6822F0DF
:10DA7800FF0203F00F031A436321ABE71A48436A16
:10DA8800D3F8902114B9C2F3032263E62B6822F479
:10DA980070621B0203F47063EDE7134B5B6AD3F803
:10DAA800902100283FF427AE2B6822F47F021B0444
:10DAB80003F47F031A4363217AE608B950216FE61D
:10DAC8001268502174E618B9074B5B6A9B698DE5AB
:10DAD800126853216CE61368044A15215A4367E615
:10DAE800102461E67C1D0020581D002000710200F2
:10DAF8000B4611B90146184652E50820704708B58B
:10DB0800024810F051FF002008BD00BF7C1D002016
:10DB180007B5019239B9014601AA0120FFF740FD76
:10DB280003B05DF804FB0820FAE7034B0846D3F876
:10DB3800BC321146DB681847581D0020F8B5494C1F
:10DB4800494D4A4F00214A4B6A6904F1240010F0FC
:10DB5800CDFEFE68736803F59C72226203F5AA7213
:10DB6800E26103F55372A26103F55A72626103F52B
:10DB78006172226103F5687203F57670E26003F55D
:10DB88006F7203F57D7323603368A260DB686060A1
:10DB980098473368A069DB68984733686069DB6831
:10DBA800984733682069DB6898473368E068DB6822
:10DBB80098473368A068DB689847336860685B6992
:10DBC80098473368A0695B699847336860695B69FF
:10DBD8009847336820695B6998473368E0685B69F0
:10DBE80098473368A0685B6998473368206A1B695F
:10DBF80098473368E0691B699847336820681B6950
:10DC08009847002173683A6903F537735360C4F87D
:10DC1800BC2201226B69597016491A70C3F80412A4
:10DC280015492A74C3F80812144B2B62144BEB6184
:10DC3800144BAB61144B6B62144BAB63144B6B63AB
:10DC4800144BAB62144BEB62144BAB64144B6B6418
:10DC5800144B6B65144B2B65144BEB65144BAB6580
:10DC6800F8BD00BF581D0020006100207086020822
:10DC78006876020875D5000841D5000807DB00085A
:10DC880031D500081DD5000809D50008F9DA0008C3
:10DC980019DB0008F1D40008D9D40008CDD4000855
:10DCA800B9D40008ADD40008D1D3000859D300086E
:10DCB80065D300080022014B5A60704700610020BC
:10DCC800022870B5144648D004D8A0B1012835D030
:10DCD80004200FE003280CD0FF28F9D1264CD4F8F3
:10DCE8008830D3F8043298476369D3F804329847E8
:10DCF80016E0202070BD126832F00303FAD11F4BE2
:10DD08001F4DDE68D207686933680BD51B699847D1
:10DD18002468326814F00204A86909D01369984786
:10DD28000020E7E7DB689847336868699B69EEE796
:10DD3800D36898473368A8699B69F0E70F4B104D83
:10DD4800DE681468286933680CB11B69E7E7DB688B
:10DD58009847336828699B69E1E7084B084DDE68F6
:10DD680014683368A868002CEFD1DB6898473368DB
:10DD7800A8689B69D3E700BF00610020708602088D
:10DD88002820002070B5184E184CF56860682B687C
:10DD98009B6998472B68A0699B6898472B686069BE
:10DDA8009B6898472B6820699B6898472B68E068B0
:10DDB8009B6898472B68A0689B6898472B68206ADF
:10DDC8009B6898472B68E0699B6898472B68206890
:10DDD8009B6898472B6860689B6898473369BDE8DB
:10DDE80070405B6A184700BF708602082820002030
:10DDF8000A460146014810F08BBF00BF4C200020A6
:10DE08000146014811F03AB84C20002010B50348EB
:10DE1800144610F054FF206010BD00BF4C200020B5
:10DE28006C2938B50C4615460BD06D2902D10A4B22
:10DE3800C3F8B8222A462146BDE83840074810F002
:10DE480030BF054BD3F8B812054B01F07F01D3F86A
:10DE5800BC309847EEE700BF282000204C20002067
:10DE68000061002008B50448D0F8BC22243011F025
:10DE780093F8002008BD00BF2820002008B50448FA
:10DE8800D0F8BC22243011F06BF8002008BD00BF88
:10DE98002820002008B50021024811F043F800208E
:10DEA80008BD00BF4C20002008B54942024811F0C7
:10DEB80039F8002008BD00BF4C20002008B50248F2
:10DEC80011F030F8002008BD4C20002038B50A4B6E
:10DED8000A4CDD6860682B689B69984701200CF044
:10DEE80035FA2B6860685B69984704F1240010F0E4
:10DEF800ACFF012038BD00BF708602082820002032
:10DF080038B50A4B0A4CDD6860682B689B699847EE
:10DF180001200CF01BFA2B6860685B69984704F1D4
:10DF2800240010F07DFF012038BD00BF7086020874
:10DF38002820002070B5114C0D4694F87430012B40
:10DF480019D0032B0BBF002228220C230F2343F0E8
:10DF5800884343F0401343EA4232042110F0A1FE03
:10DF6800D4F88830012D0CBFD3F80432D3F8083226
:10DF7800BDE87040184700220B23E8E70061002045
:10DF88002DE9F84F0027424CD4F8C462D4F8C052A7
:10DF98004FEA062949EA1569C6B24FEA052894F8F6
:10DFA800C802D4F8D45248EA0602D4F8D06249EA42
:10DFB800070301302F0E2D0245EA166504F5307C63
:10DFC8003602C0B204F5347EC4F8D062C4F8D45224
:10DFD800CCE9002384F8C80266467546002954D067
:10DFE800042805D91A466D2104F1240010F059FEC1
:10DFF8004FF0000BD4F8C0226C21264810F051FED7
:10E0080001200CF0A3F9D4F8C0226C21214810F0AB
:10E0180048FE94F8C832C5E900BB042B0CD96F211F
:10E028001C4810F04CFED5E90023814642EA0B005B
:10E0380043EA0901C5E900016E21164810F03FFEC8
:10E04800D5E9002342EA000843EAE079404694F81B
:10E05800C832C3F10803DB00A3F1200EC3F1200C82
:10E0680009FA03F208FA0EFE42EA0E0228FA0CFC3C
:10E0780042EA0C0298406A6000230022C6E90023A5
:10E088000023C4F8D00284F8C8323846BDE8F88FB7
:10E09800282000204C20002008B5024810F042FF3C
:10E0A800002008BD4C20002038B515460C46002934
:10E0B8007BD1112869D01FD804284ED008D8012850
:10E0C80040D03AD302283FD0032844D0042448E063
:10E0D8000E284ED00AD8052845D00828F6D10F2199
:10E0E800334810F0ECFD00F0010032E00F284AD070
:10E0F8001028EBD12A2137E017284ED00ED8142843
:10E1080047D005D8122842D01328DFD12B212BE085
:10E11800152840D01628D9D12D210FE01A2840D033
:10E1280005D818283BD01928D0D1302106E01B2863
:10E1380039D0D628CAD1152100E037211C4810F063
:10E14800BEFD06E02121F9E72421194810F0B7FDAA
:10E158000012286005E02221F0E7164BD3F8BC3204
:10E168001360204638BD2821114810F0A8FD801002
:10E17800EFE720210E4810F0A2FD00F00300831EF7
:10E1880058425841E5E72521D8E72921ECE727211E
:10E19800D4E72621D2E72C21D0E72E21CEE72F2164
:10E1A800CCE73321CAE73421C8E70824D9E700BF00
:10E1B8004C2000202820002038B514460D460029A0
:10E1C80040F08B80122871D022D8052860D008D85A
:10E1D800012840D039D302283FD0042843D0042551
:10E1E80037E00F285AD007D80E28F8D1002A14BFD4
:10E1F80002220122202129E0102851D01128EED135
:10E20800930D9B05002B6AD19200292135483BE0EC
:10E2180017285AD008D8142850D049D315284FD0D9
:10E228001628DCD12D2111E01A2852D005D818283B
:10E238004DD01928D3D1302108E01B284BD0D6283F
:10E24800CDD1294A1521624300E03721254810F035
:10E2580028FD284638BD2121F8E782EAE272A2EBC0
:10E26800E4722421F2E7214D202105F12400C5F8AC
:10E27800BC2210F024FD430708D5D5F8BC0210F0E5
:10E288003FFE24210246681810F00BFD0025E0E748
:10E29800950DAD051DBB92002821D7E72521D5E7AF
:10E2A800950DAD05DDB992002A21CFE72721CDE7ED
:10E2B800950DAD059DB992002B21C7E72621C5E72D
:10E2C800950DAD055DB92C21C0E72E21BEE72F21A4
:10E2D800BCE73321BAE73421B8E70825B9E71025A8
:10E2E800B7E700BF4C200020007102002820002062
:10E2F800034B0846D3F8D8321146DB68184700BFED
:10E3080028200020F8B54D4C4D4D04F124064D4B06
:10E318006A69304600214C4F10F065FD4B49304684
:10E3280010F0A8FDFE68736803F59C72226203F57D
:10E33800AA72E26103F55372A26103F55A7262612F
:10E3480003F56172226103F5687203F57670E26085
:10E3580003F56F7203F57D7323603368A260DB6891
:10E36800606098473368A069DB68984733686069DC
:10E37800DB68984733682069DB6898473368E0684A
:10E38800DB6898473368A068DB689847336860683B
:10E398005B6998473368A0695B6998473368606927
:10E3A8005B699847336820695B6998473368E06818
:10E3B8005B6998473368A0685B6998473368206A47
:10E3C8001B6998473368E0691B6998473368206878
:10E3D8001B699847002173683A6903F537735360DE
:10E3E800C4F8D82201226B69597019491A70C3F808
:10E3F800041218492A74C3F80812174B6B66174B96
:10E408002B62174BEB61174BAB61174B6B62174BCA
:10E41800AB63174B6B63174BAB62174BEB62174B36
:10E42800AB64174B6B64174B6B65174B2B65174B1E
:10E43800EB65174BAB65174BAB66F8BD2820002082
:10E448000061002068780208708602083DDF000835
:10E4580009DF0008D5DE000889DF0008A1E0000810
:10E46800C5DE0008B1DE00089DDE0008B1E0000846
:10E47800C1E1000885DE00086DDE000829DE00081D
:10E4880015DE000809DE0008C9DC0008BDDC00084C
:10E498008DDD0008F9DD00080022014B5A60704745
:10E4A8000061002070B5184E184CF56860682B683C
:10E4B8009B6998472B68A0699B6898472B68606997
:10E4C8009B6898472B6820699B6898472B68E06889
:10E4D8009B6898472B68A0689B6898472B68206AB8
:10E4E8009B6898472B68E0699B6898472B68206869
:10E4F8009B6898472B6860689B6898473369BDE8B4
:10E5080070405B6A184700BF70860208102300201D
:10E518000A460146014810F0BDBD00BF3423002063
:10E52800022870B5144649D004D890B1012836D0D5
:10E53800042432E003284FD0FF28F9D12B4CD4F81B
:10E548008830D3F8043298476369D3F8043298477F
:10E5580003E0126832F0030301D000241DE0244BCD
:10E56800244DDE68D207686933680AD51B69984765
:10E578002468326814F00204A86908D0136998471F
:10E58800EBE7DB689847336868699B69EFE7D3680E
:10E5980098473368A8699B699847204670BD144B13
:10E5A800144DDE681468286933680CB11B69E6E706
:10E5B800DB689847336828699B69EDE70C4B0D4D7C
:10E5C800DE6814683368A868002CEFD1DB689847C8
:10E5D8003368A8689B69DFE70121074810F06EFEE1
:10E5E80020600028B9D12024D7E700BF00610020AF
:10E5F80070860208102300203423002001460148B9
:10E6080010F012BF3423002010B50348144610F050
:10E6180018FD206010BD00BF342300206C2938B5D8
:10E628000C4615460BD06D2902D10A4BC3F8B82207
:10E638002A462146BDE83840074810F0F4BC054B8F
:10E64800D3F8B812054B01F07F01D3F8BC309847D6
:10E65800EEE700BF102300203423002000610020D3
:10E6680008B50448D0F8BC22243010F017FE00206A
:10E6780008BD00BF1023002008B50448D0F8BC220C
:10E68800243010F0EFFD002008BD00BF102300204B
:10E6980008B50021024810F0C7FD002008BD00BFE2
:10E6A8003423002008B54942024810F0BDFD00207F
:10E6B80008BD00BF3423002008B5024810F0B4FD9F
:10E6C800002008BD3423002038B50A4B0A4CDD6809
:10E6D80060682B689B69984701200BF037FE2B6810
:10E6E80060685B69984704F1240010F072FD01200E
:10E6F80038BD00BF708602081023002038B50A4BC9
:10E708000A4CDD6860682B689B69984701200BF00C
:10E718001DFE2B6860685B69984704F1240010F0BF
:10E7280043FD012038BD00BF708602081023002079
:10E7380070B5114C0D4694F87430012B19D0032B89
:10E748000BBF002228220C230F2343F0884343F0F9
:10E75800401343EA4232042110F065FCD4F88830B3
:10E76800012D0CBFD3F80432D3F80832BDE870404D
:10E77800184700220B23E8E7006100206F2970B5D5
:10E788000446154600F0818200F28980122900F0C3
:10E79800D1813ED8052900F0718118D8022900F0EE
:10E7A8003B8107D8002900F01A81012900F0268151
:10E7B80004241AE1032900F041810429F8D1B94E53
:10E7C800002840F04481D6F8BC3213600DE10F29CF
:10E7D80000F082810ED8082900F068810E29E7D15F
:10E7E800002840F06E812021AF4810F02AFC40003C
:10E7F8002860FAE0102900F07D811129D8D100287D
:10E8080040F08C812921A84810F01BFC801028605A
:10E81800EBE0182900F0DE811FD8152900F0B3813C
:10E828000DD8132900F094811429C1D1002840F093
:10E83800A38126219C4810F004FC2860D5E0162905
:10E8480000F0B3811729B3D1002840F0BC812E21F4
:10E85800954810F0F6FB2860C7E01B2900F0DD8121
:10E868000DD8192900F0C4811A29A1D1002840F037
:10E87800CD8133218C4810F0E4FB2860B5E06D2988
:10E8880000F0E08100F2EC816C2991D1002840F081
:10E89800D2816021844810F0D4FB2860A5E07D294E
:10E8A80000F0AB8248D8752900F0508222D872292E
:10E8B80000F01B820FD8702900F0FD8171297FF4C8
:10E8C80077AF06217848002C40F0038210F0B9FB9E
:10E8D800C0B2286089E0732900F01E8274297FF491
:10E8E80067AF002840F026826E4B5B6AD3F8703120
:10E8F80013607AE0782900F05D820ED8762900F05E
:10E908003C8277297FF454AF002840F04C825E2186
:10E91800654810F096FB286067E0792900F0588276
:10E928007C297FF445AF002840F060825C215E4876
:10E9380010F087FB286058E0882900F0AD8228D8BD
:10E94800842900F08B8215D87E2900F06482812901
:10E958007FF42EAF002800F084801468002C00F0AB
:10E9680072820121504810F0A9FC2860002878D153
:10E9780020243AE0852900F07A8286297FF418AFAE
:10E98800002840F082825221474810F05AFB286044
:10E998002BE0C82995D010D8892900F091828A29BE
:10E9A8007FF406AF3F48436AD3F89021002C40F02B
:10E9B8009D82C2F307422A6017E0D42900F0AA8298
:10E9C800D62900F0B482D1297FF4F2AE002840F0B5
:10E9D8009A825021344810F034FB286005E030B9A1
:10E9E8003721314810F02DFB2860204670BD126891
:10E9F80037212D4810F017FB0024F6E728B921210C
:10EA0800294810F01EFB2860EFE7126821212648EC
:10EA180010F009FB0024E8E730B92421224810F05F
:10EA280010FB00122860E0E7106810F0EBFB2421CF
:10EA380002461D4810F0F7FA0024D6E7002840F0F7
:10EA480086822221184810F0FCFA2860CDE7136866
:10EA5800202106F12400C6F8BC3210F0F2FA420771
:10EA680001D40024C1E7D6F8BC0210F0CBFB242166
:10EA78000246701810F0D7FA0024B6E730B92821FA
:10EA8800094810F0DEFA80102860AEE71268940D8D
:10EA9800A405002C40F05D8292002821024810F065
:10EAA800C2FAA2E71023002034230020002840F0F7
:10EAB80052820F21A34810F0C4FA00F00100286028
:10EAC80093E713682021002B0CBF012202229D48E6
:10EAD80010F0A9FA002488E728B92521994810F0F0
:10EAE800B0FA286081E712682521964810F09BFA51
:10EAF80000247AE730B92A21924810F0A2FA80104F
:10EB0800286072E71268940DA405002C40F0258255
:10EB180092002A218B4810F086FA66E71268940D55
:10EB2800A405002C40F01B8292002921854810F092
:10EB38007AFA5AE728B92721824810F082FA286021
:10EB480053E7126827217F4810F06DFA00244CE73C
:10EB580030B92B217B4810F074FA8010286044E704
:10EB68001268940DA405002C40F0FB8192002B2123
:10EB7800744810F058FA38E712682621714810F0E6
:10EB880052FA002431E728B92C216E4810F059FABE
:10EB980028602AE71268940DA405002C40F0E38150
:10EBA8002C21684810F03FFA1FE728B92D21654845
:10EBB80010F047FA286018E712682D21614810F014
:10EBC80032FA002411E712682E215E4810F02BFA61
:10EBD80000240AE728B92F215A4810F032FA286091
:10EBE80003E712682F21574810F01DFA0024FCE6AD
:10EBF80028B93021534810F024FA2860F5E6126845
:10EC08003021504810F00FFA0024EEE61268332144
:10EC18004C4810F008FA0024E7E628B9342149489E
:10EC280010F00FFA2860E0E612683421454810F029
:10EC3800FAF90024D9E612686021424810F0F3F985
:10EC48000024D2E628B961213E4810F0FAF928607C
:10EC5800CBE6126861213B4810F0E5F90024C4E6D0
:10EC68001C21384824B910F0ECF900142860BCE6DF
:10EC780010F0E7F92A68C0F3080040EA02421C21B4
:10EC8800304810F0D0F90024AFE61C212D4824B9F3
:10EC980010F0D7F9C0B22860A7E610F0D2F92B68B7
:10ECA80000F47F02C3F308031A431C21254810F01F
:10ECB800BAF9002499E628B95921224810F0C1F977
:10ECC800286092E6126859211E4810F0ACF9002419
:10ECD8008BE610F0B6F92A7820F0FF0002430621EF
:10ECE800184810F0A0F900247FE6062115482CB931
:10ECF80010F0A7F9C0F30720286076E610F0A1F914
:10ED08002B6820F47F421B029BB21A4306210D4850
:10ED180010F089F9002468E628B90B4B5B6AD3F830
:10ED28006C31136061E612685A21064810F07BF9CD
:10ED380000245AE612685B21024810F074F9002496
:10ED480053E600BF34230020102300208848436A7C
:10ED5800D3F870311CB9C3F30E03136045E612688B
:10ED680023F4FF4323F07F03C2F30E021A435B210F
:10ED7800243010F058F9002437E67D4B5B6AD3F84D
:10ED8800702118B9C2F307422A602EE62B6822F4D4
:10ED98007F021B0403F47F031A435B21754810F0BC
:10EDA80042F9002421E612685E21724810F03BF90E
:10EDB80000241AE628B918216E4810F042F9286094
:10EDC80013E6126818216B4810F02DF900240CE6A0
:10EDD80028B91921674810F034F9286005E6126847
:10EDE8001921644810F01FF90024FEE512685C211F
:10EDF800604810F018F90024F7E528B95F215D484C
:10EE080010F01FF92860F0E512685F21594810F0EA
:10EE18000AF90024E9E5062156482CB910F011F941
:10EE2800C0F307402860E0E510F00BF92B6820F4E8
:10EE38007F021B0403F47F031A4306214D4810F098
:10EE4800F2F80024D1E507214A4810F0FAF8072122
:10EE580020F48002474810F0E6F8C6E5002840F0A4
:10EE680084806521434810F0ECF82860BDE500284F
:10EE78007FF4F7AD07213F4810F0E3F8C0F3815065
:10EE8800431E584258412860AFE51268522139485C
:10EE980010F0C9F80024A8E53548436AD3F8902152
:10EEA80014B9D2B22A60A0E52B6822F0FF0203F061
:10EEB8000F031A436321243010F0B5F8002494E5B9
:10EEC8002B4B5B6AD3F8902118B9C2F303222A604E
:10EED8008BE52B6822F470621B0203F470631A43FB
:10EEE8006321244810F09FF800247EE52B6822F463
:10EEF8007F021B0403F47F031A436321243010F0BC
:10EF080092F8002471E5126850211A4810F08BF825
:10EF180000246AE520B9164B5B6ADB69136064E577
:10EF280012685321134810F07EF800245DE528B9D3
:10EF38001521104810F085F8286056E513680E4A28
:10EF480015215A430B4810F06EF800244DE50424AF
:10EF58004BE5102449E5042447E5102445E5102431
:10EF680043E5102441E510243FE504243DE500BFB6
:10EF78001023002034230020007102000B4619B929
:10EF880001461846FFF7FABB082070472DE9F84FED
:10EF98000027424CD4F8C462D4F8C0524FEA06297C
:10EFA80049EA1569C6B24FEA052894F8C802D4F8A8
:10EFB800D45248EA0602D4F8D06249EA070301307D
:10EFC8002F0E2D0245EA166504F5307C3602C0B2D4
:10EFD80004F5347EC4F8D062C4F8D452CCE90023D6
:10EFE80084F8C80266467546002954D0042805D915
:10EFF8001A466D2104F1240010F015F84FF0000BAB
:10F00800D4F8C0226C21264810F00DF801200BF02E
:10F018009DF9D4F8C0226C21214810F004F894F826
:10F02800C832C5E900BB042B0CD96F211C4810F06D
:10F0380008F8D5E90023814642EA0B0043EA0901B2
:10F04800C5E900016E2116480FF0FBFFD5E9002342
:10F0580042EA000843EAE079404694F8C832C3F12E
:10F068000803DB00A3F1200EC3F1200C09FA03F218
:10F0780008FA0EFE42EA0E0228FA0CFC42EA0C02DA
:10F0880098406A6000230022C6E900230023C4F8E0
:10F09800D00284F8C8323846BDE8F88F1023002023
:10F0A8003423002008B5024810F0BEF8002008BD3F
:10F0B8003423002007B5019239B9014601AA01207D
:10F0C800FFF75CFB03B05DF804FB0820FAE7034B8D
:10F0D8000846D3F8D8321146DB68184710230020B9
:10F0E800F8B54D4C4D4D04F124064D4B6A69304638
:10F0F80000214C4F10F039F84B49304610F07EF89B
:10F10800FE68736803F59C72226203F5AA72E261D5
:10F1180003F55372A26103F55A72626103F56172D5
:10F12800226103F5687203F57670E26003F56F7289
:10F1380003F57D7323603368A260DB6860609847DD
:10F148003368A069DB68984733686069DB6898476B
:10F1580033682069DB6898473368E068DB6898475C
:10F168003368A068DB689847336860685B699847CC
:10F178003368A0695B699847336860695B69984739
:10F18800336820695B6998473368E0685B6998472A
:10F198003368A0685B6998473368206A1B69984799
:10F1A8003368E0691B699847336820681B6998478A
:10F1B800002173683A6903F537735360C4F8D8229D
:10F1C80001226B69597019491A70C3F80412184959
:10F1D8002A74C3F80812174B6B66174B2B62174B30
:10F1E800EB61174BAB61174B6B62174BAB63174B5C
:10F1F8006B63174BAB62174BEB62174BAB64174B48
:10F208006B64174B6B65174B2B65174BEB65174BEF
:10F21800AB65174BAB66F8BD1023002000610020DA
:10F22800687A02087086020839E7000805E70008CE
:10F23800D1E6000895EF0008ADF00008C1E6000827
:10F24800ADE6000899E6000885EF0008BDF0000863
:10F2580081E6000869E6000825E6000811E60008CE
:10F2680005E6000829E50008A1E40008ADE4000867
:10F2780019E500080022014B5A6070470061002020
:10F2880070B5184E184CF56860682B689B699847EC
:10F298002B68A0699B6898472B6860699B689847AA
:10F2A8002B6820699B6898472B68E0689B6898479B
:10F2B8002B68A0689B6898472B68206A9B689847CA
:10F2C8002B68E0699B6898472B6820689B6898477B
:10F2D8002B6860689B6898473369BDE870405B6A33
:10F2E800184700BF70860208F82500200A46014624
:10F2F800014810F04DB900BF1C260020022870B547
:10F30800144649D004D890B1012836D0042432E0FC
:10F3180003284FD0FF28F9D12B4CD4F88830D3F8E4
:10F32800043298476369D3F80432984703E01268B7
:10F3380032F0030301D000241DE0244B244DDE6885
:10F34800D207686933680AD51B6998472468326808
:10F3580014F00204A86908D013699847EBE7DB6842
:10F368009847336868699B69EFE7D36898473368BB
:10F37800A8699B699847204670BD144B144DDE68F8
:10F388001468286933680CB11B69E6E7DB6898479D
:10F39800336828699B69EDE70C4B0D4DDE681468EE
:10F3A8003368A868002CEFD1DB6898473368A868F1
:10F3B8009B69DFE70121074810F024FA2060002844
:10F3C800B9D12024D7E700BF006100207086020869
:10F3D800F82500201C2600200146014810F0C8BA74
:10F3E8001C26002010B50348144610F0A8F8206029
:10F3F80010BD00BF1C2600206C2938B50C461546E8
:10F408000BD06D2902D10A4BC3F8BC222A462146EB
:10F41800BDE83840074810F084B8054BD3F8BC1253
:10F42800054B01F07F01D3F8BC309847EEE700BFE9
:10F43800F82500201C2600200061002008B504489B
:10F44800D0F8C022243010F0CDF9002008BD00BF4C
:10F45800F825002008B50448D0F8C022243010F060
:10F46800A5F9002008BD00BFF825002008B5002137
:10F47800024810F07DF9002008BD00BF1C260020BE
:10F4880008B54942024810F073F9002008BD00BFD2
:10F498001C26002008B5024810F06AF9002008BDB3
:10F4A8001C26002038B50A4B0A4CDD6860682B68BA
:10F4B8009B69984701200AF049FF2B6860685B69DF
:10F4C800984704F1240010F028F9012038BD00BF46
:10F4D80070860208F825002038B50A4B0A4CDD680A
:10F4E80060682B689B69984701200AF02FFF2B68FA
:10F4F80060685B69984704F1240010F0F9F801206E
:10F5080038BD00BF70860208F82500206F2970B545
:10F518000446154600F0818200F28980122900F025
:10F52800D1813ED8052900F0718118D8022900F050
:10F538003B8107D8002900F01A81012900F02681B3
:10F5480004241AE1032900F041810429F8D1B94EB5
:10F55800002840F04481D6F8C03213600DE10F292D
:10F5680000F082810ED8082900F068810E29E7D1C1
:10F57800002840F06E812021AF480FF0E0FF4000E6
:10F588002860FAE0102900F07D811129D8D10028DF
:10F5980040F08C812921A8480FF0D1FF8010286005
:10F5A800EBE0182900F0DE811FD8152900F0B3819F
:10F5B8000DD8132900F094811429C1D1002840F0F6
:10F5C800A38126219C480FF0BAFF2860D5E01629B0
:10F5D80000F0B3811729B3D1002840F0BC812E2157
:10F5E80095480FF0ACFF2860C7E01B2900F0DD81CB
:10F5F8000DD8192900F0C4811A29A1D1002840F09A
:10F60800CD8133218C480FF09AFF2860B5E06D2931
:10F6180000F0E08100F2EC816C2991D1002840F0E3
:10F62800D281602184480FF08AFF2860A5E07D29F7
:10F6380000F0AB8248D8752900F0508222D8722990
:10F6480000F01B820FD8702900F0FD8171297FF42A
:10F6580077AF06217848002C40F003820FF06FFF47
:10F66800C0B2286089E0732900F01E8274297FF4F3
:10F6780067AF002840F026826E4B5B6AD3F8703182
:10F6880013607AE0782900F05D820ED8762900F0C0
:10F698003C8277297FF454AF002840F04C825E21E9
:10F6A80065480FF04CFF286067E0792900F0588220
:10F6B8007C297FF445AF002840F060825C215E48D9
:10F6C8000FF03DFF286058E0882900F0AD8228D867
:10F6D800842900F08B8215D87E2900F06482812964
:10F6E8007FF42EAF002800F084801468002C00F00E
:10F6F80072820121504810F085F82860002878D1DE
:10F7080020243AE0852900F07A8286297FF418AF10
:10F71800002840F08282522147480FF010FF2860ED
:10F728002BE0C82995D010D8892900F091828A2920
:10F738007FF406AF3F48436AD3F89021002C40F08D
:10F748009D82C2F307422A6017E0D42900F0AA82FA
:10F75800D62900F0B482D1297FF4F2AE002840F017
:10F768009A82502134480FF0EAFE286005E030B94B
:10F77800372131480FF0E3FE2860204670BD12683B
:10F7880037212D480FF0CDFE0024F6E728B92121B6
:10F7980029480FF0D4FE2860EFE712682121264897
:10F7A8000FF0BFFE0024E8E730B9242122480FF00B
:10F7B800C6FE00122860E0E710680FF0C7FF24219A
:10F7C80002461D480FF0ADFE0024D6E7002840F0A1
:10F7D8008682222118480FF0B2FE2860CDE7136810
:10F7E800202106F12400C6F8C0320FF0A8FE420717
:10F7F80001D40024C1E7D6F8C0020FF0A7FF2421E6
:10F80800024670180FF08DFE0024B6E730B92821A3
:10F8180009480FF094FE80102860AEE71268940D36
:10F82800A405002C40F05D829200282102480FF0C8
:10F8380078FEA2E7F82500201C260020002840F0CA
:10F8480052820F21A3480FF07AFE00F001002860D1
:10F8580093E713682021002B0CBF012202229D4848
:10F868000FF05FFE002488E728B9252199480FF09A
:10F8780066FE286081E71268252196480FF051FE40
:10F8880000247AE730B92A2192480FF058FE8010F8
:10F89800286072E71268940DA405002C40F02582B8
:10F8A80092002A218B480FF03CFE66E71268940DFF
:10F8B800A405002C40F01B829200292185480FF0F6
:10F8C80030FE5AE728B9272182480FF038FE286011
:10F8D80053E7126827217F480FF023FE00244CE7E6
:10F8E80030B92B217B480FF02AFE8010286044E7AE
:10F8F8001268940DA405002C40F0FB8192002B2186
:10F9080074480FF00EFE38E71268262171480FF090
:10F9180008FE002431E728B92C216E480FF00FFEAD
:10F9280028602AE71268940DA405002C40F0E381B2
:10F938002C2168480FF0F5FD1FE728B92D216548EF
:10F948000FF0FDFD286018E712682D2161480FF0BF
:10F95800E8FD002411E712682E215E480FF0E1FD52
:10F9680000240AE728B92F215A480FF0E8FD28603B
:10F9780003E712682F2157480FF0D3FD0024FCE657
:10F9880028B9302153480FF0DAFD2860F5E61268EF
:10F99800302150480FF0C5FD0024EEE612683321EF
:10F9A8004C480FF0BEFD0024E7E628B93421494849
:10F9B8000FF0C5FD2860E0E61268342145480FF0D5
:10F9C800B0FD0024D9E61268602142480FF0A9FD75
:10F9D8000024D2E628B961213E480FF0B0FD286026
:10F9E800CBE6126861213B480FF09BFD0024C4E67A
:10F9F8001C21384824B90FF0A2FD00142860BCE689
:10FA08000FF09DFD2A68C0F3080040EA02421C215D
:10FA180030480FF086FD0024AFE61C212D4824B99C
:10FA28000FF08DFDC0B22860A7E60FF088FD2B68A7
:10FA380000F47F02C3F308031A431C2125480FF082
:10FA480070FD002499E628B9592122480FF077FD66
:10FA5800286092E6126859211E480FF062FD0024C2
:10FA68008BE60FF06CFD2A7820F0FF000243062198
:10FA780018480FF056FD00247FE6062115482CB9DA
:10FA88000FF05DFDC0F30720286076E60FF057FD04
:10FA98002B6820F47F421B029BB21A4306210D48B3
:10FAA8000FF03FFD002468E628B90B4B5B6AD3F8DA
:10FAB8006C31136061E612685A2106480FF031FD77
:10FAC80000245AE612685B2102480FF02AFD002440
:10FAD80053E600BF1C260020F82500208848436A0A
:10FAE800D3F870311CB9C3F30E03136045E61268EE
:10FAF80023F4FF4323F07F03C2F30E021A435B2172
:10FB080024300FF00EFD002437E67D4B5B6AD3F8F6
:10FB1800702118B9C2F307422A602EE62B6822F436
:10FB28007F021B0403F47F031A435B2175480FF01F
:10FB3800F8FC002421E612685E2172480FF0F1FCFF
:10FB480000241AE628B918216E480FF0F8FC28603E
:10FB580013E6126818216B480FF0E3FC00240CE64A
:10FB680028B9192167480FF0EAFC286005E61268F1
:10FB7800192164480FF0D5FC0024FEE512685C21C9
:10FB880060480FF0CEFC0024F7E528B95F215D48F6
:10FB98000FF0D5FC2860F0E512685F2159480FF096
:10FBA800C0FC0024E9E5062156482CB90FF0C7FC33
:10FBB800C0F307402860E0E50FF0C1FC2B6820F493
:10FBC8007F021B0403F47F031A4306214D480FF0FC
:10FBD800A8FC0024D1E507214A480FF0B0FC072112
:10FBE80020F4800247480FF09CFCC6E5002840F04E
:10FBF8008480652143480FF0A2FC2860BDE50028F9
:10FC08007FF4F7AD07213F480FF099FCC0F381500E
:10FC1800431E584258412860AFE5126852213948BE
:10FC28000FF07FFC0024A8E53548436AD3F89021FB
:10FC380014B9D2B22A60A0E52B6822F0FF0203F0C3
:10FC48000F031A43632124300FF06BFC002494E562
:10FC58002B4B5B6AD3F8902118B9C2F303222A60B0
:10FC68008BE52B6822F470621B0203F470631A435D
:10FC7800632124480FF055FC00247EE52B6822F40C
:10FC88007F021B0403F47F031A43632124300FF01F
:10FC980048FC002471E5126850211A480FF041FC15
:10FCA80000246AE520B9164B5B6ADB69136064E5DA
:10FCB8001268532113480FF034FC00245DE528B97D
:10FCC800152110480FF03BFC286056E513680E4AD2
:10FCD80015215A430B480FF024FC00244DE5042459
:10FCE8004BE5102449E5042447E5102445E5102494
:10FCF80043E5102441E510243FE504243DE500BF19
:10FD0800F82500201C260020007102000B4619B9B6
:10FD180001461846FFF7FABB082070472DE9F84F4F
:10FD28000027424CD4F8CC62D4F8C8524FEA0629CE
:10FD380049EA1569C6B24FEA052894F8D002D4F802
:10FD4800DC5248EA0602D4F8D86249EA07030130CF
:10FD58002F0E2D0245EA166504F5327C3602C0B234
:10FD680004F5367EC4F8D862C4F8DC52CCE9002326
:10FD780084F8D00266467546002954D0042805D96F
:10FD88001A466D2104F124000FF0CBFB4FF0000B55
:10FD9800D4F8C8226C2126480FF0C3FB01200AF0D2
:10FDA800D5FAD4F8C8226C2121480FF0BAFB94F890
:10FDB800D032C5E900BB042B0CD96F211C480FF0C9
:10FDC800BEFBD5E90023814642EA0B0043EA09015C
:10FDD800C5E900016E2116480FF0B1FBD5E90023F3
:10FDE80042EA000843EAE079404694F8D032C3F189
:10FDF8000803DB00A3F1200EC3F1200C09FA03F27B
:10FE080008FA0EFE42EA0E0228FA0CFC42EA0C023C
:10FE180098406A6000230022C6E900230023C4F842
:10FE2800D80284F8D0323846BDE8F88FF82500208B
:10FE38001C26002070B5154C054694F874300E4603
:10FE4800012B1BD0032B0BBF002228220C230F23CE
:10FE580043F0884343F0401343EA423204212846E2
:10FE68000FF05FFB012E0CD128460FF019FCD4F8D7
:10FE78008830D3F80432BDE87040184700220B23BD
:10FE8800E6E7D4F88830D3F80832F4E700610020B8
:10FE980008B502480FF06CFC002008BD1C260020A5
:10FEA80007B5019239B9014601AA0120FFF72EFBD7
:10FEB80003B05DF804FB0820FAE7034B0846D3F8C3
:10FEC800E0321146DB681847F8250020F8B54D4C9C
:10FED8004D4D04F124064D4B6A69304600214C4FC4
:10FEE8000FF0C1FB4B4930460FF02CFCFE687368DD
:10FEF80003F59C72226203F5AA72E26103F553725C
:10FF0800A26103F55A72626103F56172226103F519
:10FF1800687203F57670E26003F56F7203F57D731E
:10FF280023603368A260DB68606098473368A06923
:10FF3800DB68984733686069DB68984733682069ED
:10FF4800DB6898473368E068DB6898473368A068DF
:10FF5800DB689847336860685B6998473368A069CD
:10FF68005B699847336860695B69984733682069BB
:10FF78005B6998473368E0685B6998473368A068AD
:10FF88005B6998473368206A1B6998473368E0695A
:10FF98001B699847336820681B6998470021736874
:10FFA8003A6903F537735360C4F8E02201226B699C
:10FFB800597019491A70C3F8041218492A74C3F8F9
:10FFC8000812174B6B66174B2B62174BEB61174BDD
:10FFD800AB61174B6B62174BAB63174B6B63174BDC
:10FFE800AB62174BEB62174BAB64174B6B64174B49
:08FFF8006B65174B2B65174BDD
:020000040801F1
:10000000EB65174BAB65174BAB66F8BDF8250020C9
:1000100000610020687C0208708602083DFE00082E
:10002000E1F40008ADF4000825FD000899FE000881
:100030009DF4000889F4000875F4000815FD000817
:10004000A9FE00085DF4000845F4000801F400086A
:10005000EDF30008E1F3000805F300087DF2000865
:1000600089F20008F5F2000800207047012070476F
:100070000022014B5A607047006100201FB5084BF9
:1000800033F8084C5A7802949C1E019433F8041CEF
:100090000091014600200FF0E5FE04B010BD00BF46
:1000A0004C67002010B5002014460FF0ABFC206018
:1000B00010BD00200FF0C8BC10B5044618B90FF0F1
:1000C000C3FD204610BD0820FCE710B5044618B952
:1000D0000FF09CFD204610BD0820FCE70021F4E74E
:1000E0004942F2E7F1E7022804BF0C4B93F8E8001D
:1000F00030B90B4BDB681B689B690A4A10681847CC
:10010000012809D1054B93F8E830012B04D1044BA9
:10011000DB681B685B69F0E7704700BF0061002087
:1001200070860208E828002010B50020FFF7DBFFEA
:10013000BDE81040034B044ADB6810681B689B69EC
:10014000184700BF70860208E828002010B5044652
:1001500020B909680FF085FD204610BD0820FCE796
:1001600038B50D46044620B90FF069FD28602046D9
:1001700038BD0820FCE7043938B504461546FA298D
:1001800000F23987DFE811F0FB0037073707370740
:10019000370737073707370737073707370737076F
:1001A000370737073707370737073707370737075F
:1001B000370737073707370737073707370737074F
:1001C000370737073707370737073707370737073F
:1001D000370737073707370737073707370737072F
:1001E000370737070901190137072901390137078F
:1001F000370737073707370737073707370737070F
:1002000037073707370737073707370737073707FE
:1002100037073707370737073707370737073707EE
:1002200037073707370737073707370737073707DE
:1002300037073707370737073707370737073707CE
:10024000370737073707370749015701650173013A
:1002500081018F019D01AB01B901C701D501E30106
:10026000F101FF010D021B02290233023D02370793
:10027000470251025B0265026F027E028D029C0200
:10028000A502370737073707AE02B602BE02C8021B
:10029000D202370737073707DA02E202EA023707E6
:1002A000370737073707370737073707F402FE02E4
:1002B00008031203370737073707370737073707AA
:1002C0001C03260330033A03440337073707370775
:1002D000370737074E0358036803780380038C03FE
:1002E00096039F03A903B003BB03C803D503E2032E
:1002F000EF03FC0309041604370723042E043B0410
:100300004804530460046D047A0487049404A3042D
:10031000B204C104D004DF04EE04FD040D05200581
:100320003005400550056005700580059005A00565
:10033000B005C005CF053707370737073707370739
:10034000370737073707370737073707DE05EE0563
:10035000FE050E061E062E063E064E065E066D06BF
:100360007C068B069A06A906B806C706D606E406DA
:10037000F206000737070E07190727072F0728B9C6
:1003800060210FF03FFB2860204638BD12686021D5
:1003900000200FF059FB0024F6E730B9024608218F
:1003A0000FF072FB00B22860EEE7138800220821EC
:1003B00010460FF076FB0024E6E730B9024609212B
:1003C0000FF062FB00B22860DEE7138800220921EB
:1003D00010460FF066FB0024D6E730B90122082151
:1003E0000FF052FB00B22860CEE7138808210122EB
:1003F00000200FF056FB0024C6E730B90122092186
:100400000FF042FB00B22860BEE7138809210122E9
:1004100000200FF046FB0024B6E7002840F0EE85F0
:10042000012203210FF010FB2246022120460FF08B
:100430002BFB2860A8E7002840F0E3850122032178
:100440000FF002FB0122022120460FF01DFB286065
:100450009AE7002840F0D885022203210FF0F4FA31
:100460002246022120460FF00FFB28608CE700286F
:1004700040F0CD85024603210FF0E6FA2246022124
:1004800020460FF001FB28607EE7002840F0C2857F
:10049000024603210FF0D8FA0122022120460FF074
:1004A000F3FA286070E7002840F0B7850322114670
:1004B0000FF0CAFA2246022120460FF0E5FA286022
:1004C00062E7002840F0AC85042203210FF0BCFA5B
:1004D0002246022120460FF0D7FA286054E7002870
:1004E00040F0A185042203210FF0AEFA012202217F
:1004F00020460FF0C9FA286046E7002840F09685AC
:10050000052203210FF0A0FA2246022120460FF017
:10051000BBFA286038E7002840F08B8505220321CC
:100520000FF092FA0122022120460FF0ADFA286066
:100530002AE7002840F08085062203210FF084FA84
:100540002246022120460FF09FFA28601CE700286F
:1005500040F07585072203210FF076FA224602212A
:1005600020460FF091FA28600EE7002840F06A85D7
:10057000072203210FF068FA0122022120460FF022
:1005800083FA286000E7002840F05F8508220321F5
:100590000FF05AFA2246022120460FF075FA286021
:1005A000F2E6002840F05485082203210FF04CFAAF
:1005B0000122022120460FF067FA2860E4E60028B5
:1005C00040F04985092203210FF03EFA224602211C
:1005D00020460FF059FA2860D6E6002840F03E8504
:1005E000024612210FF050FA00B22860CCE6002833
:1005F00040F03785012212210FF046FA00B2286040
:10060000C2E6002840F03085024613210FF03CFA84
:1006100000B22860B8E6002840F02985024615217E
:100620000FF032FA00B22860AEE6002840F02285D2
:10063000012215210FF028FA00B22860A4E6002854
:1006400040F01B85024616210FF01EFA00B228600A
:100650009AE6002840F01485012216210FF014FAC2
:1006600000B2286090E6002840F00D850A220321A0
:100670000FF0EAF92246022120460FF005FA00B2F7
:10068000286081E6002840F001850A2203210FF04E
:10069000DBF90122022120460FF0F6F900B22860B2
:1006A00072E6002840F0F5840B2203210FF0CCF90C
:1006B0002246022120460FF0E7F900B2286063E6E7
:1006C000002840F0E984024606210FF0DDF9286099
:1006D0005AE6002840F0E384012206210FF0D4F905
:1006E000286051E6002840F0DD8441210FF08AF9AE
:1006F000286049E6002840F0D88442210FF082F9B2
:10070000286041E6002840F0D384012246210FF002
:10071000BBF900B2286037E6002840F0CC840246DE
:1007200046210FF0B1F900B228602DE6002840F014
:10073000C58447210FF066F9286025E6002840F0BF
:10074000C08421210FF05EF928601DE6002840F0EA
:10075000BB8422210FF056F9286015E6002840F0EE
:10076000B684024623210FF08FF900B228600BE611
:10077000002840F0AF8427210FF044F920F07F409B
:10078000286001E6002840F0A88428210FF03AF9FB
:1007900020F07F402860F7E5002840F0A184012286
:1007A0002A210FF071F900B22860EDE5002840F031
:1007B0009A8402462A210FF067F900B22860E3E527
:1007C000002840F09384024639210FF05DF900B211
:1007D0002860D9E5002840F08C84012239210FF0EF
:1007E00053F900B22860CFE5002840F08584024626
:1007F0003D210FF049F900B22860C5E5002840F01E
:100800007E8402463F210FF03FF900B22860BBE52D
:10081000002840F0778402463A210FF035F900B203
:100820002860B1E5002840F07084024653210FF0A3
:100830002BF900B22860A7E530B9012264210FF03E
:1008400023F900B228609FE513886421012200206B
:100850000FF027F9002497E530B9024664210FF024
:1008600013F900B228608FE5138800226421104636
:100870000FF017F9002487E5002840F0498466212D
:100880000FF0C0F828607FE520B968210FF0BAF8B2
:10089000286079E5116800200FF0D6F9002473E58F
:1008A000002840F03884012269210FF0EDF800B2F1
:1008B000286069E5002840F03184C24B59890FF067
:1008C00055F9286060E5002840F02B840246692134
:1008D0000FF0DAF800B2286056E5002840F02484D2
:1008E0000FF0ADF928604FE518B90FF0D2F9286084
:1008F0004AE5116800200FF0C8F9002444E50028FB
:1009000040F0158402466D210FF09EF86C212046C0
:100910000FF078F8286037E5002840F00B840122BA
:100920006D210FF091F86C2120460FF06BF82860D4
:100930002AE5002840F0018402226D210FF084F89E
:100940006C2120460FF05EF828601DE5002840F07D
:10095000F78303226D210FF077F86C2120460FF00A
:1009600051F8286010E5002840F0ED8304226D2145
:100970000FF06AF86C2120460FF044F8286003E578
:10098000002840F0E38305226D210FF05DF86C2113
:1009900020460FF037F82860F6E4002840F0D983AD
:1009A00006226D210FF050F86C2120460FF02AF836
:1009B0002860E9E4002840F0CF8307226D210FF082
:1009C00043F86C2120460FF01DF82860DCE418B9CC
:1009D0000FF09CF82860D7E4116800200FF088F829
:1009E0000024D1E4774B598918B90FF0B5F8286085
:1009F000CAE4126800200FF09DF80024C4E4002827
:100A000040F0AD8301226F210FF01EF86E212046C9
:100A10000EF0F8FF2860B7E418B90FF004F9286069
:100A2000B2E4116800200FF0F1F80024ACE40028D3
:100A300040F0988303226F210FF006F86E212046C4
:100A40000EF0E0FF28609FE4002840F08E8304222F
:100A50006F210EF0F9FF6E2120460EF0D3FF2860C3
:100A600092E4002840F0848305226F210EF0ECFF11
:100A70006E2120460EF0C6FF286085E4002840F075
:100A80007A8306226F210EF0DFFF6E2120460EF0E2
:100A9000B9FF286078E4002840F0708307226F21B6
:100AA0000EF0D2FF6E2120460EF0ACFF28606BE402
:100AB000002840F0668308226F210EF0C5FF224611
:100AC0006E2120460EF0E0FF00B228605CE40028B2
:100AD00040F05A8308226F210EF0B6FF01226E21EA
:100AE00020460EF0D1FF00B228604DE4002840F00F
:100AF0004E8309226F210EF0A7FF22466E21204669
:100B00000EF0C2FF00B228603EE4002840F04283AD
:100B10000A226F210EF098FF22466E2120460EF029
:100B2000B3FF00B228602FE4002840F036830A2289
:100B30006F210EF089FF01226E2120460EF0A4FFE6
:100B400000B2286020E4002840F02A830B226F21A5
:100B50000EF07AFF22466E2120460EF095FF00B27D
:100B6000286011E4002840F01E830B226F210EF054
:100B70006BFF01226E2120460EF086FF00B2286036
:100B800002E4002840F012830C226F210EF05CFF7B
:100B900022466E2120460EF077FF00B22860FFF754
:100BA000F3BB002840F005830C226F210EF04CFFB0
:100BB00001226E2120460EF067FF00B22860FFF789
:100BC000E3BB00BF44670020002840F0F5820D22FF
:100BD0006F210EF039FF22466E2120460EF054FFA1
:100BE00000B22860FFF7D0BB002840F0E8820D2259
:100BF0006F210EF029FF01226E2120460EF044FFE6
:100C000000B22860FFF7C0BB002840F0DB820E2254
:100C10006F210EF019FF22466E2120460EF034FFA0
:100C200000B22860FFF7B0BB002840F0CE820E2251
:100C30006F210EF009FF01226E2120460EF024FFE5
:100C400000B22860FFF7A0BB002840F0C1820F224D
:100C50006F210EF0F9FE22466E2120460EF014FFA1
:100C600000B22860FFF790BB002840F0B4820F224A
:100C70006F210EF0E9FE01226E2120460EF004FFE6
:100C800000B22860FFF780BB002840F0A782102246
:100C90006F210EF0D9FE22466E2120460EF0F4FEA2
:100CA00000B22860FFF770BB002840F09A82112242
:100CB0006F210EF0C9FE22466E2120460EF0E4FEA2
:100CC00000B22860FFF760BB002840F08D8211223F
:100CD0006F210EF0B9FE01226E2120460EF0D4FEE7
:100CE00000B22860FFF750BB002840F0808212223B
:100CF0006F210EF0A9FE22466E2120460EF0C4FEA2
:100D000000B22860FFF740BB002840F07382132236
:100D10006F210EF099FE22466E2120460EF0B4FEA1
:100D20002860FFF731BB002840F0678213226F2153
:100D30000EF08AFE01226E2120460EF0A5FE2860EC
:100D4000FFF722BB002840F05B82C0226F210EF02B
:100D50007BFE22466E2120460EF096FE00B22860F1
:100D6000FFF712BB002840F04E82C0226F210EF028
:100D70006BFE01226E2120460EF086FE00B2286036
:100D8000FFF702BB002840F04182C1226F210EF024
:100D90005BFE22466E2120460EF076FE00B22860F1
:100DA000FFF7F2BA002840F03482C1226F210EF022
:100DB0004BFE01226E2120460EF066FE00B2286036
:100DC000FFF7E2BA002840F02782C2226F210EF01E
:100DD0003BFE22466E2120460EF056FE00B22860F1
:100DE000FFF7D2BA002840F01A82C2226F210EF01B
:100DF0002BFE01226E2120460EF046FE00B2286036
:100E0000FFF7C2BA002840F00D82C3226F210EF016
:100E10001BFE22466E2120460EF036FE00B22860F0
:100E2000FFF7B2BA002840F00082C3226F210EF013
:100E30000BFE01226E2120460EF026FE00B2286035
:100E4000FFF7A2BA002840F0F381C4226F210EF010
:100E5000FBFD22466E2120460EF016FE2860FFF7AD
:100E600093BA002840F0E781C4226F210EF0ECFD18
:100E700001226E2120460EF007FE2860FFF784BA9B
:100E8000002840F0DB81C5226F210EF0DDFD2246F7
:100E90006E2120460EF0F8FD2860FFF775BA002895
:100EA00040F0CF81C5226F210EF0CEFD01226E21D0
:100EB00020460EF0E9FD2860FFF766BA002840F0F2
:100EC000C381C6226F210EF0BFFD22466E2120464F
:100ED0000EF0DAFD2860FFF757BA002840F0B7811E
:100EE000C6226F210EF0B0FD01226E2120460EF0C9
:100EF000CBFD2860FFF748BA002840F0AB81C7223D
:100F00006F210EF0A1FD22466E2120460EF0BCFDA1
:100F10002860FFF739BA002840F09F81C7226F216F
:100F20000EF092FD01226E2120460EF0ADFD2860EC
:100F3000FFF72ABA002840F09381C8226F210EF0F3
:100F400083FD6E2120460EF05DFD2860FFF71CBA80
:100F5000002840F08881C9226F210EF075FD6E21B6
:100F600020460EF04FFD2860FFF70EBA002840F033
:100F70007D81CA226F210EF067FD6E2120460EF0A2
:100F800041FD2860FFF700BA002840F07281CB22B3
:100F90006F210EF059FD6E2120460EF033FD2860C2
:100FA000FFF7F2B9B74B18B95B891360FFF7ECB9DB
:100FB000126800245A81FFF7E7B920B9B14B5B7A78
:100FC0001360FFF7E1B9B04A2878511C0EF054FFC6
:100FD0000024FFF7D9B9002840F04E81A94B1B7AB5
:100FE0001360FFF7D1B9002840F04981A54BDB8899
:100FF0001360FFF7C9B90424FFF7C6B90424FFF74B
:10100000C3B90424FFF7C0B90424FFF7BDB9042411
:10101000FFF7BAB90424FFF7B7B90424FFF7B4B94E
:101020000424FFF7B1B90424FFF7AEB90424FFF795
:10103000ABB90424FFF7A8B90424FFF7A5B9042429
:10104000FFF7A2B90424FFF79FB90424FFF79CB966
:101050000424FFF799B90424FFF796B90424FFF795
:1010600093B90424FFF790B90424FFF78DB9042441
:10107000FFF78AB90424FFF787B90424FFF784B97E
:101080000424FFF781B90424FFF77EB90424FFF795
:101090007BB90424FFF778B90424FFF775B9042459
:1010A000FFF772B90424FFF76FB90424FFF76CB996
:1010B0000424FFF769B90424FFF766B90424FFF795
:1010C00063B90424FFF760B90424FFF75DB9042471
:1010D000FFF75AB90424FFF757B90424FFF754B9AE
:1010E0000424FFF751B90424FFF74EB90424FFF795
:1010F0004BB90424FFF748B90424FFF745B9042489
:10110000FFF742B90424FFF73FB90424FFF73CB9C5
:101110000424FFF739B90424FFF736B90424FFF794
:1011200033B90424FFF730B90424FFF72DB90424A0
:10113000FFF72AB90424FFF727B90424FFF724B9DD
:101140000424FFF721B90424FFF71EB90424FFF794
:101150001BB90424FFF718B90424FFF715B90424B8
:10116000FFF712B90424FFF70FB90424FFF70CB9F5
:101170000424FFF709B90424FFF706B90424FFF794
:1011800003B90424FFF700B90424FFF7FDB80424D1
:10119000FFF7FAB80424FFF7F7B80424FFF7F4B810
:1011A0000424FFF7F1B80424FFF7EEB80424FFF796
:1011B000EBB80424FFF7E8B80424FFF7E5B80424EB
:1011C000FFF7E2B80424FFF7DFB80424FFF7DCB828
:1011D0000424FFF7D9B80424FFF7D6B80424FFF796
:1011E000D3B80424FFF7D0B80424FFF7CDB8042403
:1011F000FFF7CAB80424FFF7C7B80424FFF7C4B840
:101200000424FFF7C1B80424FFF7BEB80424FFF795
:10121000BBB80424FFF7B8B80424FFF7B5B804241A
:10122000FFF7B2B80424FFF7AFB80424FFF7ACB857
:101230000424FFF7A9B80424FFF7A6B80424FFF795
:10124000A3B80424FFF7A0B80424FFF79DB8042432
:10125000FFF79AB80424FFF797B80424FFF794B86F
:101260000424FFF791B80424FFF78EB80424FFF795
:101270008BB80424FFF788B80424FFF785B804244A
:10128000FFF782B8446700204C6700200B4619B96D
:1012900001461846FEF76FBF0820704701207047CF
:1012A00007B5019239B9014601AA0120FEF763FF93
:1012B00003B05DF804FB0820FAE710B40C4630B91F
:1012C000044B20465B6811469B6810BC1847002001
:1012D00010BC7047E828002070B5284E284DF468EF
:1012E00060682368C830DB68286098470120FEF7F3
:1012F000FAFE6368326903F537735360214B224964
:101300006A605A693220C2F804122049C2F80812F1
:101310000021117051701E4A1A621E4ADA611E4A7B
:101320009A611E4A5A621E4ADA641E4A9A631E4A2B
:101330005A631E4A9A621E4ADA621E4A9A641E4A1A
:101340005A641E4A5A651E4A1A651E4A1A661E4A81
:10135000DA6501221A741D4A9A6540F28A22C3E9AD
:1013600002204FF47A721A4B9A8041F270721A601E
:101370004FF4807259725A8170BD00BF70860208A6
:10138000E8280020006100206D0001089D1201087E
:10139000CB000108E5000108E1000108DD000108BB
:1013A000610101088D120108A1120108B9000108AC
:1013B0004D010108B3000108A50001087D000108E6
:1013C00069000108E700010871000108290101080E
:1013D00044670020002070470022014B5A6070478C
:1013E0000061002000200EF077BD002208B51046F5
:1013F00017210EF071FD00221A2110460EF06CFD2F
:1014000041F61912192100200EF066FD012008BDD9
:10141000EBE710B5002014460EF03CFD206010BD37
:10142000022804BF0B4B93F8E80030B90A4BDB6885
:101430001B689B69094A10681847012809D1054BA8
:1014400093F8E830012B04D1034BDB681B685B6920
:10145000F0E770470061002070860208FC28002039
:1014600010B50020FFF7DCFFBDE81040034B044A35
:10147000DB6810681B689B69184700BF708602080C
:10148000FC280020F0B50746284B85B033F8060C41
:101490005A780290981E019033F8041C244D009154
:1014A000002039460EF06AFF6B68BB4230D105B0B0
:1014B000F0BD204B1B78032B0FD11F4E20460CF0A4
:1014C0006FFAA26833689A4205D0682100200EF0B6
:1014D00003FDA36833606F60E9E7022B15D1174E57
:1014E00020460CF02CFA226933689A42F3D0662128
:1014F00000200EF0F1FC236933606B2100200EF018
:10150000C9FC0023A060E361E5E7012BE3D1F4E728
:101510000B4C94F82060002ECBD16B2130460EF09E
:10152000B9FC2661A060E661D5E700BF4A670020EC
:10153000FC28002078670020806700207C6700205E
:101540005467002038B50D46044620B90EF003FE5E
:101550002860204638BD0820FCE770B50E46E0B98B
:101560000F4D95F82040A4B10E4C2278012A02D1EB
:101570000EF0F1FD28610321002021700EF0F0FC37
:101580006B2100200EF086FC336818446860002050
:1015900070BD09680EF0F1FDF9E70820F8E700BF1B
:1015A000546700207867002070B50E46A8B90C4D2E
:1015B00095F8204074B10B4C2278012A02D10EF02C
:1015C000CAFD28610321002021700EF0C9FC6E6065
:1015D000002070BD0EF0C4FDFAE70820F9E700BF57
:1015E000546700207867002070B50E46A8B90C4DEE
:1015F00095F8204074B10B4C2278012A02D10EF0EC
:10160000AAFD28610221002021700EF0A9FCEE60E5
:10161000002070BD0EF08FFDFAE70820F9E700BF4B
:1016200054670020786700200021DDE74942DBE7AE
:10163000DAE738B515460C4600295DD1AC283BD019
:1016400018D80C2834D00AD8042829D00B2855D112
:101650005F2120460EF040FC294B5D6126E00D28FD
:1016600024D0AB284AD193B20122642120460EF047
:1016700060FC1BE0BE2833D008D8B3281FD0BD289B
:101680003CD1114620460EF07BFC0FE0FB2830D009
:10169000FC2833D11B4AE8B2511C0EF079FE05E05C
:1016A000602120460EF018FC154B1D60204638BD09
:1016B000134B83F82020F9E793B20A46D5E76B2154
:1016C00020460EF009FC104B1B78032BEED10C4B7F
:1016D0002A46C3E90155682120460EF0FDFBE5E7E7
:1016E0000A4B204619890EF078FC0122064B1A702D
:1016F000DCE7064B1A81D9E70824D7E70424D5E7AD
:10170000546700204A670020786700204467002063
:1017100038B515460C46002940F09080B22877D0A5
:1017200023D8AB2863D013D80B284DD003D8042876
:1017300041D0042446E00C284ED00D28F9D1404B6E
:1017400093F82020002A4CD01B692B60002439E03C
:10175000AD2856D053D3AE2858D0B028E9D1394B54
:10176000204619890EF055FC47E0C0285ED013D8FA
:10177000BD2851D005D8B328DBD108460EF015FDA1
:101780003BE0BE284CD0BF28D3D101226F21204698
:101790000EF0A2FB6E2135E0FC2849D004D8FB28CE
:1017A000C7D1284B1B891AE0FD2844D0FE28C0D1A0
:1017B000244B9B8813E0602120460EF06BFB204BEE
:1017C00028601860204638BD5F2120460EF062FB7D
:1017D0001B4B28605861F5E7194B93F820302B60BC
:1017E000F0E7662100200EF055FB2860AEE70122ED
:1017F000642120460EF090FB00B22860E2E70A4622
:10180000F6E7662120460EF045FBF6E76821F9E78A
:1018100008460EF0A0FCF0E708460EF0BFFBECE730
:10182000084B204619890EF0EAFBE6E70222ADE7F5
:10183000044BDB79D3E7034B9B79D0E70824C1E75E
:10184000546700204467002010B40C4630B9054BA3
:1018500020469B6811469B6810BC1847002010BCAE
:10186000704700BFFC28002070B5424E424DF4681E
:1018700060682368C830DB68286098470120FFF75C
:10188000CFFD6368326903F5377353603B4BAA6041
:101890003B495A690024C2F804123A495470C2F80C
:1018A000081201211170384A19741A62374A462108
:1018B000DA61374A20469A61364A374D5A62374ACA
:1018C000DA64374A9A63374A5A63374A9A62374A20
:1018D000DA62374A9A64374A5A64374A5A65374A4D
:1018E0001A65374A1A66374ADA65374A9A6540F206
:1018F0008A22C3E902214FF47A72344B17215A80AD
:1019000041F270721A804FF48072DC711A812246A3
:101910000EF0E2FA22461A2120460EF0DDFA41F6D8
:101920001912192120460EF0D7FA22460621204628
:101930000EF0D2FA4FF4FA625F2120460EF0CCFA94
:101940004FF47A62602120460EF0C6FA28460BF06A
:10195000EBFF1F4B60211C701E4B20461C601E4B72
:101960001C600EF097FA5F21286020460EF092FA74
:10197000686170BD70860208FC28002000610020AC
:10198000EB13010811140108E915010831160108CB
:101990002D16010829160108546700204515010875
:1019A0001117010833160108A91501085B15010874
:1019B000E51301081314010885140108D513010863
:1019C00021140108D913010861140108446700209B
:1019D00078670020806700207C6700200022014B90
:1019E0005A6070470061002070B50546074C0146FB
:1019F000261D2368324600200EF0A5FD23683246DE
:101A00002946BDE8704001200EF09DBD142900203C
:101A1000014B18680EF0F7BD1429002001280CD8DE
:101A2000074B1A68202303FA00F040F0020002EB93
:101A30008000436800200B6070470820704700BF9B
:101A400014290020012810B5144612D003D302280F
:101A50001CD004200AE0114B114ADB6824681B6883
:101A6000D2F8A8021CB15B699847002010BD9B69A1
:101A7000FAE70A4B0A4ADB68D2F8A0021B685B6AE5
:101A80009847003018BF01202060EEE7034B044A5E
:101A9000DB68D2F8A4021B685B6AF1E77086020873
:101AA00014290020022804BF0C4B93F8E80038B931
:101AB0000B4BDB681B685B690A4AD2F89C0218472B
:101AC000012809D1054B93F8E830012B04D1044BD0
:101AD000DB681B689B69EFE7704700BF006100206F
:101AE000708602081429002070B50020FFF7DAFF85
:101AF000134B144CDD68D4F89C022B689B68984704
:101B00002B68D4F8A0029B6898472B68D4F8A402ED
:101B10009B6898472B68D4F8B4029B6898472B6859
:101B2000D4F8AC029B6898472B68D4F8B0029B6845
:101B300098472B68D4F8A8029B68BDE87040184706
:101B400070860208142900202DE9F8430F469146BB
:101B50009846194C0021D4F8B83247F080009B68B1
:101B60009DF820609DF824509847D4F8B8320021A1
:101B70009B6848469847D4F8B83200219B68404695
:101B80009847D4F8B83200219B6830469847D4F87B
:101B9000B83228469B680121984748EA09282368FB
:101BA00046EA082607F07F0703EB870745EA062584
:101BB0007D60BDE8F88300BF1429002007B5D3B2CB
:101BC0000193C2F307230093C2F30743120EFFF7FA
:101BD000BBFF03B05DF804FB0020FFF7EFBF012857
:101BE0002DE9F34105460F4628D82026DFF854801A
:101BF000864018F8003074B263B1114B44F007010D
:101C000003EB8003D3F8BC22C9B2FFF7D7FF002350
:101C100008F8053044F00D0100243A46C9B22846C0
:101C2000FFF7CCFF2846CDE9004423462246F1B217
:101C3000FFF78AFF204602B0BDE8F0810820FAE7EE
:101C40001429002070000020012873B505460E46B7
:101C50001CD82024844044F0070186EAE672A2EBF7
:101C6000E672C9B2FFF7AAFF0123094A002E5355B5
:101C7000E1B2B8BF022300242846CDE90043224642
:101C80002346FFF761FF204602B070BD0820FBE746
:101C9000700000200021D7E74942D5E7D4E738B5E6
:101CA000274D01F07F042B1993F81832DB0704D479
:101CB0002B6803EB8404606838BDD5F8B832002186
:101CC0009B68204698470021D5F8B83208469B68A3
:101CD00098470021D5F8B83208469B6898470021FC
:101CE000D5F8B83208469B689847D5F8B832012134
:101CF0009B6800209847D5F8B83200219B682046A1
:101D000098470021D5F8B83208469B6898470021CB
:101D1000D5F8B83204029B68084698470021D5F8E8
:101D2000B83204439B6808469847D5F8B832240275
:101D300004439B6801210020984724022043BBE70D
:101D40001429002010B500201446FFF7A8FF2060DA
:101D500010BD38B50D462021814041F00101C9B2C6
:101D60000446FFF79CFF2968014429602046BDE82E
:101D7000384034E71C2A2DE9F84304460D461E4638
:101D800000F0188300F2A8800C2A00F048824CD89A
:101D9000052A00F0E7811AD8022A00F09B8107D8B3
:101DA000002A00F07381012A00F08381042477E186
:101DB000032A00F0A981042AF8D1CC4B8A001344ED
:101DC000002840F0B481D3F8BC32336068E1082ABF
:101DD00000F0048214D8062A00F0D581072AE5D144
:101DE00020278F4047F01007FFB239462846002CC5
:101DF00040F0E681FFF753FF00F01F0030604FE135
:101E00000A2A00F0FA810B2AD0D1002840F0DB85A5
:101E10002021A94041F01501C9B22846FFF73FFF34
:101E2000C04300F0010030603AE1122A00F0618204
:101E300027D80F2A00F0358211D80D2A00F00D8224
:101E40000E2AB3D12021A94041F01401C9B20028C3
:101E500040F021822846FFF722FF306020E1102A5F
:101E600000F03082112AA1D12021A94041F00801BF
:101E7000C9B2002840F037822846FFF710FF3060D3
:101E80000EE1152A00F05D8211D8132A00F042827B
:101E9000142A8BD12021A94041F00B01C9B200289E
:101EA00040F049822846FFF7FAFE3060F8E0172A32
:101EB00000F06982C0F05682182A7FF477AF2021A3
:101EC000A94041F01301C9B2002840F06D822846B4
:101ED000FFF7E5FE3060E3E0AC2A00F0288463D829
:101EE000A52A00F02F8331D8A22A00F0E48218D866
:101EF0001D2A00F07E828C2A7FF458AF002840F023
:101F00008682090141F06C0101F0FC012846FFF7CF
:101F1000C6FE4FF48073C0F3036043FA00F03060F4
:101F2000BEE0A32A00F0E382A42A7FF43FAF0F01B2
:101F300047F06C07FFB239462846002C40F0F38288
:101F4000FFF7ADFEC0F300303060A9E0A82A00F032
:101F50008B8314D8A62A00F03B83A72A7FF426AFF0
:101F60000F0147F06C07FFB239462846002C40F0BD
:101F70006D83FFF794FE00F00F00306090E0AA2A16
:101F80004FEA011700F0A68340F2898347F06D07FE
:101F9000FFB239462846002C40F0BA83FFF77FFE97
:101FA000C0F3411030607BE0B62A00F04C843ED88C
:101FB000B32A00F002841BD8AD2A00F0D383AE2AE6
:101FC0007FF4F4AE0F0147F06D07FFB239462846A3
:101FD000002C40F0E383FFF762FE001400F07F0363
:101FE00010F0400018BF6FF07F001843306057E0DA
:101FF000B42A00F0FE83B52A7FF4D8AE20278F40A4
:102000007FB247F014085FFA88F841462846FFF788
:1020100046FE002C40F0FD83410540F1F88347F077
:102020001101C9B22846FFF73AFE306038E0CE2AE7
:1020300000F0478414D8B82A00F01684B92A7FF437
:10204000B5AE0F0147F06C07FFB239462846002CA9
:1020500040F02784FFF723FEC0F3035030601FE0F9
:10206000D22A00F04484D32A00F05484D12A7FF489
:102070009DAE2021A94041F01901C9B2002840F0CD
:102080002F842846FFF70BFE306009E02021A9408D
:1020900041F00D01C9B230B92846FFF700FE3060AB
:1020A0002046BDE8F8831A682846FFF787FD00241C
:1020B000F6E72021A94041F00101C9B220B9284624
:1020C000FFF7EDFD3060EBE71A682846FFF776FD75
:1020D0000024E5E72021A94041F00701C9B238B941
:1020E0002846FFF7DCFD3060DAE700BF1429002046
:1020F0000122B74B28465A5532680024002AB8BF3F
:102100005242FFF75BFDCBE7002840F053842021CB
:10211000A94041F00201C9B22846FFF7C0FD10F402
:10212000000318BF4FF07F4318433060B8E7202703
:1021300032688F40002AB8BF5242F9B22846C3F82D
:10214000BC22FFF7ACFD044608B10024A8E73268C2
:1021500047F00701002AB8BF5242C9B22846FFF72C
:102160002DFD9DE72021A94041F00601C9B220B90B
:102170002846FFF794FD306092E71A682846FFF77B
:102180001DFD00248CE720278F4047F01007FFB289
:10219000394628462CB9FFF782FDC0F30420306091
:1021A0007EE7FFF77CFD336820F4F8521B0203F44E
:1021B000F8531A4339462846FFF700FD00246FE71D
:1021C000FFF76DFD336820F01F0203F01F031A4371
:1021D00039462846FFF7F2FC002461E7002840F06A
:1021E000EC832021A94041F01501C9B22846FFF730
:1021F00056FDC0F34020306052E7002840F0E083F5
:102200002021A94041F01501C9B22846FFF747FD3A
:1022100010F0020F0CBF01230023336040E720279A
:102220008F4047F01407FFB2394628462CB9FFF714
:1022300036FDC0F34000306032E7FFF730FD336811
:1022400020F00202002B14BF0023022339461A4358
:102250002846FFF7B3FC002422E720278F4047F0F1
:102260001407FFB2394628462CB9FFF718FD00F0D5
:102270000100306014E7FFF712FD326820F0010022
:10228000002A14BF024640F0010239462846FFF7F3
:1022900095FC002404E71A682846FFF78FFC002409
:1022A000FEE62021A94041F00401C9B220B9284628
:1022B000FFF7F5FC3060F3E61A682846FFF77EFC6E
:1022C0000024EDE62021A94041F00501C9B220B962
:1022D0002846FFF7E4FC3060E2E61A682846FFF77C
:1022E0006DFC0024DCE61A682846FFF767FC002432
:1022F000D6E62021A94041F00A01C9B220B92846FA
:10230000FFF7CDFC3060CBE61A682846FFF756FC95
:102310000024C5E62021A94041F00301C9B220B93B
:102320002846FFF7BCFC3060BAE61A682846FFF77B
:1023300045FC0024B4E61A682846FFF73FFC002459
:10234000AEE62021A94041F00C01C9B220B92846CF
:10235000FFF7A5FC3060A3E61A682846FFF72EFCBD
:1023600000249DE62021A94041F01101C9B220B905
:102370002846FFF794FC306092E61A682846FFF77B
:102380001DFC00248CE62021A94041F01201C9B2B5
:1023900020B92846FFF783FC306081E61A6828469A
:1023A000FFF70CFC00247BE61A682846FFF706FCC2
:1023B000002475E60F0147F06C07FFB23946284646
:1023C00044B9FFF76CFCC0F38040306068E600BFA2
:1023D00070000020FFF763FC336820F480229B0428
:1023E00003F480231A4339462846FFF7E7FB00240D
:1023F00056E6002840F0EA822020C44B88401B6843
:1024000040F0020003EB80004368336048E61B683D
:10241000102B4AD00DDC022B43D004DC012B16D04C
:102420004FF0FF3314E0042B3DD0082BF8D10523E7
:102430000EE0402B3BD003DC202BF1D1032307E03F
:10244000802B36D0B3F5807FEAD1002300E008234B
:102450003360336801333FF478AE2C0144F06C04F0
:10246000E4B221462846FFF71AFC336820F0706278
:102470001B0603F070631A4321462846FFF79EFBB4
:1024800021462846FFF70BFC336820F070621B06DC
:1024900003F0706321461A432846FFF78FFB0024A0
:1024A000FEE50723D4E70623D2E70423D0E702237F
:1024B000CEE70123CCE70F0147F06C07FFB23946A6
:1024C00028462CB9FFF7EBFBC0F3C1303060E7E5DD
:1024D000FFF7E5FB336820F4C032DB0303F4C033BD
:1024E0001A4339462846FFF769FB0024D8E50F0157
:1024F00047F06C07FFB2394628462CB9FFF7CFFBEF
:10250000C0F380303060CBE5FFF7C9FB336820F4BF
:1025100080429B0303F480431A4339462846FFF761
:102520004DFB0024BCE5FFF7BAFB336820F4805272
:102530001B0303F480531A4339462846FFF73EFB3A
:102540000024ADE50F0147F06C07FFB2394628467D
:10255000FFF7A5FB3946814600F480482846B4B908
:10256000B8F1000F05D0FFF79AFBC0F3C31030603D
:1025700096E5FFF794FB19F4006FC0F3021001D148
:102580003060E2E540F008003060444688E5B8F18C
:10259000000F0ED0FFF783FB336820F4F062DB01FD
:1025A00003F4F0631A4339462846FFF707FB00247B
:1025B00076E5FFF774FB336820F070021B0103F02F
:1025C00070031A4339462846FFF7F8FA444667E590
:1025D0000F0147F06C07FFB239462846FFF75FFB53
:1025E000394600F4804828467CB9B8F1000F05D080
:1025F000FFF755FBC0F30210306051E5FFF74FFBCA
:10260000C0F3C310306044464AE5B8F1000F0ED065
:10261000FFF745FB336820F070021B0103F07003E5
:102620001A4339462846FFF7C9FA002438E5FFF770
:1026300036FB336820F4F062DB0103F4F0631A43E5
:1026400039462846FFF7BAFA444629E5FFF727FB43
:10265000336820F00F0203F00F031A43394628466F
:10266000FFF7ACFA00241BE50F0147F06D07FFB23E
:10267000394628462CB9FFF712FBC0F3C030306052
:102680000EE5FFF70CFB336820F40042DB039BB23E
:102690001A4339462846FFF791FA002400E547F02F
:1026A0006D07FFB2394628462CB9FFF7F8FAC0F398
:1026B00041303060F4E4FFF7F2FA336820F4C042AE
:1026C0005B0303F4C0431A4339462846FFF776FA02
:1026D0000024E5E447F06D07FFB2394628462CB9DF
:1026E000FFF7DDFAC0F303203060D9E4FFF7D7FA33
:1026F000336820F470621B0203F470631A43394696
:102700002846FFF75BFA0024CAE400BF1429002022
:10271000FFF7C5FA336820F060025B0103F0600345
:102720001A4339462846FFF749FA0024B8E40F0156
:1027300047F06D07FFB2394628462CB9FFF7AFFACC
:1027400000F00F003060ABE4FFF7A9FA336820F027
:102750000F0203F00F031A4339462846FFF72EFAFB
:1027600000249DE40F0147F06D07FFB2394628466B
:102770002CB9FFF794FAC0F30060306090E4FFF7E3
:102780008EFA336820F080721B0603F080731A43C0
:1027900039462846FFF712FA002481E4FFF77FFA52
:1027A000336820F4FE021B0403F4FE031A43394687
:1027B0002846FFF703FA002472E40F0147F06C0784
:1027C000FFB2394628462CB9FFF769FAC0F34040FA
:1027D000306065E4FFF763FA336820F400325B048D
:1027E00003F400331A4339462846FFF7E7F900247B
:1027F00056E4002840F0ED80090141F06F01C9B2B4
:102800002846FFF74CFAC0F30440306048E43460D7
:1028100046E447F011013268C9B22846FFF7CEF905
:1028200041462846FFF73BFA336820F48062002BCC
:102830000CBF00234FF4806341461A432846FFF73C
:10284000BDF900242CE42021A94041F01101C9B2B6
:1028500020B92846FFF723FA306021E41A68284699
:10286000FFF7ACF900241BE40F0147F06C07FFB23F
:10287000394628462CB9FFF712FAC0F340303060D1
:102880000EE4FFF70CFA336820F400525B0303F404
:1028900000531A4339462846FFF790F90024FFF702
:1028A000FFBBFFF7FCF9336820F470021B0503F44B
:1028B00070031A4339462846FFF780F90024FFF7D2
:1028C000EFBB002840F08880090141F06F01C9B2D8
:1028D0002846FFF7E4F9C0F309003060FFF7E0BBDA
:1028E0001A682846FFF76AF90024FFF7D9BB2021B0
:1028F000A94041F01A01C9B228B92846FFF7CFF91B
:102900003060FFF7CDBB1A682846FFF757F900245F
:10291000FFF7C6BBE8B979B101297FF4C1AB014625
:102920002846FFF7BCF900F06000A0F120035842F0
:1029300058413060FFF7B4BB0846FFF7B0F900F02C
:102940001800A0F110025042504130602C46FFF7B1
:10295000A7BB21B1012917D00024FFF7A1BB08466E
:10296000FFF79DF9336853B120F0080242F01002DE
:1029700000210846FFF722F90024FFF791BB20F061
:10298000100242F00802F3E700212846FFF787F91A
:10299000336853B120F0400242F0200200210120B0
:1029A000FFF70CF90024FFF77BBB20F0200242F078
:1029B0004002F3E70424FFF773BB0424FFF770BB66
:1029C0000424FFF76DBB0424FFF76ABB0424FFF760
:1029D00067BB0424FFF764BB0424FFF761BB012934
:1029E000134603D802460020FFF7C4B908207047F9
:1029F00007B50129019207D8024601AB0120FFF774
:102A0000B9F903B05DF804FB0820FAE708B5222104
:102A10000020FFF744F950B942210120FFF73FF9A8
:102A200028B9044B1868BDE808400DF0E5BD00204A
:102A300008BD00BF1429002070B5434C434E201D33
:102A40000DF044FDF5686B6803F5AA72C4F8A02286
:102A500003F5B872C4F8A42203F56F72C4F8A82273
:102A600003F5767203F1C800C4F8AC2203F57D7259
:102A700003F58263C4F8B4322B68C4F8B022DB6873
:102A8000C4F89C0298472B68D4F8A802DB689847E2
:102A90002B68D4F8A8029B6998472B68D4F8A00249
:102AA0001B6998472B68D4F8A4021B6998472B68C8
:102AB000D4F8B4021B6998472B68D4F8AC021B69A0
:102AC00098472B68D4F8B0021B6998476B68326945
:102AD00003F5377353601E4BC4F8B8221D495A6979
:102AE0000120C2F804121C491070C2F8081200211B
:102AF00022605170194A32211A62194ADA61194A60
:102B00009A61194A5A62194A9A63194A5A63194AC8
:102B10009A62194ADA62194A9A64194A5A64194A35
:102B20005A65194A1A65194ADA64194A1A66194A1D
:102B3000DA6502221A74B622C3E90221164A9A659E
:102B4000BDE87040FEF7AEBF142900207086020871
:102B5000006100200D2A0108111A0108491C010812
:102B60009D1C0108991C0108951C0108DF2901081A
:102B7000F1290108DF1B0108531D0108D91B0108B9
:102B8000451D0108E9190108451A01081D1A010827
:102B9000A51A0108DD190108E91A010801289FBFDB
:102BA000034B53F8203000200B6088BF082070478B
:102BB000E42B00200022014B5A6070470061002086
:102BC00070B50546084C0146D4F8983222460020DC
:102BD0000DF05FFDD4F8983222462946BDE87040DA
:102BE00001200DF056BD00BFE42B0020024BD3F8AE
:102BF00098020DF098BD00BFE42B0020012810B50D
:102C0000144603D002280FD004200CE00A4B0B4AD4
:102C1000DB68D2F8A0021B685B6A9847003018BFD7
:102C200001202060002010BD034B044ADB68D2F86D
:102C3000A4021B685B6AF0E770860208E42B0020A0
:102C4000022804BF0C4B93F8E80038B90B4BDB6843
:102C50001B685B690A4AD2F89C021847012809D10F
:102C6000054B93F8E830012B04D1044BDB681B685B
:102C70009B69EFE7704700BF006100207086020883
:102C8000E42B002070B50020FFF7DAFF094B0A4C57
:102C9000DD68D4F89C022B689B6898472B68D4F8B1
:102CA000A0029B6898472B68D4F8A4029B68BDE8F3
:102CB0007040184770860208E42B00202DE9F84385
:102CC0000F4691469846194C0021D4F8A83247F097
:102CD00080009B689DF820609DF824509847D4F8A8
:102CE000A83200219B6848469847D4F8A8320021B2
:102CF0009B6840469847D4F8A83200219B6830462C
:102D00009847D4F8A83228469B680121984748EA9A
:102D10000928D4F8983246EA082607F07F0703EB23
:102D2000870745EA06257D60BDE8F883E42B00208F
:102D300007B5D3B20193C2F307230093C2F307434D
:102D4000120EFFF7BBFF03B05DF804FB0020FFF796
:102D5000EFBF01282DE9F34105460F462BD8202669
:102D6000164B864003EB000898F8942274B272B1B7
:102D7000D3F8983246F0070203EB820344F00701D0
:102D80005A68C9B2FFF7D4FF002388F8943244F0A0
:102D90000D0100243A46C9B22846FFF7C9FF28466C
:102DA000CDE9004423462246F1B2FFF787FF2046D3
:102DB00002B0BDE8F0810820FAE700BFE42B002054
:102DC000012873B505460C4620D82026864084EAA3
:102DD000E47246F00701A2EBE472C9B2FFF7A8FF64
:102DE00001220B4B002C2B4483F894224FF000045B
:102DF000ACBF134602232846019300942346224683
:102E0000F1B2FFF75BFF204602B070BD0820FBE780
:102E1000E42B00200021D3E74942D1E7D0E738B5C1
:102E2000284D01F07F042B1993F81432DB0705D4E9
:102E3000D5F8983203EB8404606838BDD5F8A83221
:102E400000219B68204698470021D5F8A832084603
:102E50009B6898470021D5F8A83208469B68984798
:102E60000021D5F8A83208469B689847D5F8A832C3
:102E700001219B6800209847D5F8A83200219B6863
:102E8000204698470021D5F8A83208469B68984705
:102E90000021D5F8A83204029B6808469847002113
:102EA000D5F8A83204439B6808469847D5F8A8325D
:102EB000240204439B6801210020984724022043F8
:102EC000BBE700BFE42B002010B500201446FFF73D
:102ED000A6FF206010BD38B50D462021814041F08D
:102EE0000101C9B20446FFF79AFF2968014429602D
:102EF0002046BDE838402CE71C2A2DE9F041044665
:102F00000D461E4600F0308300F2AF800C2A00F020
:102F10003D8253D8052A00F0DC8121D8022A00F036
:102F2000948109D8002A00F06E81012A00F07C818A
:102F300004242046BDE8F081032A00F0A181042A80
:102F4000F6D12021C64BA940D3F8983241F00707AB
:102F5000BA001344002840F0A6815B683360E8E7BC
:102F6000082A00F0F28114D8062A00F0C381072A4B
:102F7000DED120278F4047F01007FFB239462846A0
:102F8000002C40F0D481FFF74AFF00F01F003060B2
:102F9000CFE70A2A00F0E8810B2AC9D1002840F0C7
:102FA000BA852021A94041F01501C9B22846FFF792
:102FB00036FFC04300F001003060BAE7122A00F08B
:102FC0006F8227D80F2A00F0438211D80D2A00F013
:102FD0000B820E2AACD12021A94041F01401C9B2C4
:102FE000002840F02F822846FFF719FF3060A0E745
:102FF000102A00F03E82112A9AD12021A94041F0E6
:103000000801C9B2002840F045822846FFF707FFB3
:1030100030608EE7152A00F06B8211D8132A00F079
:103020005082142A84D12021A94041F00B01C9B259
:10303000002840F057822846FFF7F1FE306078E71D
:10304000172A00F07782C0F06482182A7FF470AFEC
:103050002021A94041F01301C9B2002840F07E822E
:103060002846FFF7DCFE306063E7AB2A00F02384DC
:1030700061D8A52A00F0288331D8A22A00F0DD8289
:1030800018D81D2A00F08C828C2A7FF451AF0028BA
:1030900040F08E82090141F06C0101F0FC012846EC
:1030A000FFF7BDFE4FF48073C0F3036043FA00F0F6
:1030B00030603EE7A32A00F0DC82A42A7FF438AF18
:1030C0000F0147F06C07FFB239462846002C40F04C
:1030D000EC82FFF7A4FEC0F30030306029E7A82A95
:1030E00000F09E8312D8A62A00F04483A72A7FF41A
:1030F0001FAF0F0147F06C07FFB239462846002C7E
:1031000040F08383FFF78BFE346012E7A92A00F0BA
:10311000A483AA2A7FF40CAF0F0147F06D07FFB21A
:1031200039462846002C40F0B683FFF778FEC0F3FE
:1031300003203060FDE6B52A00F04E842CD8AE2A7C
:1031400000F0078414D8AC2A00F0D683AD2A7FF4AF
:10315000EFAE0F0147F06D07FFB239462846002C4D
:1031600040F0E783FFF75BFEC0F300603060E0E60D
:10317000B32A00F01384B42A7FF4DAAE002840F0BA
:10318000D084090141F06F01C9B22846FFF747FE1C
:10319000C0F304403060CCE6CE2A00F0688414D836
:1031A000B62A00F04184B82A7FF4C2AE0F0147F07E
:1031B0006C07FFB239462846002C40F04884FFF7E0
:1031C0002EFEC0F340303060B3E6D12AFFF4B0AE3B
:1031D000D22A40F29484D32A7FF4AAAE002840F089
:1031E0006184002900F0518401297FF4A2AE0146D8
:1031F0002846FFF714FE00F06000A0F120035842BB
:103200005841306095E62021A94041F00D01C9B236
:1032100020B92846FFF703FE30608AE61A68284680
:10322000FFF786FD002484E62021A94041F001013A
:10323000C9B220B92846FFF7F2FD306079E61A6876
:103240002846FFF775FD002473E62021A94041F0D0
:103250000701C9B230B92846FFF7E1FD306068E6E2
:10326000E42B00200122B94B28462B4483F89422FA
:1032700032680024002AB8BF5242FFF759FD58E6D1
:10328000002840F03F842021A94041F00201C9B24A
:103290002846FFF7C4FD10F4000318BF4FF07F432A
:1032A0001843306045E63268C9B2002AB8BF5242BE
:1032B0005A602846FFF7B3FD044608B1002438E6FB
:1032C0003268F9B2002AB8BF52422846FFF730FDF3
:1032D0002FE62021A94041F00601C9B220B92846B5
:1032E000FFF79DFD306024E61A682846FFF720FDB1
:1032F00000241EE620278F4047F01007FFB2394612
:1033000028462CB9FFF78BFDC0F30420306010E68F
:10331000FFF785FD336820F4F8521B0203F4F853DD
:103320001A4339462846FFF703FD002401E6FFF75C
:1033300076FD336820F01F0203F01F031A4339465D
:103340002846FFF7F5FC0024F3E5002840F0DD8374
:103350002021A94041F01501C9B22846FFF75FFDC1
:10336000C0F340203060E4E5002840F0D183202104
:10337000A94041F01501C9B22846FFF750FD10F0F1
:10338000020F0CBF012300233360D2E520278F40BA
:1033900047F01407FFB2394628462CB9FFF73FFD26
:1033A000C0F340003060C4E5FFF739FD336820F01A
:1033B0000202002B0CBF0023022339461A43284681
:1033C000FFF7B6FC39462846FFF729FD336820F0A1
:1033D0000802022B14BF0023082339461A4328464B
:1033E000FFF7A6FC0024A4E520278F4047F0140730
:1033F000FFB2394628462CB9FFF711FD00F0010055
:10340000306096E5FFF70BFD326820F00100002ADE
:103410000CBF024640F0010239462846FFF788FCFF
:1034200039462846FFF7FBFC336820F00402022BE4
:1034300014BF0023042339461A432846FFF778FCBB
:10344000002476E51A682846FFF772FC002470E530
:103450002021A94041F00401C9B220B92846FFF754
:10346000DEFC306065E51A682846FFF761FC002441
:103470005FE52021A94041F00501C9B220B92846E5
:10348000FFF7CDFC306054E51A682846FFF750FC82
:1034900000244EE51A682846FFF74AFC002448E558
:1034A0002021A94041F00A01C9B220B92846FFF7FE
:1034B000B6FC30603DE51A682846FFF739FC002469
:1034C00037E52021A94041F00301C9B220B92846BF
:1034D000FFF7A5FC30602CE51A682846FFF728FCAA
:1034E000002426E51A682846FFF722FC002420E580
:1034F0002021A94041F00C01C9B220B92846FFF7AC
:103500008EFC306015E51A682846FFF711FC002490
:103510000FE52021A94041F01101C9B220B9284688
:10352000FFF77DFC306004E51A682846FFF700FCD1
:103530000024FEE42021A94041F01201C9B238B9AB
:103540002846FFF76CFC3060F3E400BFE42B00205A
:103550001A682846FFF7ECFB0024EAE41A682846BC
:10356000FFF7E6FB0024E4E40F0147F06C07FFB22D
:10357000394628462CB9FFF752FCC0F38040306032
:10358000D7E4FFF74CFC336820F480229B0403F45B
:1035900080231A4339462846FFF7CAFB0024C8E4B3
:1035A000002840F0BB82CB4B53F821303360C0E49D
:1035B0001B68102B3BD00DDC022B34D004DC012B1C
:1035C00016D04FF0FF3314E0042B2ED0082BF8D187
:1035D00005230EE0402B2CD003DC202BF1D103235C
:1035E00007E0802B27D0B3F5807FEAD1002300E0ED
:1035F00008233360336801333FF460AE2C0144F09C
:103600006C04E4B221462846FFF709FC336820F039
:1036100070621B0603F0706321461A432846FFF7C9
:1036200087FB002485E40723E3E70623E1E704237F
:10363000DFE70223DDE70123DBE70F0147F06C073B
:10364000FFB2394628462CB9FFF7E9FBC0F3C13079
:1036500030606EE4FFF7E3FB336820F4C032DB0335
:1036600003F4C0331A4339462846FFF761FB0024B0
:103670005FE40F0147F06C07FFB2394628462CB9CA
:10368000FFF7CDFBC0F38030306052E4FFF7C7FB9B
:10369000336820F480429B0303F480431A43394685
:1036A0002846FFF745FB002443E4FFF7B8FB3368E7
:1036B00020F480521B0303F480531A4339462846F2
:1036C000FFF736FB002434E40F0147F06C07FFB22C
:1036D00039462846FFF7A3FB00F48048B4B9B8F197
:1036E000000F07D039462846FFF799FBC0F3C310F7
:1036F00030601EE40311010503F0700301D4336050
:10370000DCE543F008033360444612E439462846BA
:10371000B8F1000F0FD0FFF782FB336820F4F0629E
:10372000DB0103F4F0631A4339462846FFF700FB38
:103730000024FFF7FEBBFFF772FB326820F4006045
:10374000120202F40062024339462846FFF7F0FAFB
:1037500039462846FFF763FB336820F070021B01EF
:1037600003F070031A4339462846FFF7E1FA44464E
:10377000FFF7DFBB0F0147F06C07FFB23946284661
:10378000FFF74DFB394680462846C4B918F48044FB
:1037900007D0FFF744FBC0F3021030600024FFF7AE
:1037A000C8BBFFF73CFB18F4006FC0F3C31001D196
:1037B000306083E540F008003060FFF7BABBFFF7E8
:1037C0002EFB10F48044394628460FD0FFF727FB24
:1037D000336820F070021B0103F070031A4339466E
:1037E0002846FFF7A5FA0024FFF7A3BBFFF717FB56
:1037F000336820F4F062DB0103F4F0631A433946C6
:103800002846FFF795FAFFF794BBFFF708FB394608
:1038100020F00F022846FFF78BFA0024FFF789BB40
:103820000F0147F06D07FFB23946284634B9FFF75C
:10383000F6FAC0F3C0303060FFF77BBBFFF7EFFA5A
:10384000336820F40042DB039BB21A433946284612
:10385000FFF76EFA0024FFF76CBB0F0147F06D070E
:10386000FFB23946284634B9FFF7D9FAC0F34130E0
:103870003060FFF75EBBFFF7D2FA336820F4C04236
:103880005B0303F4C0431A4339462846FFF750FA56
:103890000024FFF74EBBFFF7C2FA336820F47062D2
:1038A0001B0203F470631A4339462846FFF740FAB7
:1038B0000024FFF73EBB0F0147F06D07FFB239460A
:1038C00028464CB9FFF7ABFAC0F341103060FFF760
:1038D00030BB00BFE42B0020FFF7A1FA336820F0D3
:1038E00060025B0103F060031A4339462846FFF784
:1038F0001FFA0024FFF71DBB0F0147F06D07FFB251
:103900003946284634B9FFF78AFA00F00F003060D4
:10391000FFF70FBBFFF783FA336820F00F0203F0C5
:103920000F031A4339462846FFF702FA0024FFF72F
:1039300000BBFFF774FA336820F080721B0603F0B7
:1039400080731A4339462846FFF7F2F90024FFF73F
:10395000F0BA0F0147F06D07FFB2394628466CB93F
:10396000FFF75DFA001400F07F0310F0400018BF6D
:103970006FF07F0018433060FFF7DBBAFFF74FFAB4
:10398000336820F4FE021B0403F4FE031A43394695
:103990002846FFF7CDF90024FFF7CBBA0F0147F017
:1039A0006C07FFB23946284634B9FFF738FAC0F33E
:1039B00040403060FFF7BDBAFFF731FA336820F4BA
:1039C00000325B0403F400331A4339462846FFF7FC
:1039D000AFF90024FFF7ADBA20278F407FB247F040
:1039E0001101C9B228B92846FFF719FA3060FFF76C
:1039F000A0BA47F014041A68E4B22846FFF798F911
:103A000021462846FFF70BFA336820F48062002B2A
:103A10000CBF00234FF4806321461A432846FFF76A
:103A200087F90024FFF785BA2021A94041F0110150
:103A3000C9B228B92846FFF7F2F93060FFF779BA22
:103A40001A682846FFF774F90024FFF772BAFFF7E7
:103A5000E6F9336820F400525B0303F400531A4381
:103A600039462846FFF764F90024FFF762BA0028B8
:103A70005AD1090141F06F01C9B22846FFF7CFF9C9
:103A8000C0F309003060FFF754BA0846FFF7C7F9E2
:103A900000F01800A0F110025042504130602C4656
:103AA000FFF747BA21B1012915D00024FFF741BA29
:103AB0000846FFF7B4F9336820F0180243B142F02A
:103AC000100200210846FFF733F90024FFF731BA4E
:103AD00042F00802F5E700212846FFF7A0F9336815
:103AE00020F0600243B142F0200200210120FFF7E4
:103AF0001FF90024FFF71DBA42F04002F5E7002449
:103B0000FFF717BA0424FFF714BA0424FFF711BA19
:103B10000424FFF70EBA0424FFF70BBA0424FFF7BE
:103B200008BA0424FFF705BA0424FFF702BA07B560
:103B30000129019207D8024601AB0120FFF7DCF909
:103B400003B05DF804FB0820FAE70129134603D807
:103B500002460020FFF7D0B90820704708B522219F
:103B60000020FFF75CF958B942210120FFF757F90F
:103B700030B9044BD3F89802BDE808400CF0CABD38
:103B8000002008BDE42B002070B5304C304E20469C
:103B90000CF042FDF5686B6803F5AA7203F1C800EA
:103BA00003F5B873C4F8A4322B68C4F8A022DB680C
:103BB000C4F89C0298472B68D4F8A0021B69984768
:103BC0002B68D4F8A4021B6998476B68326903F527
:103BD000377353601F4BC4F8A8221F495A6902204B
:103BE000C2F804121D49C4F89822C2F80812012133
:103BF0001170002151701A4A32211A62194A187440
:103C0000DA61194A9A61194A5A62194A9A63194A39
:103C10005A63194A9A62194ADA62194A9A64194A25
:103C20005A64194A5A65194A1A65194ADA64194ACE
:103C30001A66194ADA654FF48C72C3E90221174AF1
:103C40009A65BDE87040FEF7FBBF00BFE42B002083
:103C500070860208006100205D3B0108ED2B010821
:103C6000C12D01081D2E0108192E0108152E01086D
:103C70004B3B01082F3B0108532D0108D72E0108AB
:103C80004D2D0108C92E0108C12B0108FD2B01088B
:103C90009D2B0108412C0108B52B0108852C01083A
:103CA00001289FBF044B03EB8000C369002094BF31
:103CB0000B600820704700BF9C2E00200022014BA3
:103CC0005A60704700610020014601480CF0C1BEF7
:103CD0009C2E00200A46014601480CF059BD00BF49
:103CE0009C2E002010B500201446FFF7F3FF206043
:103CF00010BD38B514460A46014603481D460CF06F
:103D000047FD2040E84038BD9C2E002013460A465F
:103D1000014601480CF038BD9C2E00200020F5E73C
:103D20002DE9F0470C4D994606460F4690460A4647
:103D300001462846089C0CF02BFD04FA09F242408B
:103D400002EA080282EA000331463A462846BDE804
:103D5000F0470CF019BD00BF9C2E002001480CF06C
:103D6000D8BD00BF9C2E002008B522210020FFF7FF
:103D7000B1FF48B942210120FFF7ACFF20B9BDE8EF
:103D8000084002480CF0ADBD002008BD9C2E00206C
:103D9000012810B5144612D003D302281CD00420E9
:103DA0000AE0114B114ADB6824681B68D2F8B002A4
:103DB0001CB15B699847002010BD9B69FAE70A4B6C
:103DC0000A4ADB68D2F8A8021B685B6A9847003091
:103DD00018BF01202060EEE7034B044ADB68D2F8ED
:103DE000AC021B685B6AF1E7708602089C2E00201B
:103DF000022804BF0C4B93F8E80038B90B4BDB6882
:103E00001B685B690A4AD2F8A4021847012809D145
:103E1000054B93F8E830012B04D1044BDB681B6899
:103E20009B69EFE7704700BF0061002070860208C1
:103E30009C2E002070B50020FFF7DAFF134B144CC6
:103E4000DD68D4F8A4022B689B6898472B68D4F8E7
:103E5000A8029B6898472B68D4F8AC029B689847E7
:103E60002B68D4F8BC029B6898472B68D4F8B4023E
:103E70009B6898472B68D4F8B8029B6898472B68D2
:103E8000D4F8B0029B68BDE87040184770860208FD
:103E90009C2E002001282DE9F041044688461FD8B9
:103EA0002025104F854007EB8007D7F8C0226EB25F
:103EB0003AB146F00701C9B2FFF728FF0023C7F85F
:103EC000C03246F00D014246C9B22046FFF71EFF40
:103ED00020460022E9B2FFF719FF0020BDE8F0817B
:103EE0000820FBE79C2E002038B50D46202181409C
:103EF00041F00101C9B20446FFF7ECFE2968014414
:103F000029602046BDE83840C4E701282DE9F0418A
:103F10000446884623D82025124F854007EB8007AA
:103F2000D7F8C03245F00706F6B223B93146FFF79D
:103F3000D1FEC7F8C00288EAE872A2EBE872314607
:103F40002046FFF7E3FEB8F1000F2046B4BF02227F
:103F50000122E9B2FFF7DAFE0020BDE8F081082077
:103F6000FBE700BF9C2E00200021CEE74942CCE7B2
:103F7000CBE71C2A2DE9F34104460D461E4600F00E
:103F8000FB8200F2AE800C2A00F03B8252D8052A58
:103F900000F0E3811FD8022A00F0A28107D8002A8E
:103FA00000F07781012A00F0888104247BE1032A54
:103FB00000F0AA81042AF8D12021C84BA940D3F8E7
:103FC000C83241F00707BA001344002840F0AF811F
:103FD0005B68336067E1082A00F0F18113D8062A94
:103FE00000F0CC81072AE0D12021A94041F0100146
:103FF000C9B2002840F0DA8103461F222846FFF7A5
:1040000078FE30604FE10A2A00F0E9810B2ACCD11A
:10401000002840F04C852021A94041F015010346BD
:104020000122C9B22846FFF764FEB0FA80F04009C9
:10403000306038E1122A00F03E8227D80F2A00F0C3
:10404000128211D80D2A00F0F2810E2AADD1202162
:10405000A94041F01401C9B2002840F0FE81284671
:10406000FFF738FE30601EE1102A00F00D82112AA1
:104070009BD12021A94041F00801C9B2002840F09D
:1040800014822846FFF726FE30600CE1152A00F066
:104090003A8211D8132A00F01F82142A85D12021D8
:1040A000A94041F00B01C9B2002840F02682284601
:1040B000FFF710FE3060F6E0172A00F04682C0F0ED
:1040C0003382182A7FF471AF2021A94041F01301F7
:1040D000C9B2002840F04A822846FFF7FBFD306055
:1040E000E1E0AC2A00F0C98362D8A52A00F0DA82A8
:1040F00032D8A22A00F09E8219D81D2A00F05382DD
:104100008C2A7FF452AF002840F05682090141F01A
:104110006C0118234FF0706201F0FC012846FFF794
:10412000E8FD4FF4807343FA00F03060BBE0A32A4F
:1041300000F09782A42A7FF438AF090141F06C01A6
:10414000C9B2002840F0A4820C234FF480522846C4
:10415000FFF7CFFD3060A6E0A82A00F0428313D815
:10416000A62A00F0F282A72A7FF41FAF090141F0CE
:104170006C01C9B2002840F02B8303460F22284669
:10418000FFF7B7FD30608EE0AA2A4FEA011100F078
:10419000558340F23D8341F06D01C9B2002840F0E3
:1041A0006383052360222846FFF7A3FD30607AE091
:1041B000B62A00F0D6833DD8B32A00F097831AD8E8
:1041C000AD2A00F07283AE2A7FF4EFAE090141F010
:1041D0006D01C9B2002840F07F8310234FF4FE0226
:1041E0002846FFF786FD10F0400318BF6FF07F03ED
:1041F0001843306057E0B42A00F08F83B52A7FF46B
:10420000D4AE20278F407FB247F014085FFA88F8B9
:10421000002840F0918341462846FFF75BFD4105A9
:1042200040F1908047F01101C9B22846FFF752FDD6
:10423000306038E0CE2A00F0C68314D8B82A00F0E7
:10424000A183B92A7FF4B1AE090141F06C01C9B272
:10425000002840F0AE8314234FF470022846FFF785
:1042600048FD30601FE0D22A00F0C183D32A00F05D
:10427000CF83D12A7FF499AE2021A94041F01901C2
:10428000C9B2002840F0AD832846FFF723FD306017
:1042900009E02021A94041F00D01C9B238B92846F2
:1042A000FFF718FD3060204602B0BDE8F0811A68C3
:1042B0002846FFF72BFD0024F5E72021A94041F017
:1042C0000101C9B220B92846FFF704FD3060EAE7D2
:1042D0001A682846FFF71AFD0024E4E79C2E002008
:1042E0002021A94041F00701C9B220B92846FFF7B3
:1042F000F1FC3060D7E71A682846002AB8BF52425E
:10430000FFF704FD0024CEE7002840F0C8832021F9
:10431000A94041F00201C9B22846FFF7DBFC10F4C6
:10432000000318BF4FF07F4318433060BBE732688B
:10433000C9B2002AB8BF52425A602846FFF7CAFCE9
:10434000044608B10024AEE73268F9B2002AB8BFCB
:1043500052422846FFF7DAFCA5E72021A94041F0A8
:104360000601C9B220B92846FFF7B4FC30609AE7CD
:104370001A682846FFF7CAFC002494E72021A940C8
:1043800041F01001C9B238B908234FF4F852284659
:10439000FFF7AFFC306086E71B684FF4F8520093DC
:1043A00028460823FFF7BCFC00247CE71B681F227B
:1043B000009328460023FFF7B3FC002473E700288E
:1043C00040F06F832021A94041F0150109234FF4EB
:1043D0000072C9B22846FFF78CFC306063E7002802
:1043E00040F062832021A94041F0150101230222FF
:1043F000C9B22846FFF77DFCB0FA80F04009306072
:1044000051E72021A94041F01401C9B230B901237C
:1044100002222846FFF76DFC306044E71B68022249
:10442000009328460123FFF77BFC00243BE7202173
:10443000A94041F01401C9B230B900230122284635
:10444000FFF757FC30602EE71B68012200932846D7
:104450000023FFF765FC002425E71A682846FFF7CC
:1044600055FC00241FE72021A94041F00401C9B2F6
:1044700020B92846FFF72EFC306014E71A6828465A
:10448000FFF744FC00240EE72021A94041F005017C
:10449000C9B220B92846FFF71DFC306003E71A684F
:1044A0002846FFF733FC0024FDE61A682846FFF78C
:1044B0002DFC0024F7E62021A94041F00A01C9B2F1
:1044C00020B92846FFF706FC3060ECE61A6828465B
:1044D000FFF71CFC0024E6E62021A94041F003017F
:1044E000C9B220B92846FFF7F5FB3060DBE61A6851
:1044F0002846FFF70BFC0024D5E61A682846FFF78C
:1045000005FC0024CFE62021A94041F00C01C9B2EE
:1045100020B92846FFF7DEFB3060C4E61A6828465B
:10452000FFF7F4FB0024BEE62021A94041F0110171
:10453000C9B220B92846FFF7CDFB3060B3E61A6850
:104540002846FFF7E3FB0024ADE62021A94041F017
:104550001201C9B220B92846FFF7BCFB3060A2E6C1
:104560001A682846FFF7D2FB00249CE61A68284602
:10457000FFF7CCFB002496E6090141F06C01C9B2BB
:1045800038B912234FF480222846FFF7B2FB30607F
:1045900089E61B684FF48022009328461223FFF718
:1045A000BFFB00247FE6002840F08482B94800EB7E
:1045B0008100C369336076E61B68102B34D00DDCB4
:1045C000022B2DD004DC012B16D04FF0FF3314E06A
:1045D000042B27D0082BF8D105230EE0402B25D043
:1045E00003DC202BF1D1032307E0802B20D0B3F58F
:1045F000807FEAD1002300E0082333603368581C31
:104600003FF4A0AE290141F06C0100934FF07062BD
:10461000182301F0FC012846FFF782FB002442E644
:104620000723EAE70623E8E70423E6E70223E4E7B3
:104630000123E2E7090141F06C01C9B238B90F2347
:104640004FF4C0322846FFF754FB30602BE61B685E
:104650004FF4C032009328460F23FFF761FB00247C
:1046600021E6090141F06C01C9B238B90E234FF4BB
:1046700080422846FFF73DFB306014E61B684FF48C
:104680008042009328460E23FFF74AFB00240AE6E7
:104690001B684FF48052009328460C23FFF740FB21
:1046A000002400E60F0147F06C07FFB240BB0E2369
:1046B0004FF4804239462846FFF71BFB804640B145
:1046C00007234FF4F06239462846FFF712FB3060AB
:1046D000E9E50423702239462846FFF70AFB0B233D
:1046E00030604FF4006239462846FFF702FB00288D
:1046F0003FF428AE3368444643F008033360D2E504
:1047000039462846FFF7E6FA10F48044336809D0AA
:1047100000934FF4F062072339462846FFF700FB69
:104720000024C0E5C3F3C0030093394628460B2399
:104730004FF40062FFF7F4FA3368702200933946B1
:1047400004232846FFF7ECFAADE50F0147F06C07AC
:10475000FFB23946284624BBFFF7BCFA10F4804468
:1047600008D00423702239462846FFF7C2FA0024F5
:10477000306098E507234FF4F06239462846FFF78A
:10478000B8FA0B2330604FF4006239462846FFF731
:10479000B0FA00283FF4D6AD336843F00803336025
:1047A00081E5FFF797FA336810F48044009307D04F
:1047B0000423702239462846FFF7B2FA002472E536
:1047C00007234FF4F06239462846FFF7A9FA6AE555
:1047D0001B680F22009328460023FFF7A1FA00244C
:1047E00061E5090141F06D01C9B238B90F234FF4F9
:1047F00000422846FFF77DFA306054E51B684FF40D
:104800000042009328460F23FFF78AFA00244AE566
:1048100041F06D01C9B238B90D234FF4C0422846AA
:10482000FFF767FA30603EE51B684FF4C042009323
:1048300028460D23FFF774FA002434E541F06D019A
:10484000C9B238B908234FF470622846FFF751FA0D
:10485000306028E51B684FF47062009328460823F7
:10486000FFF75EFA00241EE51B68602200932846CD
:104870000523FFF755FA002415E5090141F06D0104
:10488000C9B248B903460F222846FFF732FA306012
:1048900009E500BF9C2E00201B680F2200932846CC
:1048A0000023FFF73DFA0024FDE4090141F06D010A
:1048B000C9B238B918234FF080722846FFF719FAA9
:1048C0003060F0E41B684FF0807200932846182394
:1048D000FFF726FA0024E6E41B684FF4FE0200937B
:1048E00028461023FFF71CFA0024DCE4090141F0FC
:1048F0006C01C9B238B911234FF400322846FFF7D2
:10490000F8F93060CFE41B684FF40032009328467A
:104910001123FFF705FA0024C5E4002840F0CD80FC
:10492000090141F06F0110234FF4F812C9B2284673
:10493000FFF7DFF93060B6E447F011011A68C9B239
:104940002846FFF7E3F933684FF48062003318BF5D
:1049500001234146009328460A23FFF7E1F900248A
:10496000A1E42021A94041F01101C9B220B9284693
:10497000FFF7B0F9306096E41A682846FFF7C6F9E9
:10498000002490E4090141F06C01C9B238B90D234B
:104990004FF400522846FFF7ACF9306083E41B68FF
:1049A0004FF40052009328460D23FFF7B9F9002475
:1049B00079E41B684FF47002009328461423FFF734
:1049C000AFF900246FE400287AD1090141F06F01AA
:1049D000034640F2FF32C9B22846FFF78AF9306039
:1049E00061E41A682846FFF791F900245BE420216E
:1049F000A94041F01A01C9B220B92846FFF76AF967
:104A0000306050E41A682846FFF780F900244AE431
:104A1000D8B971B101297FF446AC01462846FFF7A9
:104A200059F900F06000A0F120035842584130606D
:104A300039E40846FFF74EF900F01800A0F1100223
:104A40005042504130602C462DE419B1012913D059
:104A5000002428E40846FFF73DF9336820F01802E7
:104A60003BB142F0100200210846FFF74FF9002445
:104A700019E442F00802F6E700212846FFF72AF978
:104A8000336820F060023BB142F020020021012097
:104A9000FFF73CF9002406E442F04002F6E7042464
:104AA00001E40424FFF7FFBB0424FFF7FCBB04244C
:104AB000FFF7F9BB0424FFF7F6BB0424FFF7F3BBB1
:104AC0000424FFF7F0BB07B50129019207D802467D
:104AD00001AB0120FFF74DFA03B05DF804FB08209D
:104AE000FAE7012938B505460C460FD1084B1022CC
:104AF00000210BF049FE2846054B214618220BF0F9
:104B000043FEBDE8384003480BF0B6BE38BD00BFD9
:104B1000C80405009C2E00200129134603D8024634
:104B20000020FFF726BA08207047012810B40C4671
:104B300007D8054B2046D3F8CC3211469B6810BCF1
:104B40001847002010BC70479C2E00202DE9F04132
:104B50000127604C604D6169604B8CB0C5F8C8128C
:104B60005F4ACDE9007328460023DFF8DC810BF0B3
:104B70005BFE5C4928460BF0B0FED8F80C60736809
:104B800003F5AA72C5F8A82203F5B872C5F8AC22DD
:104B900003F56F72C5F8B02203F5767203F1C80011
:104BA000C5F8B42203F57D7203F58263C5F8BC3203
:104BB0003368C5F8B822DB68C5F8A40298473368A3
:104BC000D5F8B002DB6898473368D5F8B0029B6926
:104BD00098473368D5F8A8021B6998473368D5F819
:104BE000AC021B6998473368D5F8BC021B6998472B
:104BF0003368D5F8B4021B6998473368D5F8B80212
:104C00001B6998476FF080617368D8F8102003F52E
:104C100037735360344BC5F8CC22029303F19F23C2
:104C200003F56A0356330393304A314B3148CDE9DB
:104C30000423314B02AACDE90613A3F1D943A3F50E
:104C40009113A3F2272308932C4B0021CDE90903EC
:104C50004FF477432846ADF82C300BF094FF02AAAE
:104C6000394628460BF08FFF6369254A1F70C3F849
:104C70000422244A3225C3F8082200225A70224B0B
:104C800038462362214BE361214BA361214B6362D0
:104C9000214BA363214B6363214BA362214BE3624E
:104CA000214BA364214B6364214B6365214B236536
:104CB000214BE364214B2366214BE36502232374DC
:104CC000DE23C4E902351F4BA365FFF791F80CB052
:104CD000BDE8F081006100209C2E00200024F4003B
:104CE000687E0208E34A010854B5AAAA2929492482
:104CF00022421010224240007D77BBB580FFFF5654
:104D0000693D01085D3D01080B3F0108713F010845
:104D10006D3F0108693F0108194B0108C74A0108A6
:104D2000953E0108E93E01081D3D0108E53C0108EA
:104D3000C93C0108913D0108A13C0108F13D010871
:104D4000BD3C0108353E01087086020801289FBF5E
:104D5000044B03EB8000C368002094BF0B60082065
:104D6000704700BF783100200022014B5A60704725
:104D70000061002038B50546054C014620460CF080
:104D800099F829462046BDE838400CF093B800BF9A
:104D90007831002010B5034814460CF01EF820604E
:104DA00010BD00BF7831002001480CF008B800BFEA
:104DB0007831002010B5044605480B4600EB84020C
:104DC000D2F8982221460CF064F9002010BD00BFF3
:104DD0007831002010B5044605480A4600EB8403EC
:104DE000D3F8983221460CF036F9002010BD00BFF0
:104DF0007831002008B5014602480CF029F900205E
:104E000008BD00BF7831002008B50A4601460248B7
:104E10000CF01BF9002008BD7831002008B50A46C7
:104E2000014602480CF00FF9002008BD783100203F
:104E300008B50A46014602480CF0E7F8002008BD14
:104E40007831002001480CF0C7B800BF783100204D
:104E500008B5222107480BF0C0FF48B94221054898
:104E60000BF0BBFF20B9BDE8084002480CF09CB82D
:104E7000002008BD78310020012810B5144612D05A
:104E800003D302281CD004200AE0114B114ADB682E
:104E900024681B68D2F8AC021CB15B6998470020FB
:104EA00010BD9B69FAE70A4B0A4ADB68D2F8A402F4
:104EB0001B685B6A9847003018BF01202060EEE74E
:104EC000034B044ADB68D2F8A8021B685B6AF1E76F
:104ED0007086020878310020022804BF0C4B93F83A
:104EE000E80038B90B4BDB681B685B690A4AD2F8EB
:104EF000A0021847012809D1054B93F8E830012B8F
:104F000004D1044BDB681B689B69EFE7704700BF67
:104F100000610020708602087831002070B5002002
:104F2000FFF7DAFF134B144CDD68D4F8A0022B68AE
:104F30009B6898472B68D4F8A4029B6898472B6815
:104F4000D4F8A8029B6898472B68D4F8B8029B68ED
:104F500098472B68D4F8B0029B6898472B68D4F820
:104F6000B4029B6898472B68D4F8AC029B68BDE8F4
:104F70007040184770860208783100201C2A2DE9FD
:104F8000F04106460C461F4600F0278300F2A98038
:104F90000C2A00F033824DD8052A00F0D4811BD8AA
:104FA000022A00F08C8107D8002A00F06481012ACF
:104FB00000F07481042668E1032A00F09781042A36
:104FC000F8D1DFF824838D004544002840F0A1810A
:104FD000D5F898323B6058E1082A00F0F18115D8E5
:104FE000062A00F0C181072AE4D1202101FA04F445
:104FF00044F01004E4B22146BB48002E40F0D281B8
:105000000BF0EBFE00F01F0038603EE10A2A00F0D2
:10501000E6810B2ACED1002840F0F0852021A14066
:1050200041F01501C9B2B0480BF0D7FE00F0010005
:1050300038602AE1122A00F06D8227D80F2A00F08A
:10504000418211D80D2A00F008820E2AB2D1202107
:10505000A14041F01401C9B2002840F02D82A248BD
:105060000BF0BBFE386010E1102A00F03C82112AE0
:10507000A0D12021A14041F00801C9B2002840F090
:10508000438299480BF0A9FE3860FEE0152A00F033
:10509000698211D8132A00F04E82142A8AD1202165
:1050A000A14041F00B01C9B2002840F055828E4862
:1050B0000BF093FE3860E8E0172A00F07782C0F02A
:1050C0006282182A7FF476AF2021A14041F01301BB
:1050D000C9B2002840F07B8283480BF07EFE386026
:1050E000D3E0AB2A00F00D8463D8A52A00F0268314
:1050F00031D8A22A00F0DB8218D81D2A00F089825C
:105100008C2A7FF457AF002840F08C82090141F0CF
:105110006C0101F0FC0174480BF05FFE4FF48073EA
:1051200000F00F0043FA00F03860AEE0A32A00F070
:10513000DA82A42A7FF43EAF0C0144F06C04E4B29E
:1051400021466948002E40F0EA820BF046FEC0F38B
:105150000030386099E0A82A00F08B8314D8A62A82
:1051600000F03583A72A7FF425AF0C0144F06C04CE
:10517000E4B221465C48002E40F06D830BF02DFE1A
:1051800000F00F00386080E0A92A00F08F83AA2A7F
:105190007FF410AF0C0144F06D04E4B22146524894
:1051A000002E40F09F830BF018FEC0F30320386000
:1051B0006BE0B52A00F02A842CD8AE2A00F0E783F1
:1051C00014D8AC2A00F0B983AD2A7FF4F3AE0C01F9
:1051D00044F06D04E4B221464348002E40F0C883F9
:1051E0000BF0FBFDC0F3006038604EE0B32A00F026
:1051F000F183B42A7FF4DEAE002840F00585090172
:1052000041F06F01C9B238480BF0E7FDC0F304402C
:1052100038603AE0CE2A00F0508414D8B62A00F064
:105220002984B82A7FF4C6AE0C0144F06C04E4B2C1
:1052300021462D48002E40F030840BF0CEFDC0F307
:105240004030386021E0D22A00F05084D32A00F0A8
:105250006084D12A7FF4AEAE202101FA04F444F038
:105260001904E4B221462048002E40F035840BF0AA
:10527000B4FD386009E02021A14041F00D01C9B220
:1052800030B919480BF0A9FD38603046BDE8F0810F
:105290001A6815480BF093FD0026F6E72021A1407F
:1052A00041F00101C9B220B90F480BF096FD3860FA
:1052B000EBE71A680C480BF082FD0026E5E7202199
:1052C000A14041F00701C9B220B907480BF085FDA4
:1052D0003860DAE71A680448002AB8BF52420BF077
:1052E0006EFD0026D1E700BF78310020002840F095
:1052F0007C842021A14041F00201C9B2AA480BF0F0
:105300006CFD10F4000318BF4FF07F431843386062
:10531000BBE720261B688E40002BB8BF5B42F1B272
:105320004046C5F898320BF058FD044608B10026F7
:10533000ABE746F00701D5F89822C9B240460BF01A
:105340003EFD2646A1E72021A14041F00601C9B259
:1053500020B995480BF041FD386096E71A689248ED
:105360000BF02DFD002690E7202101FA04F444F013
:105370001004E4B221468C482EB90BF02EFDC0F388
:105380000420386081E70BF028FD3B6820F4F852D8
:105390001B0203F4F8531A43214683480BF00FFD18
:1053A000002672E70BF019FD3B6820F01F0203F0A6
:1053B0001F031A4321467C480BF001FD002664E7D9
:1053C000002840F015842021A14041F01501C9B208
:1053D00075480BF002FDC0F34020386055E7002807
:1053E00040F009842021A14041F01501C9B26E4866
:1053F0000BF0F3FCC0F34000386046E7202101FACF
:1054000004F444F01404E4B2214667482EB90BF0CA
:10541000E4FCC0F34000386037E70BF0DEFC3B688B
:1054200020F00202002BD4BF0023022321461A439E
:105430005D480BF0C4FC21465B480BF0CEFC3B689A
:1054400020F00802022B14BF0023082321461A4330
:1054500055480BF0B4FC002617E7202101FA04F4AC
:1054600044F01404E4B221464F482EB90BF0B5FCC9
:1054700000F00100386008E70BF0AFFC3A6820F05C
:105480000100002AD4BF024640F0010221464648EE
:105490000BF095FC214644480BF09FFC3B6820F044
:1054A0000402022B14BF0023042321461A433E4862
:1054B0000BF085FC0026E8E61A683B480BF07FFC01
:1054C0000026E2E62021A14041F00401C9B220B942
:1054D00035480BF082FC3860D7E61A6832480BF08A
:1054E0006EFC0026D1E62021A14041F00501C9B2A1
:1054F00020B92D480BF071FC3860C6E61A682A48BE
:105500000BF05DFC0026C0E61A6827480BF057FC3C
:105510000026BAE62021A14041F00A01C9B220B913
:1055200021480BF05AFC3860AFE61A681E480BF0B1
:1055300046FC0026A9E62021A14041F00301C9B2A2
:1055400020B919480BF049FC38609EE61A681648E5
:105550000BF035FC002698E61A6813480BF02FFC78
:10556000002692E62021A14041F00C01C9B220B9E9
:105570000D480BF032FC386087E61A680A480BF0D9
:105580001EFC002681E62021A14041F01101C9B294
:1055900020B905480BF021FC386076E61A6802480D
:1055A0000BF00DFC002670E6783100202021A14090
:1055B00041F01201C9B220B9B4480BF00EFC3860BA
:1055C00063E61A68B1480BF0FAFB00265DE61A683C
:1055D000AE480BF0F4FB002657E60C0144F06C04D7
:1055E000E4B22146A9482EB90BF0F7FBC0F3804086
:1055F00038604AE60BF0F1FB3B6820F480229B0404
:1056000003F480231A432146A0480BF0D8FB002660
:105610003BE6002840F0F5829C4901EB8404E368F6
:105620003B6032E61B68102B3BD00DDC022B34D0E4
:1056300004DC012B16D04FF0FF3314E0042B2ED0E6
:10564000082BF8D105230EE0402B2CD003DC202BB7
:10565000F1D1032307E0802B27D0B3F5807FEAD177
:10566000002300E008233B603B6801333FF45FAE5A
:10567000240144F06C04E4B2214684480BF0ADFBF5
:105680003B6820F070621B0603F070631A432146EA
:105690007E480BF094FB0026F7E50723E3E706239B
:1056A000E1E70423DFE70223DDE70123DBE70C0169
:1056B00044F06C04E4B2214674482EB90BF08DFB23
:1056C000C0F3C1303860E0E50BF087FB3B6820F4A5
:1056D000C032DB0303F4C0331A4321466B480BF09E
:1056E0006EFB0026D1E50C0144F06C04E4B22146C7
:1056F00066482EB90BF071FBC0F340303860C4E54A
:105700000BF06BFB3B6820F400525B0303F4005387
:105710001A4321465D480BF052FB0026B5E50BF01D
:105720005CFB3B6820F480521B0303F480531A4354
:10573000214656480BF043FB0026A6E50D0145F037
:105740006C05EDB2294651480BF047FB2946C0F3E2
:1057500080344E486EB92CB10BF03FFBC0F3C31040
:10576000386092E50BF039FBC0F302103860264632
:105770008BE574B10BF031FB3B6820F4F062DB0188
:1057800003F4F0631A43294640480BF018FB002647
:105790007BE50BF022FB3A6820F40060120202F471
:1057A00000620243294639480BF009FB2946374875
:1057B0000BF013FB3B6820F070021B0103F0700339
:1057C0001A43294631480BF0FAFA26465DE50D01E9
:1057D00045F06C05EDB229462C480BF0FEFA29463F
:1057E000C0F380342948BEB92CB10BF0F6FAC0F3EF
:1057F0000210386049E50BF0F0FAC0F3C3103860CE
:10580000294622480BF0E9FA3B68000A00F008003C
:1058100003433B60264638E574B10BF0DEFA3B6883
:1058200020F070021B0103F070031A432946174849
:105830000BF0C5FA002628E50BF0CFFA3B6820F400
:10584000F062DB0103F4F0631A4329460F480BF0C2
:10585000B6FA264619E50BF0C0FA3B6820F00F02B5
:1058600003F00F031A43214608480BF0A8FA00265C
:105870000BE50C0144F06D04E4B2214603483EB947
:105880000BF0ABFAC0F3C0303860FEE47831002092
:105890000BF0A3FA3B6820F40042DB039BB21A43EF
:1058A0002146AE480BF08BFA0026EEE40C0144F0E2
:1058B0006D04E4B22146A9482EB90BF08EFAC0F36C
:1058C00041303860E1E40BF088FA3B6820F4C042D4
:1058D0005B0303F4C0431A432146A0480BF06FFA60
:1058E0000026D2E40BF079FA3B6820F470621B02C8
:1058F00003F470631A43214698480BF060FA0026BF
:10590000C3E40C0144F06D04E4B2214693482EB97F
:105910000BF063FAC0F341103860B6E40BF05DFAA7
:105920003B6820F060025B0103F060031A432146EC
:105930008A480BF044FA0026A7E40C0144F06D04F9
:10594000E4B2214685482EB90BF047FA00F00F006B
:1059500038609AE40BF041FA3B6820F00F0203F044
:105960000F031A4321467D480BF029FA00268CE4E8
:105970000BF033FA3B6820F080721B0603F0807353
:105980001A43214675480BF01AFA00267DE40C01F3
:1059900044F06D04E4B22146704866B90BF01DFA7C
:1059A000001400F07F0310F0400018BF6FF07F007C
:1059B0001843386069E40BF010FA3B6820F4FE02EB
:1059C0001B0403F4FE031A43214664480BF0F7F965
:1059D00000265AE40C0144F06C04E4B221465F480E
:1059E0002EB90BF0FAF9C0F3404038604DE40BF0EB
:1059F000F4F93B6820F400325B0403F400331A43EB
:105A0000214656480BF0DBF900263EE4202505FA36
:105A100001F14DB245F01404E4B288B921464F4873
:105A20000BF0DBF910F4806007D045F01101C9B22A
:105A30004A480BF0D2F9386027E43860064624E47F
:105A400045F011011A68C9B244480BF0B8F9214673
:105A500042480BF0C2F93B6820F48062002B0CBF77
:105A600000234FF4806321461A433C480BF0A7F90A
:105A700000260AE42021A14041F01101C9B228B951
:105A800036480BF0AAF93860FFF7FFBB1A683348B5
:105A90000BF095F90026FFF7F8BB0BF09EF93B6879
:105AA00020F400525B0303F400531A4321462B48B1
:105AB0000BF085F90026FFF7E8BB002840F0A7802F
:105AC000090141F06F01C9B224480BF086F9C0F317
:105AD00009003860FFF7D9BB0BF07FF93A6821461F
:105AE0001E480BF06CF90026FFF7CFBB2021A14028
:105AF00041F01A01C9B228B918480BF06EF93860A4
:105B0000FFF7C3BB1A6815480BF059F90026FFF7D9
:105B1000BCBBE8B979B101297FF4B7AB01460F48A6
:105B20000BF05BF900F06000A0F1200358425841EF
:105B30003860FFF7AABB09480BF04FF900F01800D6
:105B4000A0F110025042504138602646FFF79DBB3D
:105B500031B1012926D00026FFF797BB783100200C
:105B60002C480BF03AF93B6820F00802002B14BFD8
:105B70000023082321461A4326480BF020F921462A
:105B800024480BF02AF93B6820F01002002B0CBFD0
:105B90000023102321461A431E480BF010F9264615
:105BA000FFF773BB00211B480BF017F93B6820F08F
:105BB0002002002B0CBF0023202300211A4315488C
:105BC0000BF0FDF8002113480BF007F93B6820F0BB
:105BD0004002002B14BF0023402300211A430D482C
:105BE0000BF0EDF80026FFF750BB0426FFF74DBB86
:105BF0000426FFF74ABB0426FFF747BB0426FFF73E
:105C000044BB0426FFF741BB0426FFF73EBB042636
:105C1000FFF73BBB7831002007B50129019207D877
:105C2000024601AB0120FFF7A9F903B05DF804FBC0
:105C30000820FAE7012910B504460DD1074A1021C2
:105C40000BF0BDF82046054A18210BF0B8F8BDE866
:105C5000104003480BF008B910BD00BFC804050090
:105C6000783100200129134603D802460020FFF7AF
:105C700085B908207047034B0846D3F8BC3211465B
:105C8000DB68184778310020F8B54B4C4B4D626902
:105C90004B4B28464B4F00210BF0C7F84A4928468A
:105CA0000BF0AFF9FE68736803F5AA72C5F8A42279
:105CB00003F5B872C5F8A82203F56F72C5F8AC22D7
:105CC00003F5767203F1C800C5F8B02203F57D72C2
:105CD00003F58263C5F8B8323368C5F8B422DB68CF
:105CE000C5F8A00298473368D5F8AC02DB6898473E
:105CF0003368D5F8AC029B6998473368D5F8A4029D
:105D00001B6998473368D5F8A8021B699847336820
:105D1000D5F8B8021B6998473368D5F8B0021B69FB
:105D200098473368D5F8B4021B69984773683A6995
:105D300003F537735360C5F8BC226369234A022018
:105D4000C3F80422224AC3F8082201221A70002252
:105D50005A70204B322223621F4B2074E3611F4B89
:105D6000A3611F4B63621F4BA3631F4B63631F4BF6
:105D7000A3621F4BE3621F4BA3641F4B63641F4B63
:105D800063651F4B23651F4BE3641F4B23661F4B4B
:105D9000E3654FF48C73C4E902321D4BA3652B6895
:105DA000D3F8A020D3F82031C5F89822C5F89C324A
:105DB000BDE8F840FFF790B800610020783100207E
:105DC0006880020870860208355C0108514E01089F
:105DD000454E0108314E01081D4E0108094E0108CB
:105DE000F54D0108655C0108195C0108D54D0108F5
:105DF000B54D0108A94D0108954D0108754D0108E3
:105E0000794E01084D4D0108D94E0108694D010830
:105E10001D4F010818B9034B5B680B6070470820E1
:105E2000704700BF443400200022014B5A60704785
:105E3000006100200428F8B514467FD008D8012856
:105E40004BD020D3022867D0032834D0042433E079
:105E5000062800F0A080C0F09280072800F0A38000
:105E6000FC28F3D1584B594DDE6814683368D5F8D7
:105E7000A002002C00F0A380DB6898473368D5F8B7
:105E8000A0029B6916E0126832F0030340F099808B
:105E90004D4B4E4DDE68D207D5F8940233680DD5D0
:105EA0001B6998472468326814F00204D5F8900200
:105EB0000BD01369984700242046F8BDDB6898474B
:105EC0003368D5F894029B69EBE7D3689847336849
:105ED000D5F890029B699847EEE744F62063126874
:105EE0009A426EDC42F21071384B8A42D3F8B40207
:105EF000354BDB681B68CCBF5B699B69984742F2F6
:105F000011732268002092FBF3F103FB1121304B47
:105F100089B29B689847CEE72B4B1468DD68D5E9BA
:105F2000003000F506703CB1DB689847D5E90030D9
:105F30009B6900F50670BDE79B68CCE7224B234EBA
:105F4000DF6815683B68D6F8A0024DB1012D11D06D
:105F50001B6998473B68D6F8A0025B6A984707E040
:105F6000DB6898473B689B69D6F8A00298472846AB
:105F70002060A0E7DB6898473B685B69F4E7124B59
:105F8000124ADB68D2F8AC021B685B6A98470030A3
:105F900018BF0120ECE70C4B0C4ADB68D2F8B002CA
:105FA0001B685B6AF2E7094B1268D3F8A802064B3C
:105FB000012ADB681B680CBF5B699B697AE71B6978
:105FC00089E7102478E700BF708602084434002077
:105FD00078090020224B70B5DD68224C2B68D4F87C
:105FE00098029B6998472B68D4F8B8029B68984739
:105FF0002B68D4F8B4029B6898472B68D4F89C02AD
:106000009B6898472B68D4F8A0029B6898472B6838
:10601000D4F8A4029B6898472B68D4F890029B6838
:1060200098472B68D4F894029B6898472B68D4F85B
:10603000AC029B6898472B68D4F8B0029B689847DD
:106040002B68D4F8A8029B6898472B68D4F898026C
:106050009B689847BDE87040034B5B68184700BFDA
:1060600070860208443400207809002001480BF0B3
:106070005AB800BF44340020014601480BF0FDB877
:106080004434002010B5034814460BF05AF8206041
:1060900010BD00BF4434002008B50348D0F8BC222E
:1060A0000BF07AF9002008BD4434002008B50348FD
:1060B000D0F8BC220BF05CF9002008BD443400206D
:1060C00008B502480BF051F9002008BD4434002007
:1060D00008B502480BF046F9002008BD4434002002
:1060E00008B502480BF03CF9002008BD44340020FC
:1060F00008B502480BF020F9002008BD4434002008
:1061000001480BF0A1B800BF4434002038B522216B
:106110000D480BF016F80C4C10B920460BF07CF82B
:106120000A4BD4F8B402DD682B689B6998472B684A
:10613000D4F890021B6998472B68D4F894021B6925
:106140009847012038BD00BF443400207086020803
:10615000022804BF0C4B93F8E80038B90B4BDB68FE
:106160001B685B690A4AD2F898021847012809D1CE
:10617000054B93F8E830012B04D1044BDB681B6816
:106180009B69EFE7704700BF00610020708602083E
:1061900044340020012908B508D1054A70210AF0CD
:1061A000C2FFBDE8084003480BF010B808BD00BFAF
:1061B000C8040500443400208C2970B504461546F7
:1061C00000F01A8300F298800E2900F02F8241D847
:1061D000062900F0B38119D8022900F06C8107D894
:1061E000002900F04B81012900F0578104244BE184
:1061F000042900F07D8140F26C81002840F09781F5
:106200002621BE480AF09DFF28603DE10A2900F0E2
:10621000C4810FD8072900F0A9810829E6D10028F8
:1062200040F00C863521B5480AF08BFFC0F34020C2
:10623000286029E10C2900F0CA8140F2BC81342198
:10624000AE48002C40F0DF810AF07BFF00F0010037
:10625000286019E1152900F03D821FD8112900F0AE
:1062600008820DD80F2900F0EF811029BED1002837
:1062700040F0F8812521A1480AF063FF286003E17E
:10628000132900F0128240F20282002840F01B82A3
:106290002B219A480AF055FF2860F5E01C2900F0F0
:1062A0005F821AD8182900F035821B2900F040823D
:1062B00017299BD1924E002840F01A8215218F4851
:1062C0000AF03FFF30B14FF08073B3FBF0F086422D
:1062D00028BF06462E600024D6E0212900F058820F
:1062E000222900F06F821D2980D1002840F0AF855F
:1062F000824B5B681360C7E0B32900F0308457D845
:10630000A82900F0958324D8A42900F0EB8210D8A6
:10631000A22900F0C082A3297FF468AF6C217748DE
:10632000002C40F0D0820AF00CFFC0F380302860CF
:10633000AAE0A62900F02C8340F2EC826C216F4881
:10634000002C40F067830AF0FCFE00F00F0028608C
:106350009AE0AB2900F0AD8310D8A92900F07F8323
:10636000AA297FF443AF6D216448002C40F092834A
:106370000AF0E7FEC0F30320286085E0AD2900F0B5
:10638000C783C0F0AE83AE297FF430AF6D215B4888
:10639000002C40F0D5830AF0D4FE001400F07F03F7
:1063A00010F0400018BF6FF07F00184328606BE0CA
:1063B000BB2900F0898436D8B62900F017841FD88D
:1063C000B42900F0E483B5297FF410AF34214B48A1
:1063D000002C40F0E9830AF0B4FE430540F1E2836B
:1063E000142146480AF0ADFE454B30B14FF08072A3
:1063F000B2FBF0F0834228BF03462B60002443E049
:10640000B92900F0248400F23A84B8297FF4EEAE72
:106410006C213A48002C40F00B840AF092FEC0F345
:106420004030286030E0CC2900F0C88412D8BF2961
:1064300000F08084C02900F09D84BC297FF4D6AE92
:1064400070212E48002C40F068840AF07AFEC0B219
:10645000286019E0D12900F0CB84D22900F0D8843B
:10646000CE297FF4C3AE002840F0F7846F21234883
:106470000AF067FEC0F30900286005E030B92D215D
:106480001E480AF05EFE2860204670BD12682D216D
:106490001A480AF048FE0024F6E728B921211748D7
:1064A0000AF04FFE2860EFE71268212113480AF036
:1064B0003AFE0024E8E728B9272110480AF041FEF7
:1064C0002860E1E7126827210C480AF02CFE00241E
:1064D000DAE7002840F0AC84222108480AF031FEB7
:1064E00010F4000318BF4FF07F4318432860CBE738
:1064F000024E38B9D6F8BC321360C5E744340020E8
:10650000FFFF0F0013682021002BB8BF5B42AC488F
:10651000C6F8BC320AF015FE0446002840F08B8411
:10652000D6F8BC222721A6480AF0FDFDACE7126888
:106530002621A3480AF0F7FD0024A5E71021A04872
:106540002CB90AF0FEFDC0F3042028609CE70AF095
:10655000F8FD2B6820F4F8521B0203F4F8531A4399
:10656000102197480AF0DFFD00248DE710219448A0
:106570002CB90AF0E6FD00F01F00286084E70AF05D
:10658000E0FD2B6820F01F0203F01F031A431021C7
:106590008B480AF0C8FD002476E7002840F05184BB
:1065A000352187480AF0CDFD10F0020F0CBF012302
:1065B00000232B6068E7002840F04684352180489E
:1065C0000AF0BFFDC04300F0010028605CE7342101
:1065D0007B482CB90AF0B5FDC0F34000286053E7B2
:1065E0000AF0AFFD2C6834B940F00202342174483F
:1065F0000AF099FD48E720F00202342170480AF0C1
:1066000092FD002440E70AF09CFD2C6834B940F06C
:10661000010234216A480AF086FD35E720F00102C4
:10662000342167480AF07FFD00242DE728B9342182
:1066300063480AF086FD286026E712683421604826
:106640000AF071FD00241FE728B924215C480AF0F4
:1066500078FD286018E71268242159480AF063FD84
:10666000002411E71268252155480AF05CFD00243A
:106670000AE728B9282152480AF063FD286003E799
:10668000126828214E480AF04EFD0024FCE628B985
:106690002A214B480AF055FD2860F5E612682A21A8
:1066A00047480AF040FD0024EEE628B9232144487B
:1066B0000AF047FD2860E7E61268232140480AF007
:1066C00032FD0024E0E612682B213D480AF02BFD44
:1066D0000024D9E628B92C2139480AF032FD286077
:1066E000D2E612682C2136480AF01DFD0024CBE6C4
:1066F00013686BB14FF0807292FBF3F2B242A8BF05
:1067000032462A6015212E480AF00DFD0024BBE612
:106710003246F6E728B9332129480AF012FD2860ED
:10672000B2E61268332126480AF0FDFC0024ABE6ED
:106730006C2123482CB90AF004FDC0F3C040286046
:10674000A2E60AF0FEFC2B6820F40022DB0403F42E
:1067500000231A436C211A480AF0E5FC002493E652
:106760006C2117482CB90AF0ECFCC0F3804028607B
:106770008AE60AF0E6FC2B6820F480229B0403F4EE
:1067800080231A436C210E480AF0CDFC00247BE6DE
:1067900000210B482CB90AF0D4FC00F0010028605D
:1067A00072E60AF0CEFC2B6820F0010203F0010330
:1067B0001A43002102480AF0B6FC002464E600BF38
:1067C0004434002038B90146B1480AF0BAFCC0F39D
:1067D0004000286058E60021AD480AF0B2FC2B6862
:1067E00020F002025B0003F002031A430021A848D4
:1067F0000AF099FC002447E658B96C21A4480AF035
:10680000A0FC4FF48073C0F3036043FA00F02860EB
:106810003AE61368102B27D00DDC022B20D004DCC5
:10682000012B16D04FF0FF3314E0042B1AD0082BA5
:10683000F8D105230EE0402B18D003DC202BF1D13A
:10684000032307E0802B13D0B3F5807FEAD1002328
:1068500000E008232B602B6801330BD1102413E6D2
:106860000723F7E70623F5E70423F3E70223F1E71D
:106870000123EFE76C2186480AF063FC2B6820F0C7
:1068800070621B0603F070631A436C2180480AF0A3
:106890004AFC0024F8E56C217D482CB90AF051FC33
:1068A000C0F3C1302860EFE50AF04BFC2B6820F400
:1068B000C032DB0303F4C0331A436C2174480AF07E
:1068C00032FC0024E0E50AF03CFC2B6820F4804216
:1068D0009B0303F480431A436C216D480AF023FCA8
:1068E0000024D1E56C216A482CB90AF02AFCC0F3D7
:1068F00000302860C8E50AF024FC2B6820F48052A0
:106900001B0303F480531A436C2161480AF00BFC0B
:106910000024B9E56C215E480AF013FC00F48043C2
:1069200094B93BB16C215A480AF00BFCC0F3C31078
:106930002860A9E5C0F3021300F4006003430CBF14
:10694000002308232B609FE583B16C2150480AF097
:10695000F8FB2B6820F4F062DB0103F4F0631A43C8
:106960006C214B480AF0DFFB00248DE52A680024E7
:1069700011074CBF40F4006020F40060120120F0C9
:106980007000D2B202436C2141480AF0CCFB7BE597
:106990006C213F480AF0D5FBACB910F4804307D016
:1069A0006C213B480AF0CDFBC0F3021028606BE578
:1069B000C0F3C31200F4006002430CBF002208229F
:1069C0001C462A6060E56C2131480AF0BAFB10F4DD
:1069D00080444FF06C012E480ED00AF0B2FB2B68B9
:1069E00020F070021B0103F070031A436C21284849
:1069F0000AF099FB002447E50AF0A3FB2B6820F47A
:106A0000F062DB0103F4F0631A436C2120480AF0C2
:106A10008AFB39E50AF095FB2B6820F00F0203F0A2
:106A20000F031A436C211A480AF07DFB00242BE562
:106A30006D2117482CB90AF084FBC0F3C0302860E0
:106A400022E50AF07EFB2B6820F40042DB039BB2B8
:106A50001A436D210E480AF066FB002414E56D21EF
:106A60000B482CB90AF06DFBC0F3413028600BE5F0
:106A70000AF067FB2B6820F4C0425B0303F4C043B9
:106A80001A436D2102480AF04EFB0024FCE400BFCB
:106A9000443400200AF055FB2B6820F470621B027E
:106AA00003F470631A436D21B7480AF03CFB0024DD
:106AB000EAE46D21B4482CB90AF043FBC0F341105D
:106AC0002860E1E40AF03DFB2B6820F060025B01E6
:106AD00003F060031A436D21AB480AF024FB002445
:106AE000D2E46D21A8482CB90AF02BFB00F00F006E
:106AF0002860C9E40AF025FB2B6820F00F0203F0A0
:106B00000F031A436D21A0480AF00DFB0024BBE4DB
:106B10006D219D482CB90AF014FBC0F30060286079
:106B2000B2E40AF00EFB2B6820F080721B0603F023
:106B300080731A436D2194480AF0F5FA0024A3E407
:106B40000AF0FFFA2B6820F4FE021B0403F4FE0394
:106B50001A436D218C480AF0E6FA002494E46C2173
:106B600089482CB90AF0EDFAC0F3404028608BE464
:106B70000AF0E7FA2B6820F400325B0403F40033D8
:106B80001A436C2180480AF0CEFA00247CE40028E5
:106B900040F060816F217C480AF0D3FAC0F30440D2
:106BA000286071E42C606FE40AF0CBFA2B6820F4C3
:106BB0008062002B0CBF00234FF4806334211A4302
:106BC00071480AF0B0FA2968704B69B14FF08072D1
:106BD00092FBF1F29A42A8BF1A462A6014216A4831
:106BE0000AF0A1FA00244FE41A46F6E7674E70B99E
:106BF000142165480AF0A5FA30B14FF08072B2FB5B
:106C0000F0F2964228BF16462E6000243CE413683A
:106C100063B14FF0807292FBF3F2B242A8BF3246EA
:106C2000142159480AF07FFA00242DE43246F7E790
:106C30000AF087FA2B6820F400525B0303F4005338
:106C40001A436C2150480AF06EFA00241CE46C21AF
:106C50004D482CB90AF075FAC0F30350286013E4CC
:106C60000AF06FFA2B6820F470021B0503F470031E
:106C70001A436C2144480AF056FA002404E4434EB7
:106C800078B9132140480AF05CFA30B14FF08073B4
:106C9000B3FBF0F0864228BF06462E600024FFF7C3
:106CA000F3BB136873B14FF0807292FBF3F2B24200
:106CB000A8BF32462A60132133480AF034FA002470
:106CC000FFF7E2BB3246F5E770212F4834B90AF0EE
:106CD00038FAC0F307202860FFF7D6BB0AF031FA74
:106CE0002A6820F47F40120292B2024370212648A3
:106CF0000AF019FA002124480AF023FA2B6820F040
:106D00000402002B0CBF0023042300211A431E4859
:106D10000AF009FA0024FFF7B7BB0AF012FA2A7842
:106D200020F0FF000243702117480AF0FCF900240C
:106D3000FFF7AABB40B9702113480AF002FAC0F36A
:106D400001402860FFF7A0BB1368032B3FF686AD18
:106D500070210D480AF0F5F92B6820F440321B042D
:106D600003F440331A43702107480AF0DCF9002489
:106D7000FFF78ABB60B9702103480AF0E2F9C0F35B
:106D800080402860FFF780BB44340020FFFF0F00E5
:106D90001368012B3FF662AD702131480AF0D1F93A
:106DA0002B6820F480229B0403F480231A43702173
:106DB0002B480AF0B8F90024FFF766BB7021284879
:106DC00034B90AF0BEF9C0F301502860FFF75CBB8C
:106DD0000AF0B7F92B6820F440121B0503F44013A6
:106DE0001A4370211E480AF09EF90024FFF74CBB9D
:106DF00030B939211A480AF0A4F92860FFF744BBDA
:106E00001268392116480AF08EF90024FFF73CBBBE
:106E100030B93A2112480AF094F92860FFF734BBE0
:106E200012683A210E480AF07EF90024FFF72CBBC5
:106E30000424FFF729BB0024FFF726BB0424FFF737
:106E400023BB0424FFF720BB0424FFF71DBB04244D
:106E5000FFF71ABB0424FFF717BB0424FFF714BB8A
:106E60004434002007B5019239B9014601AA012036
:106E7000FFF7A2F903B05DF804FB0820FAE70B4620
:106E800019B901461846FFF797B908207047034B18
:106E90000846D3F8C0321146DB6818474434002056
:106EA0002DE9F041654E664CF56801276B6803F1EA
:106EB000C802C4F8982203F58072C4F89C2203F536
:106EC0008E72C4F8A02203F5B872C4F8902203F5BC
:106ED000C672C4F8942203F5F072C4F8B42203F524
:106EE000FE72C4F8B82203F5617203F1E400C4F83D
:106EF000A82203F5687203F56F73C4F8AC322B68EF
:106F0000C4F8B0221B69C4F8A40298472B68D4F8CF
:106F1000A0021B6998472B68D4F89C021B6998470C
:106F20002B68D4F8AC021B6998472B68D4F8B002E0
:106F30001B6998472B68D4F8A802DB6898472B6830
:106F4000D4F890021B6998472B68D4F894021B6907
:106F500098472B68D4F89802DB6898472B68D4F8D8
:106F6000B402DB6898472B68D4F8B802DB6898470E
:106F70002B68D4F8A8029B699847326900266B6891
:106F8000C4F8C02203F5377353602E4B2E495A695B
:106F90003220C2F804122D491770C2F808122C4989
:106FA000567019622B491F74D9612B4999612B497D
:106FB00059622B4999632B4959632B4999622B4993
:106FC000D9622B4999642B4959642B4959652B493E
:106FD00019652B49D9642B4919662B49D9654FF49A
:106FE000F071C3E90210294920469965284B3146C2
:106FF0000AF0CFF8274920460AF03BF9236802201F
:10700000D3F8A030C4F8BC32FFF7A2F80222D4F8BB
:10701000B832197C5A7418683A460BF09BFD2B68FD
:10702000D4F8B8021C4C1B68984723689847A3689B
:1070300031463046BDE8F041184700BF708602086F
:1070400044340020006100200D6101080161010845
:10705000F1600108E1600108D1600108C160010828
:107060007F6E0108656E0108AD6001089960010836
:107070006D6001088560010879600108355E0108CE
:10708000155E010851610108295E0108D55F0108FC
:1070900068820208956101087809002018B9034B3D
:1070A0001B680B6070470820704700BF1437002032
:1070B0000022014B5A60704700610020234B70B5DD
:1070C000DD68234C2B68D4F898029B6998472B689D
:1070D000D4F8A8029B6998472B68D4F8AC029B6946
:1070E00098472B68D4F89C029B6898472B68D4F883
:1070F000A0029B6898472B68D4F8A4029B68984725
:107100002B68D4F890029B6898472B68D4F89402B7
:107110009B6898472B68D4F8B0029B6898472B6807
:10712000D4F8B4029B6898472B68D4F898029B68FF
:1071300098472B68D4F8A8029B6898472B68D4F826
:10714000AC029B68BDE87040184700BF708602081B
:1071500014370020034A0146D2F8B83200200AF062
:1071600062B900BF14370020024BD3F8B8020AF00E
:1071700094B900BF1437002038B5284D00F07F04C3
:107180002B1993F80C32DB0705D4D5F8B83203EB92
:107190008404606838BDD5F8BC3200219B68204665
:1071A00098470021D5F8BC3208469B6898470021D3
:1071B000D5F8BC3208469B6898470021D5F8BC3208
:1071C00008469B689847D5F8BC3201219B6800208F
:1071D0009847D5F8BC3200219B682046984700218B
:1071E000D5F8BC3208469B6898470021D5F8BC32D8
:1071F00004029B68084698470021D5F8BC32044336
:107200009B6808469847D5F8BC32240204439B6823
:1072100001210020984724022043BBE714370020B7
:10722000022804BF0C4B93F8E80038B90B4BDB681D
:107230001B685B690A4AD2F898021847012809D1ED
:10724000054B93F8E830012B04D1044BDB681B6835
:107250009B69EFE7704700BF00610020708602085D
:1072600014370020012870B506460F4D0F4C07D18A
:10727000EB6AC4F8C0325B68984784F8C46270BD9A
:1072800094F8C432012B03D1D4F8C0329B689847DC
:10729000EB682A695B68C4F8BC2203F53773536056
:1072A000002384F8C432EAE770860208143700200D
:1072B0000528F8B50C46154600F0A6801FD8022810
:1072C0006BD003D800283ED0042455E0032876D0A4
:1072D0000428F9D1614B624EDF6814683B68D6F828
:1072E000A002002C00F08180012C00F088801B6936
:1072F00098473B68D6F8A0025B6A98477DE008286B
:1073000000F08E8009D80628DED1544B544ADB6841
:10731000D2F8B4021B685B6A7DE0092800F089801E
:10732000FC28D1D14D4B4E4EDF6814683B68D6F82F
:10733000A002002C00F08D80DB6898473B68D6F8EF
:10734000A0029B6916E0126832F0030340F08380CC
:10735000424B434EDF68D207D6F894023B680DD506
:107360001B6998472C683B6814F00204D6F8900219
:107370000BD01B69984700242046F8BDDB6898476E
:107380003B68D6F894029B69EBE7DB6898473B685B
:10739000D6F890029B699847EEE7304B1468DE6898
:1073A000D6E9003000F506703CB1DB689847D6E9B5
:1073B00000309B6900F50670DCE79B68EBE7284B23
:1073C000D3F8A802254BDB681B6839B1146814F0A8
:1073D000010401D05B69CDE79B69DCE75B6A9847F4
:1073E000003018BF01202860C6E7DB6898473B687B
:1073F0009B69D6F8A002984720462860BBE7DB6867
:1074000098473B685B69F4E7144B154ADB68D2F890
:10741000B0021B685B6A9847003018BF0120ECE798
:1074200010680F4B00F0010083F8C502FFF71AFF48
:10743000A1E70A4B1268DC68012AD4E9003000F5A4
:10744000067004D1DB689847D4E90030B1E79B6847
:1074500090E71B699FE710248EE700BF7086020843
:10746000143700207FB52C4B00F07F041A1992F8D6
:107470000C221D4612F0010F06D1D3F8B83203EBEF
:107480008404606804B070BD05230122032101A8B3
:10749000ADF804308DF8064006F0FAF9D5F8C032A0
:1074A0008DF80700DB6998470421D5F8C0320DEB51
:1074B00001005B69984702F047FF0646D5F8C032E5
:1074C0001B6A984707281FD90821D5F8C0320DEB51
:1074D00001009B6998470122072102A89DF80F50DF
:1074E00006F0D6F9854214D19DF80830052B10D14D
:1074F0009DF80930FF2B0CD19DF80A30A34208D12A
:10750000DDF80B0000BABDE7304602F02DFF32284F
:10751000D4D94FF0FF30B5E714370020024B93F871
:10752000C53203B19EE727E61437002038B5222084
:10753000FFF7F4FF094C18B9D4F8B80209F0A4FF1A
:10754000074BD4F89002DD682B681B6998472B68BD
:10755000D4F894021B699847012038BD14370020E5
:107560007086020810B508461446FFF7D7FF206062
:1075700010BD2DE9F74F354D01F07F0995F8C56233
:1075800090469A469DF830409DF8347049F080004E
:10759000AB469EB305238DF802008DF8032007212A
:1075A00001226846ADF800308DF804A08DF8054042
:1075B0008DF8067006F06CF9D5F8C0328DF807002A
:1075C000DB6998470025DBF8C0321DF80500DB6851
:1075D00001359847082DF6D1022002F0BBFE47EA9C
:1075E0000424DBF8B83244EA0A4403EB890944EA8C
:1075F0000864C9F8044003B0BDE8F08FD5F8BC3288
:1076000031469B689847D5F8BC3231469B68404666
:107610009847D5F8BC3231469B6850469847D5F814
:10762000BC3231469B6820469847D5F8BC320121D0
:107630009B68384698474AEA082344EA0324D5F869
:10764000B83247EA042403EB8909D2E71437002053
:1076500007B5D3B20193C2F307230093C2F30743E4
:10766000120EFFF786FF03B05DF804FB0020FFF762
:10767000EFBF73B50D460646E8B9104C94F8C63214
:1076800043B1D4F8B8322721D3F8A020FFF7E0FFA8
:1076900084F8C66200242A462D210020FFF7D8FF77
:1076A0002046CDE90044234622462021FFF761FF12
:1076B000204602B070BD0820FBE700BF1437002051
:1076C00038B50C4605462120FFF728FF2368C1186E
:1076D00021602846BDE83840CBE737B50D46044663
:1076E000C8B901220D4B83F8C62281EAE172A2EBF0
:1076F000E1722721FFF7ACFF002DACBF012302236D
:107700002046CDE90043224623462021FFF731FFE2
:10771000204603B030BD0820FBE700BF143700202F
:107720000021DAE74942D8E7D7E7222970B50446B5
:10773000154600F0D88200F286800E2900F0038200
:107740003ED8062900F0958118D8022900F04B8117
:1077500007D8002900F02C81012900F0378104248A
:107760002BE1042900F0618140F25181002840F0B2
:1077700079812620FFF7D2FE28601EE10A2900F059
:10778000A5810ED8072900F08B810829E7D10028B0
:1077900040F0B1853520FFF7C1FEC0F340202860DE
:1077A0000BE10C2900F0AA8140F29D813420002CCD
:1077B00040F0BB81FFF7B2FE00F001002860FCE062
:1077C000152900F00F821DD8112900F0DD810CD899
:1077D0000F2900F0C5811029C1D1002840F0CD81CA
:1077E0002520FFF79BFE2860E7E0132900F0E681E3
:1077F00040F2D781002840F0EE812B20FFF78EFE6B
:107800002860DAE01B2900F02A820CD8172900F042
:10781000FB811829A3D1002840F01A823320FFF7FA
:107820007DFE2860C9E01D2900F04782C0F02E824D
:10783000212994D1002840F04782FFF76FFE00F025
:1078400001002860B9E0AE2900F0F7834FD8A729DE
:1078500000F0658328D8A32900F0B8820FD88C29BE
:1078600000F05882A2297FF47AAF6C20002C40F0FF
:107870009E82FFF753FEC0F3C13028609DE0A5292A
:1078800000F0D28240F2B9826C20FFF747FE00F48C
:107890008046002C40F01F83002E00F01183000969
:1078A00000F07000286088E0AA2900F073830FD8E8
:1078B000A82900F04A83A9297FF451AF6D20002C3C
:1078C00040F05983FFF72AFEC0F34130286074E08E
:1078D000AC2900F08D8340F274836D20002C40F0C1
:1078E0009D83FFF71BFEC0F30060286065E0BB29A5
:1078F00000F0598433D8B62900F0EB831DD8B429A1
:1079000000F0B983B5297FF42AAF3420002C40F071
:10791000BE83FFF703FE430540F1B7831420FFF752
:10792000FDFDB74B30B14FF08072B2FBF0F08342F7
:1079300028BF03462B6000243FE0B92900F0FA83FA
:1079400000F20F84B8297FF40AAF6C20002C40F0BD
:10795000E283FFF7E3FDC0F3403028602DE0CC293F
:1079600000F08F8411D8BF2900F04F84C02900F0A7
:107970006A84BC297FF4F3AE7020002C40F0388478
:10798000FFF7CCFDC0B2286017E0D12900F0928447
:10799000D22900F09E84CE297FF4E1AE002840F089
:1079A000B9846F20FFF7BAFDC0F30900286004E036
:1079B00028B92D20FFF7B2FD2860204670BD12685F
:1079C0002D210020FFF744FE0024F6E720B92120F6
:1079D000FFF7A4FD2860F0E7126821210020FFF7DF
:1079E00037FE0024E9E720B92720FFF797FD28603C
:1079F000E3E712682721002AB8BF52420020FFF7B0
:107A000027FE01227F4B002483F8C622D5E70028F9
:107A100040F06E842220FFF781FD10F4000318BFB0
:107A20004FF07F4318432860C7E7764BD3F8B8225E
:107A300018B9D2F8A0302B60BFE72B682020002BAC
:107A4000B8BF5B42C2F8A030FFF768FD044608B13A
:107A50000024B2E72A682721002AB8BF5242FFF764
:107A6000F7FDAAE7126826210020FFF7F1FD0024A8
:107A7000A3E710202CB9FFF751FDC0F304202860C4
:107A80009BE7FFF74BFD2B6820F4F8521B0203F431
:107A9000F8531A4310210020FFF7DAFD00248CE789
:107AA00010202CB9FFF73AFD00F01F00286084E792
:107AB000FFF734FD2B6820F01F0203F01F031A4369
:107AC00010210020FFF7C4FD002476E7002840F0D5
:107AD00015843520FFF722FD10F0020F0CBF0123A3
:107AE00000232B6069E7002840F00B843520FFF766
:107AF00015FDC04300F0010028605EE734202CB97A
:107B0000FFF70CFDC0F34000286056E7FFF706FDC5
:107B10002B6820F002025B0003F002031A433421B9
:107B20000020FFF795FD002447E7FFF7F7FC2B68DF
:107B300020F0010203F001031A4334210020FFF773
:107B400087FD002439E720B93420FFF7E7FC2860DF
:107B500033E7126834210020FFF77AFD00242CE778
:107B600020B92420FFF7DAFC286026E712682421D8
:107B70000020FFF76DFD00241FE71268252100207B
:107B8000FFF766FD002418E720B92820FFF7C6FCA0
:107B9000286012E7126828210020FFF759FD002411
:107BA0000BE720B92A20FFF7B9FC286005E7126827
:107BB0002A210020FFF74CFD0024FEE620B92320F7
:107BC000FFF7ACFC2860F8E6126823210020FFF7DD
:107BD0003FFD0024F1E612682B210020FFF738FD5D
:107BE0000024EAE620B92C20FFF798FC2860E4E6A0
:107BF00012682C210020FFF72BFD0024DDE600BFDA
:107C0000FFFF0F0014370020BB4E78B91520FFF797
:107C100085FC48B14FF08073B3FBF0F0B04288BFF1
:107C2000304628600024C8E6B348FAE713686BB111
:107C30004FF0807292FBF3F2B242A8BF32462A6044
:107C400015210020FFF704FD0024B6E6AA4AF6E756
:107C5000126833210020FFF7FBFC0024ADE66C2006
:107C60002CB9FFF75BFCC0F3C0402860A5E6FFF726
:107C700055FC2B6820F40022DB0403F400231A4394
:107C80006C210020FFF7E4FC002496E66C202CB960
:107C9000FFF744FCC0F3804028608EE6FFF73EFC0F
:107CA0002B6820F480229B0403F480231A436C2168
:107CB0000020FFF7CDFC00247FE6002840F024835D
:107CC0008E4B1B68136078E60020FFF727FC00212D
:107CD0002B6820F0010203F001031A430846FFF766
:107CE000B7FC002469E628B9FFF718FCC0F3400090
:107CF000286062E60020FFF711FC00212B6820F0CD
:107D000002025B0003F002031A430846FFF7A0FCDF
:107D1000002452E650B96C20FFF700FC4FF480734A
:107D2000C0F3036043FA00F0286046E61368102BA6
:107D300027D00DDC022B20D004DC012B16D04FF015
:107D4000FF3314E0042B1AD0082BF8D105230EE0E2
:107D5000402B18D003DC202BF1D1032307E0802B2C
:107D600013D0B3F5807FEAD1002300E008232B6015
:107D70002B6801330BD110241FE60723F7E70623F6
:107D8000F5E70423F3E70223F1E70123EFE76C2093
:107D9000FFF7C4FB2B6820F070621B0603F07063D2
:107DA0001A436C210020FFF753FC002405E6FFF77F
:107DB000B5FB2B6820F4C032DB0303F4C0331A4355
:107DC0006C210020FFF744FC0024F6E56C202CB960
:107DD000FFF7A4FBC0F380302860EEE5FFF79EFBC1
:107DE0002B6820F480429B0303F480431A436C21E8
:107DF0000020FFF72DFC0024DFE56C202CB9FFF7F5
:107E00008DFBC0F300302860D7E5FFF787FB2B68B8
:107E100020F480521B0303F480531A436C2100208A
:107E2000FFF716FC0024C8E56C20FFF777FB064639
:107E3000C4B910F4804405D0C60906F4F0662E607B
:107E40000024BAE56C20FFF769FB16F00B0F4FEA30
:107E5000201000F0700001D12860F9E540F0080022
:107E60002860AAE56C20FFF759FB10F480444FF01E
:107E70006C000ED0FFF752FB2B6820F4F062DB01A0
:107E800003F4F0631A436C210020FFF7E1FB0024A8
:107E900093E5FFF743FB6C2120F400622046FFF7D7
:107EA000D7FB6C20FFF73AFB2B6820F070021B0118
:107EB00003F070031A436C212046FFF7C9FB7CE5F1
:107EC000C309020503F4F06301D42B60C0E543F05D
:107ED00008032B6071E56C2096B1FFF71FFB2B6840
:107EE00020F070021B0103F070031A436C21002084
:107EF000FFF7AEFB002460E5FFFF0F001437002002
:107F0000FFF70CFB2B6820F4F062DB0103F4F06355
:107F10001A436C213046FFF79BFB34464DE56C203D
:107F20002CB9FFF7FBFA00F00F00286045E5FFF7DA
:107F3000F5FA2B6820F00F0203F00F031A436C21AF
:107F40000020FFF785FB002437E56D202CB9FFF7F3
:107F5000E5FAC0F3C03028602FE5FFF7DFFA2B68A1
:107F600020F40042DB039BB21A436D210020FFF78F
:107F70006FFB002421E5FFF7D1FA2B6820F4C04203
:107F80005B0303F4C0431A436D210020FFF760FB3D
:107F9000002412E56D202CB9FFF7C0FAC0F30320CE
:107FA00028600AE5FFF7BAFA2B6820F470621B021A
:107FB00003F470631A436D210020FFF749FB00248E
:107FC000FBE46D202CB9FFF7A9FAC0F3411028603B
:107FD000F3E4FFF7A3FA2B6820F060025B0103F0E3
:107FE00060031A436D210020FFF732FB0024E4E414
:107FF0006D202CB9FFF792FA00F00F002860DCE446
:10800000FFF78CFA2B6820F00F0203F00F031A43DE
:108010006D210020FFF71CFB0024CEE4FFF77EFA61
:108020002B6820F080721B0603F080731A436D21C9
:108030000020FFF70DFB0024BFE46D2064B9FFF7BB
:108040006DFA001400F07F0310F0400018BF6FF0CD
:108050007F0018432860B0E4FFF760FA2B6820F433
:10806000FE021B0403F4FE031A436D210020FFF7F8
:10807000EFFA0024A1E4002840F049816F20FFF7C7
:108080004DFAC0F30440286097E42C6095E4FFF7B4
:1080900045FA2B6820F48062002B0CBF00234FF4BC
:1080A000806334211A430020FFF7D2FA29689B4BE2
:1080B00069B14FF0807292FBF1F29A42A8BF1A4662
:1080C0002A6014210020FFF7C3FA002475E41A4641
:1080D000F6E7924E68B91420FFF720FA30B14FF05E
:1080E0008073B3FBF0F0864228BF06462E60002462
:1080F00063E413686BB14FF0807292FBF3F2B2420B
:10810000A8BF32462A6014210020FFF7A1FA0024FC
:1081100053E43246F6E7FFF701FA2B6820F40052E9
:108120005B0303F400531A436C210020FFF790FA1D
:10813000002442E46C202CB9FFF7F0F9C0F303509F
:1081400028603AE4FFF7EAF92B6820F470021B0577
:1081500003F470031A436C210020FFF779FA00241E
:108160002BE46E4E68B91320FFF7D8F930B14FF009
:108170008073B3FBF0F0864228BF06462E600024D1
:108180001BE413686BB14FF0807292FBF3F2B242C2
:10819000A8BF32462A6013210020FFF759FA0024B5
:1081A0000BE43246F6E770202CB9FFF7B7F9C0F3BD
:1081B0000720286001E4FFF7B1F92A6820F47F4026
:1081C000120292B2024370210020FFF741FA002010
:1081D000FFF7A4F900212B6820F004029B0003F0B4
:1081E00004031A430846FFF733FA0024FFF7E5BB00
:1081F000FFF794F92A7820F0FF0002437021002055
:10820000FFF726FA0024FFF7D8BB38B97020FFF734
:1082100085F9C0F301402860FFF7CFBB1368032B3B
:108220003FF6A9AD7020FFF779F92B6820F44032B2
:108230001B0403F440331A4370210020FFF708FAAF
:108240000024FFF7BABB38B97020FFF767F9C0F315
:1082500080402860FFF7B1BB1368012B3FF68BAD60
:108260007020FFF75BF92B6820F480229B0403F455
:1082700080231A4370210020FFF7EAF90024FFF75A
:108280009CBB702034B9FFF749F9C0F30150286056
:10829000FFF793BBFFF742F92B6820F440121B0550
:1082A00003F440131A4370210020FFF7D1F9002492
:1082B000FFF783BB28B93920FFF730F92860FFF7B3
:1082C0007CBB126839210020FFF7C2F90024FFF7B8
:1082D00074BB28B93A20FFF721F92860FFF76DBB7E
:1082E00012683A210020FFF7B3F90024FFF765BBBD
:1082F0000424FFF762BB0424FFF75FBB0424FFF7ED
:108300005CBB0424FFF759BB0424FFF756BB0424CD
:10831000FFF753BB0424FFF750BB00BFFFFF0F0064
:1083200007B5019239B9014601AA0120FFF7FDF90D
:1083300003B05DF804FB0820FAE70B4619B90146C3
:108340001846FFF7F2B908207047044B084693F827
:10835000C5320BB1FFF786B8FEF70EBF1437002009
:1083600038B5554C204609F027F8544BDD686B684A
:1083700003F1E402C4F8A42203F58072C4F89C223D
:1083800003F58E72C4F8A02203F5B872C4F89022E7
:1083900003F5C672C4F8942203F5E272C4F8A82269
:1083A00003F5FE7203F1C800C4F8AC2203F568724D
:1083B00003F56F73C4F8B0322B68C4F8B422DB68DD
:1083C000C4F8980298472B68D4F8A802DB6898474D
:1083D0002B68D4F8AC02DB6898472B68D4F8980275
:1083E0005B6998472B68D4F8A8029B6998472B686B
:1083F000D4F8AC025B6998472B68D4F8A4021B69D7
:1084000098472B68D4F8A0021B6998472B68D4F8CA
:108410009C021B6998472B68D4F8B0021B699847E7
:108420002B68D4F8B4021B6998472B68D4F89002E3
:108430001B6998472B68D4F894021B69984794F8F5
:10844000C502FEF70FFF1E4B1E495A690020C2F8F5
:1084500004121D495070C2F808120121C4F8B82254
:1084600011701A4A19741A62194A3221DA61194ACA
:1084700002209A61184A5A62184A9A63184A5A6343
:10848000184A9A62184ADA62184A9A64184A5A6470
:10849000184A5A65184A1A65184ADA64184A1A6658
:1084A000184ADA654FF42572C3E90221164A9A6523
:1084B000BDE83840FEF7B4BE1437002070860208CD
:1084C000006100202D75010869710108DB76010843
:1084D0002977010825770108217701083B830108E6
:1084E0002183010873760108C17601086D760108C1
:1084F0006575010855710108B17201089D70010888
:1085000021720108B1700108BD70010818B9034B50
:108510005B680B6070470820704700BFE839002097
:108520000022014B5A607047006100200428F8B512
:108530000C46154670D005D8022845D056D8C8B18B
:10854000042430E0062800F09480C0F08680FC28E7
:10855000F6D14E4B4E4EDF6814683B68D6F8A00249
:10856000002C00F08E80DB6898473B68D6F8A002AC
:108570009B6916E0126832F0030340F08480434B9D
:10858000434EDF68D207D6F894023B680DD51B69CD
:1085900098472C683B6814F00204D6F890020BD080
:1085A0001B69984700242046F8BDDB6898473B6864
:1085B000D6F894029B69EBE7DB6898473B68D6F8EE
:1085C00090029B699847EEE7304B1468DE68D6E965
:1085D000003000F506703CB1DB689847D6E9003002
:1085E0009B6900F50670DCE79B68EBE7284BD3F846
:1085F000A802264BDB681B6839B1146814F001042B
:1086000001D05B69CDE79B69DCE75B6A9847003086
:1086100018BF01202860C6E71C4B1D4EDF68146898
:108620003B68D6F8A0024CB1012C11D01B699847C9
:108630003B68D6F8A0025B6A984707E0DB6898477A
:108640003B689B69D6F8A002984720462860A9E7B6
:10865000DB6898473B685B69F4E70C4B0C4ADB68C6
:10866000D2F8B0021B685B6A9847003018BF01203F
:10867000ECE7064B064ADB68D2F8B4021B685B6A7B
:10868000F2E71B699EE710248DE700BF70860208A1
:10869000E8390020234B70B5DD68234C2B68D4F8F3
:1086A00098029B6998472B68D4F8A8029B69984761
:1086B0002B68D4F8AC029B6998472B68D4F89C02CD
:1086C0009B6898472B68D4F8A0029B6898472B6852
:1086D000D4F8A4029B6898472B68D4F890029B6852
:1086E00098472B68D4F894029B6898472B68D4F875
:1086F000B0029B6898472B68D4F8B4029B689847EF
:108700002B68D4F898029B6898472B68D4F8A80285
:108710009B6898472B68D4F8AC029B68BDE8704012
:10872000184700BF70860208E8390020014601485A
:1087300008F040BFE839002010B50348144608F09F
:10874000F6FE206010BD00BFE8390020014808F0A7
:10875000E0BE00BFE839002008B50348D0F8B822D1
:1087600008F0E6FF002008BDE839002008B50348FE
:10877000D0F8B82208F0C8FF002008BDE839002072
:1087800008B5024808F0BDFF002008BDE839002008
:1087900008B5024808F0B2FF002008BDE839002003
:1087A00008B5024808F0A8FF002008BDE8390020FD
:1087B00008B5024808F08CFF002008BDE839002009
:1087C000014808F06CBF00BFE839002038B522210D
:1087D0000A4808F0ACFE094C10B9204608F04AFFE0
:1087E000074BD4F89002DD682B681B6998472B680B
:1087F000D4F894021B699847012038BDE83900205D
:1088000070860208022804BF0C4B93F8E80038B9C0
:108810000B4BDB681B685B690A4AD2F89802184761
:10882000012809D1054B93F8E830012B04D1044B02
:10883000DB681B689B69EFE7704700BF00610020A1
:1088400070860208E8390020222970B504461546D2
:1088500000F0FC8200F28E800E2900F01C8241D8CC
:10886000062900F0A98119D8022900F05E8107D8F5
:10887000002900F03D81012900F0498104243DE1F7
:10888000042900F0728140F26181002840F08D815E
:108890002621B94808F04BFE28602FE10A2900F094
:1088A000BA810FD8072900F09F810829E6D1002856
:1088B00040F0F9853521B04808F039FEC0F340207A
:1088C00028601BE10C2900F0C08140F2B281342104
:1088D000A948002C40F0D18108F029FE00F00100E9
:1088E00028600BE1152900F02A821FD8112900F019
:1088F000F5810DD80F2900F0DC811029BED10028A8
:1089000040F0E58125219C4808F011FE2860F5E043
:10891000132900F0FF8140F2EF81002840F0088227
:108920002B21954808F003FE2860E7E01B2900F0A2
:1089300041820DD8172900F0108218299ED10028F5
:1089400040F0318233218C4808F0F1FD2860D5E0F9
:108950001D2900F05F82C0F0458221298ED10028B8
:1089600040F064820146844808F0E1FD00F0010017
:108970002860C3E0AE2900F0238453D8A72900F073
:108980008A832AD8A32900F0D98210D88C2900F034
:108990007782A2297FF472AF6C217748002C40F0D7
:1089A000BE8208F0C4FDC0F3C1302860A6E0A5294E
:1089B00000F0F48240F2DA826C216F4808F0B7FDD3
:1089C00000F48046002C40F04583002E00F03783F1
:1089D000000900F07000286090E0AA2900F09A8356
:1089E00010D8A82900F06E83A9297FF447AF6D2124
:1089F0006148002C40F07D8308F099FDC0F34130C0
:108A000028607BE0AC2900F0B58340F29B836D21A8
:108A10005948002C40F0C58308F089FDC0F3006080
:108A200028606BE0BB2900F0888436D8B62900F0B6
:108A300015841FD8B42900F0E283B5297FF41EAF56
:108A400034214D48002C40F0E78308F070FD4305C9
:108A500040F1E0831421484808F069FD474B30B1EC
:108A60004FF08072B2FBF0F0834228BF03462B60C8
:108A7000002443E0B92900F0238400F23984B829A6
:108A80007FF4FCAE6C213C48002C40F00A8408F0D6
:108A90004EFDC0F34030286030E0CC2900F0C684A1
:108AA00012D8BF2900F07E84C02900F09B84BC2925
:108AB0007FF4E4AE70213048002C40F0668408F06A
:108AC00036FDC0B2286019E0D12900F0C984D2294E
:108AD00000F0D684CE297FF4D1AE002840F0F28495
:108AE0006F21254808F023FDC0F30900286005E048
:108AF00030B92D21204808F01AFD2860204670BDAD
:108B000012682D211C4808F004FD0024F6E728B95E
:108B10002121194808F00BFD2860EFE71268212198
:108B2000154808F0F6FC0024E8E728B92721124888
:108B300008F0FDFC2860E1E712682721002AB8BF91
:108B400052420D4808F0E5FC0024D7E7002840F029
:108B5000A7842221084808F0EAFC10F4000318BF9B
:108B60004FF07F4318432860C8E7034E40B9D6F85A
:108B7000B8321360C2E700BFE8390020FFFF0F00E2
:108B800013682021002BB8BF5B42A648C6F8B83254
:108B900008F0CDFC044608B10024AFE7D6F8B822AF
:108BA0002721A04808F0B5FCA8E7126826219D48B7
:108BB00008F0AFFC0024A1E710219A482CB908F076
:108BC000B6FCC0F30420286098E708F0B0FC2B68DE
:108BD00020F4F8521B0203F4F8531A431021914871
:108BE00008F097FC002489E710218E482CB908F082
:108BF0009EFC00F01F00286080E708F098FC2B68BE
:108C000020F01F0203F01F031A431021854808F0CB
:108C100080FC002472E7002840F048843521814818
:108C200008F085FC10F0020F0CBF012300232B601D
:108C300064E7002840F03D8435217A4808F077FC4D
:108C4000C04300F00100286058E7342175482CB972
:108C500008F06DFCC0F3400028604FE708F067FCA7
:108C60002B6820F002025B0003F002031A43342158
:108C70006C4808F04EFC002440E708F058FC2B68D4
:108C800020F0010203F001031A433421654808F083
:108C900040FC002432E728B93421624808F047FC40
:108CA00028602BE7126834215E4808F032FC00246B
:108CB00024E728B924215B4808F039FC28601DE727
:108CC00012682421574808F024FC002416E7126893
:108CD0002521544808F01DFC00240FE728B928215D
:108CE000504808F024FC286008E7126828214D4805
:108CF00008F00FFC002401E728B92A21494808F0B0
:108D000016FC2860FAE612682A21464808F001FCA1
:108D10000024F3E628B92321424808F008FC286023
:108D2000ECE6126823213F4808F0F3FB0024E5E657
:108D300012682B213B4808F0ECFB0024DEE628B942
:108D40002C21384808F0F3FB2860D7E612682C2164
:108D5000344808F0DEFB0024D0E688B915213148FC
:108D600008F0E5FB50B14FF08073B3FBF0F02E4BF1
:108D7000984228BF184628600024BFE62A48FAE730
:108D8000136873B14FF0807292FBF3F2264B9A4254
:108D9000A8BF1A462A601521224808F0BAFB002411
:108DA000ACE6214AF6E7126833211E4808F0B1FB11
:108DB0000024A3E66C211B482CB908F0B8FBC0F3D3
:108DC000C04028609AE608F0B2FB2B6820F400222D
:108DD000DB0403F400231A436C21124808F099FBCA
:108DE00000248BE66C210F482CB908F0A0FBC0F3DF
:108DF0008040286082E608F09AFB2B6820F48022ED
:108E00009B0403F480231A436C21064808F081FB7D
:108E1000002473E6002840F04F83024B5B68136028
:108E20006CE600BFE8390020FFFF0F000021B848C2
:108E300008F07DFB2B6820F0010203F001031A43C8
:108E40000021B34808F065FB002457E638B9014615
:108E5000AF4808F06CFBC0F3400028604EE60021EC
:108E6000AB4808F064FB2B6820F002025B0003F0C3
:108E700002031A430021A64808F04BFB00243DE6FC
:108E800058B96C21A24808F052FB4FF48073C0F32C
:108E9000036043FA00F0286030E61368102B27D0F7
:108EA0000DDC022B20D004DC012B16D04FF0FF3359
:108EB00014E0042B1AD0082BF8D105230EE0402B28
:108EC00018D003DC202BF1D1032307E0802B13D033
:108ED000B3F5807FEAD1002300E008232B602B68E4
:108EE00001330BD1102409E60723F7E70623F5E742
:108EF0000423F3E70223F1E70123EFE76C21844821
:108F000008F015FB2B6820F070621B0603F07063FD
:108F10001A436C217E4808F0FCFA0024EEE508F0C4
:108F200006FB2B6820F4C032DB0303F4C0331A4382
:108F30006C21774808F0EDFA0024DFE56C217448D5
:108F40002CB908F0F4FAC0F380302860D6E508F0B8
:108F5000EEFA2B6820F480429B0303F480431A430B
:108F60006C216B4808F0D5FA0024C7E56C216848ED
:108F70002CB908F0DCFAC0F300302860BEE508F038
:108F8000D6FA2B6820F480521B0303F480531A4353
:108F90006C215F4808F0BDFA0024AFE56C215C4805
:108FA00008F0C5FA0646CCB910F4804405D0C609CD
:108FB00006F4F0662E600024A0E56C21544808F009
:108FC000B6FA16F00B0F4FEA201000F0700001D136
:108FD0002860E1E540F0080028608FE56C214C48EE
:108FE00008F0A5FA10F480444FF06C0148480ED008
:108FF00008F09DFA2B6820F4F062DB0103F4F063C3
:109000001A436C21424808F084FA002476E508F0FF
:109010008EFA6C2120F400623D4808F07AFA6C2147
:109020003B4808F084FA2B6820F070021B0103F023
:1090300070031A436C21364808F06BFA5EE5C309E9
:10904000020503F4F06301D42B60A5E543F00803A7
:109050002B6053E56C212E4876B108F068FA2B6836
:1090600020F070021B0103F070031A436C212848A2
:1090700008F04FFA002441E508F059FA2B6820F473
:10908000F062DB0103F4F0631A436C21204808F01E
:1090900040FA344632E56C211D482CB908F047FAF5
:1090A00000F00F00286029E508F041FA2B6820F055
:1090B0000F0203F00F031A436C21154808F029FA38
:1090C00000241BE56D2112482CB908F030FAC0F3DA
:1090D000C030286012E508F02AFA2B6820F400421C
:1090E000DB039BB21A436D21094808F012FA0024F1
:1090F00004E508F01CFA2B6820F4C0425B0303F47B
:10910000C0431A436D21024808F003FA0024F5E435
:10911000E83900206D21B8482CB908F008FAC0F3EE
:1091200003202860EAE408F002FA2B6820F4706259
:109130001B0203F470631A436D21AF4808F0E9F98C
:109140000024DBE46D21AC482CB908F0F0F9C0F341
:1091500041102860D2E408F0EAF92B6820F06002A0
:109160005B0103F060031A436D21A34808F0D1F9B5
:109170000024C3E46D21A0482CB908F0D8F900F010
:109180000F002860BAE408F0D2F92B6820F00F0233
:1091900003F00F031A436D21974808F0BAF9002431
:1091A000ACE408F0C4F92B6820F080721B0603F0D1
:1091B00080731A436D21904808F0ABF900249DE4B8
:1091C0006D218D4864B908F0B2F9001400F07F03F6
:1091D00010F0400018BF6FF07F00184328608DE446
:1091E00008F0A5F92B6820F4FE021B0403F4FE032B
:1091F0001A436D21804808F08CF900247EE4002891
:1092000040F05D816F217C4808F091F9C0F3044083
:10921000286073E42C6071E408F089F92B6820F46D
:109220008062002B0CBF00234FF4806334211A436B
:10923000714808F06EF92968704B69B14FF080727F
:1092400092FBF1F29A42A8BF1A462A6014216A489A
:1092500008F05FF9002451E41A46F6E7674E70B94A
:109260001421654808F063F930B14FF08073B3FB07
:10927000F0F0864228BF06462E6000243EE41368C4
:109280006BB14FF0807292FBF3F2B242A8BF32464C
:109290002A601421584808F03CF900242EE4324694
:1092A000F6E708F044F92B6820F400525B0303F45E
:1092B00000531A436C21504808F02BF900241DE498
:1092C0006C214D482CB908F032F9C0F303502860E6
:1092D00014E408F02CF92B6820F470021B0503F449
:1092E00070031A436C21444808F013F9002405E484
:1092F000424E78B91321404808F019F930B14FF0C7
:109300008073B3FBF0F0864228BF06462E6000242F
:10931000FFF7F4BB136873B14FF0807292FBF3F266
:10932000B242A8BF32462A601321334808F0F1F850
:109330000024FFF7E3BB3246F5E770212E4834B92D
:1093400008F0F5F8C0F307202860FFF7D7BB08F056
:10935000EEF82A6820F47F40120292B20243702194
:10936000254808F0D6F80021234808F0E0F82B68DB
:1093700020F004029B0003F004031A4300211E485E
:1093800008F0C7F80024FFF7B9BB08F0D0F82A7836
:1093900020F0FF0002437021174808F0BAF80024BB
:1093A000FFF7ACBB40B97021134808F0C0F8C0F318
:1093B00001402860FFF7A2BB1368032B3FF692AD74
:1093C00070210D4808F0B3F82B6820F440321B04DC
:1093D00003F440331A437021074808F09AF8002438
:1093E000FFF78CBB60B97021034808F0A0F8C0F308
:1093F00080402860FFF782BBE8390020FFFF0F00A4
:109400001368012B3FF66EAD7021304808F08FF8DD
:109410002B6820F480229B0403F480231A437021DC
:109420002A4808F076F80024FFF768BB7021274827
:1094300034B908F07CF8C0F301502860FFF75EBB38
:1094400008F075F82B6820F440121B0503F4401354
:109450001A4370211D4808F05CF80024FFF74EBB4A
:1094600030B93921194808F062F82860FFF746BB87
:1094700012683921154808F04CF80024FFF73EBB6C
:1094800030B93A21114808F052F82860FFF736BB8E
:1094900012683A210D4808F03CF80024FFF72EBB73
:1094A0000424FFF72BBB0424FFF728BB0424FFF799
:1094B00025BB0424FFF722BB0424FFF71FBB0424B1
:1094C000FFF71CBB0424FFF719BB00BFE8390020DD
:1094D00007B5019239B9014601AA0120FFF7B4F995
:1094E00003B05DF804FB0820FAE7012910B5044633
:1094F0000FD1084A092108F00CF82046064A0A2133
:1095000008F007F82046BDE81040044A702108F032
:1095100000B810BD0C0C0100000208001E000CC4B5
:109520000B4619B901461846FFF78EB90820704757
:10953000034B0846D3F8BC321146DB68184700BF1E
:10954000E8390020F8B55C4C5C4D5D4B6A692046FB
:109550005C4F002108F010F85B49204608F0B4F891
:10956000FE68736803F1E402C4F8A42203F5807274
:10957000C4F89C2203F58E72C4F8A02203F5B872D9
:10958000C4F8902203F5C672C4F8942203F5E2727F
:10959000C4F8A82203F5FE7203F1C800C4F8AC2297
:1095A00003F5687203F56F73C4F8B0323368C4F81A
:1095B000B422DB68C4F8980298473368D4F8A8024C
:1095C000DB6898473368D4F8AC02DB6898473368A7
:1095D000D4F898025B6998473368D4F8A8029B696D
:1095E00098473368D4F8AC025B6998473368D4F87D
:1095F000A4021B6998473368D4F8A0021B699847F6
:109600003368D4F89C021B6998473368D4F8B002D9
:109610001B6998473368D4F8B4021B6998473368CC
:10962000D4F890021B6998473368D4F894021B69F8
:10963000984773683A6903F537735360C4F8BC22DE
:109640006B69224A0021C3F80422214A5970C3F8E9
:10965000082201221A701F4B2A742B621E4B3222E1
:10966000EB611E4B0220AB611D4B6B621D4BAB636C
:109670001D4B6B631D4BAB621D4BEB621D4BAB6413
:109680001D4B6B641D4B6B651D4B2B651D4BEB64BC
:109690001D4B2B661D4BEB654FF42573C5E902325C
:1096A0001B4BAB652368D3F8A030C4F8B832BDE8D3
:1096B000F840FFF7A7B800BFE8390020006100209C
:1096C0006884020870860208EB940108CD870108BF
:1096D000C1870108B1870108A187010891870108A6
:1096E0008187010821950108D19401086D8701083F
:1096F000598701084D870108398701082D8701081E
:109700002D8501080D8501080588010821850108BE
:1097100095860108002814BF082000207047002803
:1097200014BF082000207047002814BF0820002024
:109730007047002914BF082004207047002914BF77
:1097400008200420704770470022014B9A67704739
:10975000006100200020704770477047002008F02B
:1097600019B8002208B51046114608F013F8012078
:1097700008BDF6E710B50020144607F0E9FF2060A9
:1097800010BD002814BF082000207047002814BF17
:10979000082000207047002814BF082000207047D0
:1097A000002814BF08200020704710B40C4630B9C0
:1097B000044B20461B6811469B6810BC18470020CC
:1097C00010BC704784670020294B2A491A69DB685E
:1097D00002F114005B68086003F50D739361264B7A
:1097E000264AD3F888100120C1F80422244A0870C0
:1097F000C1F8082200224A70224983F88400C3F885
:10980000941021493220C3F890102049C3F88C10DD
:109810001F49C3F898101F49C3F8AC101E49C3F87C
:10982000A8101E49C3F89C101D49C3F8A0101D497B
:10983000C3F8BC101C49C3F8B8101C49C3F8C810C1
:109840001B49C3F8C4101B49C3F8C0101A49C3F818
:10985000D4101A49C3F8D0104FF42571C3E91F1072
:1098600017491046C3F8CC10114607F093BF00BF4C
:109870007086020884670020006100206397010859
:10988000739701088D9701081597010897970108AC
:109890001F9701083D97010833970108A197010818
:1098A000299701085D9701087597010847970108F6
:1098B00055970108839701085B97010849970108AC
:1098C0005997010870477047704701207047002280
:1098D000014B5A609A6770470061002041EA0021FD
:1098E000D2B2014808F070B89067002010B541EA84
:1098F00000210348144608F032F8206010BD00BF74
:109900009067002070B40C4BFF28D6B2C2F3072535
:10991000C2F307444FEA126209BFDA71DA701E71AE
:109920005D710FBF9C711E705D709C700901024AD1
:10993000024870BC08F00EB9B43C002090670020CB
:10994000012838B5144616D004D3022855D0042077
:10995000106018E052224121484808F035F84522AD
:109960004121464808F030F853224121434808F08D
:109970002BF8002007E04FF4A061404807F0E1FF1A
:10998000C20701D4402038BD40F201513B4807F0E6
:10999000D8FF40F00102D2B240F20151374808F03E
:1099A00013F8364D40F20251284607F0D8FF030461
:1099B000F8D4226840F20451304808F01EF840F212
:1099C00002512E4807F0CBFF4FF6FF02024042F44F
:1099D000807240F20251294808F001F8274D40F208
:1099E0000251284607F0BBFF0004F8D44FF4A161F0
:1099F000224807F0C3FF2060BBE74FF4A0611F4877
:109A0000146807F09EFFC107BCD540F201511B4806
:109A100007F097FF40F00102D2B240F2015117481F
:109A200007F0D2FF154D40F20251284607F097FF8C
:109A30000204F8D4220C40F20451104807F0DDFF74
:109A4000A2B24FF4A1610D4807F0D7FF40F20251D6
:109A50000A4807F084FF4FF6FF02024042F400720A
:109A600040F20251054807F0BAFF044C40F202519F
:109A7000204607F074FF0304F8D47AE790670020CB
:109A800070B50646084C0901154601F0F00104F1D5
:109A90000802064807F0FCFF0EB1FF2E01D0A368B4
:109AA00000E0E3682B6070BDB43C002090670020AC
:109AB000012070470B46114618B1012806D000203E
:109AC0007047034A1268184692681047014AF9E73E
:109AD00098670020886700201B4B1C491A69DB68C7
:109AE00002F114005B68086003F50D739361184B75
:109AF0001849D3F888201848C2F804121749C2F848
:109B0000081200215170117083F88410C3F880107E
:109B10004FF0FF31C3F8BC001148D967C3F8B80053
:109B200010485969C3F8C8000F48C3F8C4000F486B
:109B3000C3F8D4000E48C3F8D0000E48C3F8CC00D8
:109B40000D4808F01BB800BF708602088867002027
:109B500000610020CB980108DD980108B19A010846
:109B6000ED980108C598010841990108C7980108B6
:109B7000CF980108C99801089067002070B51B4D67
:109B80001B4EEC6860682368C8303060DB6898471B
:109B9000236830685B6998472A69164B1A606368C6
:109BA00003F537735360144B144A5969C1F8042202
:109BB000134AC1F8082200224A700A701A74DA6047
:109BC0004FF0FF32BDE870400E499A6099640E492B
:109BD00059640E4959650E4919650E4919660E49B1
:109BE000D9650E499965FFF777BF00BF70860208F7
:109BF0008C6700209867002000610020CB98010846
